:020000040800F2
:1000000000000220ADA1000895A1000895A10008FC
:1000100095A1000895A1000895A100080000000026
:1000200000000000000000000000000095A1000892
:1000300095A100080000000095A100089DA10008FE
:1000400095A1000895A1000895A1000895A10008B8
:1000500095A1000895A1000895A1000895A10008A8
:1000600095A1000895A1000895A10008891E000827
:1000700095A1000895A1000895A1000895A1000888
:1000800095A1000895A100086D0D000895A1000834
:1000900095A1000895A1000895A1000895A1000868
:1000A00095A1000895A1000895A1000895A1000858
:1000B000051000082910000895A10008391400084F
:1000C000091C000895A1000895A1000895A1000849
:1000D000550F0008DD13000895A1000895A1000840
:1000E00095A1000895A1000895A1000895A1000818
:1000F00095A1000895A1000895A10008951E00088B
:1001000095A1000895A1000895A1000895A10008F7
:1001100095A1000895A1000895A1000895A10008E7
:1001200095A1000895A1000895A1000895A10008D7
:1001300095A10008000000000000000095A1000843
:1001400095A1000895A1000895A1000895A10008B7
:100150002D14000895A100082114000895A100089D
:1001600095A1000895A1000895A1000895A1000897
:1001700095A1000895A1000895A1000800000000C5
:100180000000000095A10008000000000000000031
:1001900095A10008000000000000000095A10008E3
:1001A00000000000000000000000000095A1000811
:1001B00095A1000895A1000895A1000895A1000847
:0401C00095A10008FD
:10020000BFF34F8F0549064BCA6802F4E06040EA2D
:100210000302CA60BFF34F8F00BFFDE700ED00E0AF
:100220000400FA0500B5154BDB68C3F30223A3F104
:10023000030EBEF1040F94BFC3F1070304234FF074
:10024000FF3C88BF4FF0000E0CFA03F321EA0301D4
:100250000CFA0EF322EA030201FA0EF11143431CD9
:100260004FEA011106D000F1604000F5614C8CF8B6
:10027000001300BD014B83F8231000BD00ED00E02A
:1002800010B54A490268D1F800C002234FF0000EB1
:1002900080F8353080F834E0146824F001031360EE
:1002A000026804E00B68A3EB0C04052C4FD814681B
:1002B000E407F7D4D0E902414368D2F800C02343F1
:1002C0000B43D0E90441234384690B43C1692343B1
:1002D0000B43374C016A0B430CEA0401446A042CBB
:1002E00043EA010339D013600168426A4B69042A6A
:1002F00023F0070444EA02040BD1826AD0F818C044
:100300001443BCF1000F2DD1012A49D0022A30D06C
:100310007AB34C610368DFF89CC0DAB2A2F1100432
:100320006FF3090318215F2CB4FBF1F21CF80210E3
:10033000C16588BF04333F248C404FF0000C01227C
:1003400083659C60C0F854C080F8352010BD202122
:100350000322416580F8352010BDD0E90B142143FC
:100360000B43C0E7BCF5005F0CD0022A04D9032A76
:10037000CFD1C26AD201CCD540210124416580F899
:10038000354010BD032AC4D80FF2040C5CF822F0EB
:10039000790300087303000879030008A10300082B
:1003A000C36AB3F1C07FB4D1E6E700BF48000120C3
:1003B0003F8010F024A7000890F834C0BCF1010F72
:1003C00044D030B590F83540856D4FF0010E74453E
:1003D00080F834E003D0002380F8343030BDD0F80A
:1003E00000E002244FF0000C80F83540C0F854C003
:1003F000DEF800C02CF4802CCEF800C004686360E6
:1004000084680368402C1DD099600168CA60C46D7F
:100410003F23A340AB6001680A6842F016040C60F9
:1004200005686B6943F080016961026C22B1046860
:10043000256845F0080323600068016841F0010267
:10044000026030BD9A600268D160E0E7704700BF8B
:1004500070B584B00023846D74490393C36D226822
:100460000E68082505FA03F1114207D0D0F800C044
:10047000DCF800E01EF0040F40F0A8806C499940C1
:10048000114206D00568D5F814C01CF0800F40F06A
:10049000968068499940114206D00568D5F800C099
:1004A0001CF0020F40F0848010219940114205D0C9
:1004B0000568D5F800C01CF0080F63D1202505FAA7
:1004C00003F1114216D003681A68D50612D5A1604F
:1004D00090F835500368052D196834D04C0340F16D
:1004E0008C801968090340F19780C46B14B10090A7
:1004F000A0470098426D002A42D0456DEA071CD5FE
:1005000001684D4C4FF0050C80F835C00B68A4FB1A
:10051000064623F00105B20A0D6003E003681C687B
:10052000E30704D50399013191420391F6D90025DF
:10053000012680F8345080F83560C36C03B304B0F2
:10054000BDE87040184721F016021A6001684D6935
:1005500025F080064E61036C002B62D001680D68A7
:1005600025F008060E60C26D3F239340A360036D23
:100570000024012180F8344080F83510002BDED1B2
:1005800004B070BDA1600368196849032DD41D68CB
:10059000E90503D4196821F008051D60016C0029E4
:1005A00029D0CDE9000288470098019AC36D85E7FC
:1005B000A160436D43F004014165C36D74E7A16020
:1005C000436D43F002014165C36D62E7DCF8003022
:1005D00023F00401CCF80010C36D9D40A560456D6B
:1005E000C36D45F00101416548E71B681D03D5D582
:1005F000816C0029D5D1C36D60E71C6814F4807C40
:100600007FF473AF1A6822F010051D60012380F893
:1006100034C080F8353068E7446C002C7FF467AF55
:1006200068E7826C002A99D19DE700BF0000002096
:100630000100800004008000B5814E1B2DE9F04FC1
:100640000023694DDFF8ACE183B001244FF00309CA
:1006500003E00133102B00F0B9800F6804FA03F2B5
:1006600002EA070A32EA0707F3D14F6827F01006BB
:10067000022E14D1DF0800EB870803F007064FEACB
:10068000860CD8F820B00F690F2606FA0CF607FA88
:100690000CF72BEA06063743C8F820704F68D0F8ED
:1006A00000B007F003064FEA430C06FA0CF709FA0C
:1006B0000CF62BEA060847EA080707604F6827F0A0
:1006C000100B0BF1FF37012F12D8876827EA0608B5
:1006D000CF6807FA0CFB4BEA080787604F68D0F831
:1006E0000480C7F300179F4028EA020217434760BF
:1006F000C7688A6827EA060602FA0CF73743C7601C
:100700004E68F700A5D5002201926F6C47F4804631
:100710006E646A6C23F0030C02F4804701970CF1BD
:10072000804B019A0BF59C3203F0030697684FEA61
:10073000860C4FF00F0808FA0CF627EA06072B4E36
:10074000B04211D006F5806B584542D0284EB042D9
:1007500044D0DFF8A48040450CBF4FF003084FF0B1
:10076000080808FA0CF6374397604E68DEF8002058
:10077000F60354BF22EA0A024AEA0202CEF8002037
:100780004F68DEF80460BF0354BF26EA0A064AEA4F
:100790000606CEF804604F68DEF80820FE0254BF5B
:1007A00022EA0A024AEA0202CEF808204E68DEF87F
:1007B0000C70B20203F1010354BF27EA0A074AEAA8
:1007C0000707102BCEF80C707FF447AF03B0BDE8DD
:1007D000F08F012606FA0CF63743C5E7022606FA23
:1007E0000CF63743C0E700BF00380240000002406B
:1007F00000080240003C0140000C024003681968F8
:1008000011F4807C0CD1826B1068A2F826C0436979
:1008100023F0800141611268D06840F04003D3604A
:10082000704700BF704700BF0368196811F4807CEF
:1008300015D1826B1068A2F82EC0C36823F48071B2
:10084000C1601168486920F001034B611168486973
:100850004FF0200C20F040034B6182F83AC0704703
:10086000704700BF836B1A68506993F839102129CB
:1008700009D0506993F83A10222916D0D96B41F06B
:100880001002DA6370470006F3D50020D884D168DF
:1008900021F0C000D0601A684FF0200C83F839C0F6
:1008A000506993F83A102229E8D14106E6D5002094
:1008B000D885D16821F49070D06019684A694FF0EA
:1008C000200C22F00100486183F83AC0D96B41F056
:1008D0001002DA63704700BF38B50022184CDFF809
:1008E00064E00B461546014663F30F02012063F3F3
:1008F0001F4284F83C00606B2564C4E909124FF084
:10090000210C626884F83DC0C0F83CE0DFF838C0D4
:10091000DFF838E00565C0F840C0C0F84CE00432AC
:10092000FFF74AFD63686FF040011960626884F860
:100930003C505469284644F08005556138BD00BFDD
:1009400048000120FD070008250800086508000888
:100950000D4B0E4A1868A2FB00218B09013BB3F135
:10096000807F0BD24FF0E022094853614FF0F00C2A
:100970000021072380F823C09161136100220F2119
:100980004FF0FF304EE400BF00000020D34D621056
:1009900000ED00E030B5DFF85CE01D46030C012BF4
:1009A0001446DEF8442005D110E0DEF80000431BB9
:1009B0009C4215D39069C0F340039942F5D00020C2
:1009C00030BDDEF800305B1B9C4209D3536920EA3E
:1009D00003039BB2B3FA83F35B098B42F1D0EEE7DA
:1009E00000212024CEF874108EF880108EF88140FB
:1009F000032030BD48000120836B93F83D1093F82D
:100A00003E202129C8B2D2B226D0222822D019688D
:100A1000086820F480620A601968086840F400726F
:100A20000A601868426822F480524260186842687E
:100A3000002122F40062426059858C46196C41B94C
:100A4000202083F83D0093F83E2083F83EC0402AE2
:100A500011D07047202ADAD11968486820F4006262
:100A60004A6019684FF0000CA3F82AC04B6843F4A1
:100A70004070486070477047836B1868026822F4C2
:100A80008062026000212020598583F83D0083F8B0
:100A90003E10196C41F010021A647047836B18689D
:100AA000016821F480610160586B00225A8502655B
:100AB000996B0A65944693F83D20202283F83D20E7
:100AC00083F83EC0704700BF30B51B4C0D46D4F8CC
:100AD00044E0114608E0DEF8142012F480630CD1E3
:100AE0002268521A95421FD3DEF8143020EA03021E
:100AF00093B2002BEFD1184630BDDEF8001041F460
:100B00000073CEF80030626C00256FF48060042121
:100B10004FF0200C5061C4F8841084F88050656751
:100B200084F881C0012030BD2020636784F88030C4
:100B300084F88100032030BD4800012030B5224CEC
:100B4000236F042B054683B0606C07D0012B05D0C2
:100B500013F5803F02D0636F122B03D1036843F477
:100B600080730360606C03E023689B1A994220D372
:100B70004369DB07F8D5636DB3F5804F0BD1056191
:100B80001248FFF7A1FF20B1D4F88410042917D12F
:100B9000012003B030BDF02303610D4801920091A4
:100BA000FFF792FFDDE900120028EDD1636C1D61B3
:100BB000E6E700212022616784F8801084F8812014
:100BC000032003B030BD00BF480001200200010037
:100BD000080001001849D1F844C0DCF8143013F0C3
:100BE000800327D1DCF8142012F4806212D10B6844
:100BF0001B1A012BF1D9D1F8840081F880204FF025
:100C0000200C40EA0C03C1F8843003204A6781F8C5
:100C100081C070476FF48062CCF8142004204FF03C
:100C2000200CC1F8840081F880304B67012081F8E6
:100C300081C070470020704748000120DFF858C08D
:100C4000DCF8441008E04A6912F010020AD1DCF81E
:100C500000301B1A012B13D84B6913F04003F2D05C
:100C6000002070476FF0100020224861CCF88430DB
:100C70000120CCF874308CF880308CF881207047DB
:100C8000DCF884008CF8802020210843CCF8840014
:100C90008CF8811003207047480001202E4A036819
:100CA00090422CD0B0F1804F29D02C4A90423DD0B8
:100CB00002F5806C604539D0294A904236D0294AE5
:100CC000904233D0284A904234D002F5806C60457F
:100CD00030D00CF5806290422CD0A2F5983C604553
:100CE00028D00CF58062904224D002F5806C6045DB
:100CF00020D003608B68C3620968816228E010B469
:100D00004C68CA6823F07003234323F440731343F1
:100D100003608A68104CC2620B688362A04201D1F2
:100D200009690163012210BC426170474A6823F0DF
:100D300070031343CA6823F44073134303608A6843
:100D4000C262084B0A688262984204BF0B6903635F
:100D500001214161704700BF0000014000040040D4
:100D6000000C00400004014000400140784AD2F8E5
:100D7000983019685868890701D580065BD41968CE
:100D80005868490701D500061CD419685868C90776
:100D900001D5410607D419685868890602D5410172
:100DA00000F1928070471968C807F4D5D2F8D810BE
:100DB0006FF0010041F48031C2F8D8101860D2F809
:100DC0009830E8E7D2F8D810C90605D4D2F8D80090
:100DD00040F40051C2F8D810986810F4401F24D194
:100DE000996B11F4401F02D0986840051DD45968D2
:100DF00049051AD49968D2F8B00001F04051014376
:100E000013D1586820F080015960D2F8D80020F43E
:100E10008051C2F8D810D2F8D800C00505D4D2F855
:100E2000D81041F00100C2F8D8006FF00C01196031
:100E3000D2F89830A9E7D2F8D810C90605D4D2F86C
:100E4000D80040F40071C2F8D8109968D2F8B00008
:100E500001F04051014344D0D96C44F27C7089B216
:100E600000FB01F1C1F30F3C42F61F308445A2F8AC
:100E7000E0C064D942F62D418C4563D942F6E55075
:100E8000844562D943F2C7218C458CBF4FF0040CD6
:100E90004FF0030C92F8D40082F8E2C001280DD084
:100EA000012182F8D410986820F0010199609868B7
:100EB000C0072FD54FF0000C82F8D4C06FF012019C
:100EC0001960D2F898305AE7D2F8DC106FF02000A1
:100ED00041F00201C2F8DC101860D2F898201060CE
:100EE0007047D86A10F4700F25D1586820F020019F
:100EF0005960D2F8D80020F48071C2F8D810D2F826
:100F0000D800C104A8D4D2F8D81041F00100C2F82A
:100F1000D800A1E7596821F0806020F020015960D5
:100F2000D2F8D80020F4885C2CF0010141F00100D7
:100F3000C2F8D800BEE7996848058DD4D5E74FF0D0
:100F4000000CA7E74FF0010CA4E74FF0020CA1E75B
:100F5000480001200A4B0B4AD3F8E400D3F81C11D7
:100F6000C0680880D3F8E4104B684FF4007C4FF45D
:100F7000806023F040034B60C2F818C09061704756
:100F800048000120000402401B4A02F59E73D2F87B
:100F900000C0D2F8E410C2F81401C2F81C3104E019
:100FA0001368A3EB0C03642B16D88B689B07F7D54B
:100FB00082B00288CA6000200190CB6801938A68E1
:100FC0000192019B486840F040034B600A6842F080
:100FD0004000086002B07047084B4FF400624FF0C9
:100FE000080EC3F818E040209A6180214FF4805227
:100FF000986199619A61FEE7480001200000024073
:10100000704700BF08B54FF080431A69D30708D571
:101010000448416888474FF080431A6922F0010074
:10102000186108BD000000204E4B1869C30700D4AA
:1010300070474D4B93F83E214AB193F83F2162B976
:101040004A494FF480508861013283F83F21454A74
:10105000136923F001011161704793F8E210481CF5
:10106000B2EB400F75DB042973D0122AECD993F848
:10107000D42082B00020012A019060D0D3F89810CB
:101080004FF0010C83F8D4C08A68D00715D43848D3
:10109000DFF8E8C002688868ACFB02C2920C40F03E
:1010A000010002EB420288600192019828B1019A86
:1010B000501E0190019A002AF9D18868C2073ED5D6
:1010C000D3F8D82022F4E06020F0010C4CF48072B8
:1010D000C3F8D8204868400507D5D3F8D82022F4B3
:1010E000405040F48052C3F8D820D3F8D80010F410
:1010F000805218BFD3F8DC204FF0000C18BF22F04C
:1011000006026FF0220083F8D4C0C3F8DC20086028
:10111000D3F8981017484A6842F0806C4CF02002CF
:101120004A604068C20602D0134A914207D18868DB
:1011300010F0405F03D18A6842F080408860094A1D
:10114000002183F83F11136923F00100106102B000
:1011500070470648416981F4805C4CF080518161A0
:1011600083E700BF00040040480001200000024067
:1011700000000020002301400020014083DE1B43CB
:1011800010B51E4CD4F84001C36823F00101C160C2
:10119000036A41F2111213420AD1026A40F2444139
:1011A0000A4205D1036823F001020260D4F840012D
:1011B00013491123C4F84C31FFF770FDD4F84021D6
:1011C000D4F84801136823F070030343D4F85001A6
:1011D00023F4407303431360D4F84031D4F84C0136
:1011E000D4F84441D86201219C625961DA680A430B
:1011F000DA6018680843186010BD00BF480001207D
:101200008C010120724B93F83D20202A01D0002050
:101210007047704A4FF0400C0529C2F818C040F2E0
:10122000D180002800F0CE8010B54FF40474A3F8EC
:101230007C414C1E14F0030C00EB01024FF0020144
:101240003ED010F801EBBEF1100F04D183F87EE11F
:1012500010F801EC03215C18BCF1010F84F87CE16B
:1012600001F101012CD0BCF1020F14D010F8014B98
:10127000102C07D103EB010E01318EF87C4110F8E0
:10128000014C89B201F1010E194481F87C411FFA29
:101290008EF1FC2967D810F8014B102C07D103EB15
:1012A000010E01318EF87C4110F8014C89B201F138
:1012B000010E194481F87C411FFA8EF1FC2952D8A5
:1012C00010F8014B102C07D103EB010E01318EF801
:1012D0007C4110F8014C89B203EB010E82428EF87A
:1012E0007C4101F101041FFA84FC42D0BCF1FC0FE7
:1012F00039D8014611F801EBBEF1100F09D103EB0B
:101300000C0484F87CE111F801EC0CF101041FFAE3
:1013100084FC0CF1010189B29C44FC298CF87CE12D
:1013200021D890F801E0BEF1100F06D15C18013110
:1013300084F87CE190F801E089B24C1C194481F8F2
:101340007CE1A1B2FC290ED890F802E0BEF1100FAA
:1013500000F103002DD00C46611C89B21C44FC290D
:1013600084F87CE1ACD91B484FF4800282610020F4
:1013700010BD8A1C93F83D0013FA82F49C444FF090
:10138000100E032220288CF87CE184F87C210AD1FD
:1013900093F83C30012B06D003310F4889B2FFF798
:1013A0009BFA012000E000200A494FF480048C6180
:1013B00010BD03EB010C01318CF87CE110F801EC5D
:1013C0008CB2C9E7034B4FF4800199611FE700BF5E
:1013D0004800012000080240C40101200F494B6869
:1013E0001A68D86812F0200F02D010F0200F04D134
:1013F000520601D5420607D47047D1F87C12002965
:10140000FAD05B68D8B20847DA684FF0200C22F0B7
:101410004000D86081F83DC0704700BF48000120FF
:101420000148FFF715B800BFC80201200148FFF7C7
:101430000FB800BF28030120F0B5AA4B5A6CD2F8B0
:1014400018E05169D2F804C093F8820010288BB0DC
:101450004FD0C4B2402C4CD0A34D01EA0506002E5B
:1014600000F0C9801CF4007F40F064819F4D0EEABB
:101470000506DFF880E201EA0E0E002E00F0F7808C
:101480009B4F01EA0700002800F071811CF4806F77
:1014900000F06D81BEF1000F40F06D8193F8810086
:1014A000B3F86EC01FFA8CF1C4B201B39D6E05F1A2
:1014B000010CC3F868C02E781661B3F86E70781E00
:1014C000A3F86E00B3F86E108DB285B9292C0ED139
:1014D000546824F480662825566093F8817093F848
:1014E000822007F0030002435A6783F881500BB053
:1014F000F0BD11F0011F30D01CF4007F40F00281DC
:101500007A4D7C4A0EEA050001EA0207002847D01E
:10151000774A01EA0205002D3ED01CF4806F3BD0D3
:10152000002F00F03E811CF4007FE0D01F6F93F885
:101530008140212CDBD1B3F86E10586C8EB2002E96
:1015400000F038829E6E711C996632780261B3F8A1
:101550006E506F1EA3F86E70C9E7674D01EA050073
:10156000002840F0B580604C01EA0406002EC7D088
:101570001CF4007FC4D093F882701E6FFDB25F6FC1
:1015800093F88140222C00F08181019050690190F4
:1015900092690192019AB3E7002FC4D10BB0F0BD5C
:1015A000564C214019B31CF4806F20D0002F00F05E
:1015B00026811CF4007F9AD01E6FB3F86EC05F6C5A
:1015C0001FFA8CF2032A00F0AA81B3F86E50A8B279
:1015D000022800F0B9819C6E3969601C9866217000
:1015E000B3F86EC00CF1FF36A3F86E607FE7002FF2
:1015F000DFD10BB0F0BD424F01EA070000283FF4F5
:1016000035AF1CF4007F3FF431AF93F88110D2F86E
:1016100004C02CF4E06CC2F804C00996D2F814C0DF
:10162000CDF824C0D2F800C04CF0010CC2F800C0C4
:10163000D3F844C0099ADCF80020A1F1280422F470
:101640008065022C5FFA81FECCF8005040F24081A8
:101650005E6F222E03D0BEF1220F7FF448AF002729
:1016600020205F6783F8810083F882703FE7234F73
:1016700001EA0700002860D01CF4806F5DD0BEF145
:10168000000F5ED193F88100B3F86EC01FFA8CF1A1
:10169000C4B200293FF42BAF9D6E126905F1010C15
:1016A000C3F868C02A70B3F86E60771EA3F86E7036
:1016B000B3F86E0081B200297FF419AF2A2C7FF4B1
:1016C00016AF5C6C626822F480662825666004E7C9
:1016D0001CF4007F3FF414AFD3F88840E6B21661E3
:1016E0000EE700BF480001200200010004001000C6
:1016F000800001000400010008000100400001001A
:101700001000010093F88270402F00F0EA805D6DB8
:10171000B5F5804F00F0AD80D3F89400002840F07C
:10172000E980D3F88840E61106F0060747F0F00597
:101730001561E5E693699369D9E6BEF1000F3FF4C0
:10174000D6AE1CF4007F3FF4D2AEB3F86EC01FFAE1
:101750008CF100293FF4CBAE9C6E1269651C9D662E
:101760002270B3F86E60771EA3F86E70BFE6BEF10C
:10177000000F3FF4BCAE1CF4007F3FF4B8AEB3F8EA
:101780006EC01FFA8CF100293FF4B1AE9C6E651C4F
:101790009D6626781661B3F86E20571EA3F86E700A
:1017A000A5E693F88140B3F86C0093F88260D3F813
:1017B00070C0E2B2F1B2002840F0BD80212A00F0F2
:1017C000568140297FF493AE222A7FF490AEB3F87D
:1017D0006E50AFB2002F00F0448193F88240402C4D
:1017E00000F0CB819F6E5C6C781C98663E78266119
:1017F000B3F86EC00CF1FF32A3F86E2077E693F8D1
:101800008170222F7FF473AEB3F86E205F6C95B2B7
:10181000032D3FF6E0AEA81E01281C6F40F2158193
:101820003968022C14BF21F4806141F48061396071
:101830005E6C776827F4E06272609D6E3469681CA4
:1018400098662C70B3F86E104E1EA3F86E6093F875
:10185000817093F8822007F003052A434FF0200C93
:101860005A6783F881C0002493F8822083F882406D
:101870003DE693F88100D3F88840212816BF44F054
:10188000010404F0FE04E4B2146139E6D3F8944094
:1018900014B9402D00F00881D3F8945025B9586D43
:1018A000B0F5404F00F01981B3F86E40A5B2002D9D
:1018B00040F09980069554690694966906960698B4
:1018C000176847F4007515600022C3F8942017E6E6
:1018D0009E49196720245E6783F8814083F88260FF
:1018E00005E6D3F894609EB9D3F8884004F0FE066C
:1018F000166105E6D3F89440012C7FF401AED3F8CD
:101900008860F71107F0060545F0F1001061F7E572
:10191000D3F8887047F00105E8B21061F0E5042EB5
:101920000DD0082E0BD016F5803F08D09C6E5E6C53
:10193000601C316952E6212A7FF443AF47E73C68D7
:1019400024F480613960F1E7042E65D0082E63D05D
:1019500016F5803F60D03A68022E14BF22F48062F0
:1019600042F480623A6093F8817093F8825007F0F5
:10197000030005435D679C6E596C661C0A699E6690
:101980002270B3F86EC09F6E5D6C0CF1FF30A3F84F
:101990006E002C69791C99663C70B3F86E605F6CC0
:1019A000721EA3F86E207D6825F440704FF0200C65
:1019B000786056E7042F36D0082F34D017F5803FD3
:1019C00031D0426822F4E065456093F881C093F815
:1019D00082700CF00300074320245F6783F8826065
:1019E00083F8814083E5B3F86E0084B2012C00F0E7
:1019F0008480B3F86E60B7B2022F00F0A98015683A
:101A000045F4806010605C6C002202926669029668
:101A1000A7690297029A57E712245C67396841F474
:101A200000763E60A7E7426822F4E06747600468FA
:101A30000025202144F4007606605D6783F881105C
:101A400093F8822083F8825051E5022C386800F028
:101A5000A78020F480663E605F6C3A6842F40065BF
:101A60003D605A6C536823F4806151603FE5BCF1DE
:101A7000040F5D6C1FD0BCF1080F1CD01CF5803F1B
:101A800019D06F6827F4E0646C6093F8815093F884
:101A9000826005F0030216434FF0200C5E6783F866
:101AA000820083F881C022E5089450690890926909
:101AB0000892089A24E56F6827F4E06068602E6851
:101AC0000024202246F4007129605C6783F881209D
:101AD00093F8822083F8824009E5079550690790C2
:101AE000946907940798166846F480771760D3F8CE
:101AF00094500135C3F8945002E5042E15D0082EF9
:101B000013D0122F11D01C6F1668022C14BF26F4AC
:101B1000806646F4806616605F6C002205927D69DF
:101B20000595B8690590059ACEE6156825F480609C
:101B300010605C6C0022049266690496A7690497A1
:101B40000498256845F400702060BDE60000FFFFA2
:101B50001D6F1068022D27D020F4806616605F6C20
:101B60003A6842F400653D605C6C00200390666951
:101B70000396A7690397039AA6E6D3F89400B8B929
:101B8000D3F89020596CD3F88C50012A23D0C5F398
:101B900007270F61D3F894400134C3F89440A6E4BA
:101BA00040F4806139605CE740F480641460DBE7F6
:101BB000D3F89460012E16D0D3F89420022A7FF433
:101BC00096AC93F88110222918D093F88150212DDA
:101BD0007FF48DAC06E6E8B20861D3F89460023673
:101BE000C3F8946083E4D3F88C705C6CF8B2206125
:101BF000D3F894600136C3F8946078E4596C0B68AC
:101C000043F480750D6072E410B59B4B9B485A6C91
:101C10005169D2F804C0014201F4813E4CD01CF459
:101C2000807F01F4823443D0D3F884C04CF0010C9F
:101C3000C3F884C06FF4807CC2F814C0BEF1000FFA
:101C400000F09380D3F884C04CF0020CC3F884C039
:101C50006FF4007CC2F814C0002C00F0898093F867
:101C600082E0B3F86E0093F88140BEF1200F5FFA76
:101C700084FC80B25C6F00F08480D3F8844044F030
:101C80000400C3F88400146844F4007010605A6CB7
:101C90006FF4806C11F4843FC2F814C008D0D3F8FC
:101CA00084106FF4006441F00800C3F884005461AC
:101CB000D3F884204AB910BDBEF1000F45D01CF402
:101CC000807FF5D001F48234BCE793F881C0ACF199
:101CD0002901012943D993F88140602C4FF000007D
:101CE0001CBF202483F88140586783F882005C6C15
:101CF000206820F4006121605A6C1468210564D5C5
:101D0000516821F400645460986F002865D090F801
:101D100035205B490165022A63D080234365FEF7C5
:101D2000BDFE554B93F881102829C4D1D3F88440C7
:101D30006207C0D50022534818674FF0200C5A673D
:101D400083F881C083F8822010BD11F4823F13D143
:101D500011F4843FACD01CF4807FA0D1A8E700210F
:101D60002822596783F88120C1E7002C7FF477AFE0
:101D700011F4843F93D19BE71CF4807F7FF46FAF15
:101D800096E700287FF479AF0CF0F700212806D001
:101D9000BCF1280F7FF471AF212C7FF46EAF93F864
:101DA0008140D3F870C0BCF1040FE0B223D0BCF185
:101DB000080F20D0212801F484313BD06FF48064D7
:101DC000546100297FF46BAF72E793F881006028BB
:101DD00004BF202083F88100A4E7D86F002896D1A3
:101DE000A0E704684FF0050C80F835C0206820F0AB
:101DF0000102226096E72828DCD12248186754683F
:101E00006FF4806C24F4E0605060C2F814C0146871
:101E100024F4806010604FF0000C202211F4843F05
:101E2000C3F874C083F8812083F882C03FF440AFC8
:101E30005A6C34E71348186793F8814093F882008E
:101E400004F0030420434FF0000C2024586783F86B
:101E5000814083F882C050686FF4806C20F4E064A5
:101E60005460C2F814C0106800EA0C041460002921
:101E70003FF41EAFDCE700BF480001200001010075
:101E80009D0A00080000FFFF014BD86FFEF7E0BA83
:101E900048000120014B986FFEF7DABA4800012094
:101EA000B0F5804F00B536DA10F5804F31DB00F524
:101EB00080404000194BD3F84023D3F84413521A02
:101EC000B2F5807F13D116494FF0800E154AC2F843
:101ED00018E00A6922F004020A6130BFD3F84023F7
:101EE000D3F844C3A2EB0C02B2F5807FEED0D3F856
:101EF00040230C49D2B203EB42024FF4000CA2F88B
:101F00004803D3F840030130C3F84003C1F818C0B8
:101F100000BD0020CEE74FF6FF70CBE74800012060
:101F200000ED00E000080240174BD3F84023D3F83F
:101F30004413501AB0F5807F12D114494FF0800C31
:101F4000134AC2F818C0086920F004020A6130BFC1
:101F5000D3F84023D3F84403121AB2F5807FEFD0B0
:101F6000D3F84013C8B203EB40024FF4004CA2F880
:101F700048C3D3F8402306494FF400000132C3F8A8
:101F800040238861704700BF4800012000ED00E059
:101F900000080240034AD2F848350133C2F84835F8
:101FA000704700BF4800012008B5224B2249D3F8F2
:101FB00048254FF080600132C3F848258861D3F886
:101FC0004013D3F84423914221D0D3F84003D3F8EF
:101FD0004413884218D0D3F84423D0B203EB400E08
:101FE000BEF848C3D3F844130131C3F8441313486F
:101FF000A3F84CC5FEF7C8FF114A536983F02000CF
:1020000040F40011916108BD4FF6FF7CEFE793F8B3
:102010004E3553B90B48FEF7B7FF0948416981F0C7
:10202000400242F48003836108BD0748FEF7ACFF1D
:10203000F3E700BF4800012000040240940501209E
:10204000000802402EA700082CA7000810B5254B59
:1020500093F84F15D3F8482582B051B1D3F85015F5
:1020600039B1D3F85445121B132A30D90021C3F8D3
:102070005015D3F85845D3F85CC5D3F86025013422
:102080009445C3F8584527D0D3F86045E2B203EB36
:10209000420EBEF86415D3F860450134C3F86045BC
:1020A0008E46D3F86427DFF844C0A0F800E0013280
:1020B000DCF80800C3F864270B4B0180C2F30E0460
:1020C00003EB44020120CCF8082002B010BD0190BF
:1020D00088470198034BC9E74FF0FF3E4FF6FF7169
:1020E000DFE700BF4800012044000020000000207E
:1020F000024B93F84F1501700120704748000120F2
:10210000024BB3F8E0100180022070474800012024
:1021100001207047024B197B01700120704700BFFE
:10212000000000204379012B01D001207047807905
:10213000421E072A9CBF024A10730120704700BF4D
:10214000000000200020704708B5024B024A1A60C8
:10215000FEF756F800C00120AD700DB001207047A9
:10216000054B06491B69064A591A8B1002FB03F3FB
:1021700003700120704700BF0000002030A7000856
:10218000ABAAAAAA01207047064B4FF0000C197D9C
:102190005B7D80F800C0012241708270C370042012
:1021A000704700BF00000020024B93F86B170170CE
:1021B000012070474800012070B500EB010E11F0BE
:1021C00003010246DFF8A0C04FF000001AD0012939
:1021D0000BD0022941D112F8014B80EA0425C5F346
:1021E00007263CF8161081EA052012F8013B80EA28
:1021F0000320C0F3072496453CF8145085EA0026D6
:10220000B0B229D01346517813F8015BD47880EA34
:102210000520C0F307265D783CF8163083EA0020DD
:1022200080EA0126C6F3072104323CF8113083EA24
:10223000062080EA0525C5F3072696453CF81610CA
:1022400081EA052383EA0424C4F307203CF81050F4
:1022500085EA0426B0B2D5D170BD12F8010B3CF866
:10226000103083EA0040B6E748A70008114BB3F8E6
:102270006C270280B3F86E174180B3F87027828014
:10228000B3F87217C180B3F874270281B3F87617D8
:102290004181B3F878278281B3F87A17C181B3F806
:1022A0007C270282B3F87E174182B3F8803783829D
:1022B0001620704748000120012070470020704719
:1022C00010B5074A074BD18A074A0446A1FB030110
:1022D000002305F0ABF802462280022010BD00BFAB
:1022E0000000002040420F0000EE02004379022B64
:1022F00001D001207047C0880649074A01FB00F061
:102300009042F6D8054B0649A3FB0020820CCA82F6
:102310000120704700EE02003F62B00783DE1B43DE
:1023200000000020024B93F88217017001207047D3
:10233000480001204379012B01D0012070478079AA
:102340000228FAD8084A012882F88207F5D192F8C3
:10235000831721B105494FF400628A61EDE7034B11
:102360004FF000609861E8E7480001200008024053
:1023700001207047064B074AD3F884374FF47A712F
:1023800001FB03F3A2FB03231A0B02600420704736
:1023900048000120F11976054379042B01D0012072
:1023A0007047D0F806000649064A01FB00F0A2FB80
:1023B000002305499809C1F884070120704700BF30
:1023C00000EE0200D34D621048000120002070474B
:1023D00008B5FDF715FF00BF034B13211A7E0270ED
:1023E00041700220704700BF00000020074B1A7F99
:1023F000597F42709B8C81704FF0000C012280F855
:1024000000C0C27083800620704700BF000000201B
:1024100001207047074A084BD26A642101FB02F28F
:1024200012F5001C02EB030158BF61468A150270C9
:102430000120704700000020FFFF5F004379012B5F
:1024400001D0012070478079421E632AF9D8054ADD
:10245000054983053233A2FB03204209CA620120E9
:10246000704700BF1F85EB51000000201C4B93F804
:102470008827032A32D800B51A49DFF86CC08A6869
:10248000B0F807E0A2EB0C02002190F806C083F838
:1024900089175210C3F88C17C3F8642783F888C7CC
:1024A000B0F80910A3F890171EF4004F1FFA8EF031
:1024B0001CBF4FF4004E704689B208BF8646814269
:1024C00088BFA3F89007BCF1010FA3F892E704BFFF
:1024D00083F889C7C3F88C27012000BD002070470E
:1024E0004800012000000020440000200020704728
:1024F00001207047194B93F8312093F830100132C6
:102500008B1A48BF03339A10013212F0FF0321D017
:10251000134A012BB2F8941701801BD0B2F896171A
:102520004180022B16D0B2F898178180032B11D06E
:10253000B2F89A17C180042B0CD0B2F89C17018115
:10254000052B07D0B2F89E174181062B1CBFB2F8AD
:10255000A0278281580000F0FE0070470000002094
:10256000480001200020704700207047002070477D
:102570004379012B01D001207047827922B10549AE
:10258000012081F8A2377047024880F8A227012075
:10259000704700BF48000120044B93F8A217024681
:1025A0000B1E18BF01230120137070474800012043
:1025B00000207047094B93F8301093F83130002217
:1025C00061F3070263F30F228908013361F31742B5
:1025D0009B1063F31F62026004207047000000201C
:1025E0004379022B01D00120704781798B089A1E14
:1025F000062A0ED80F4991F8312001324FEA830C98
:10260000B3EB920F81F830C0BCBF0CF1FF3C81F8F6
:1026100031C0C07901308308991E0629E3D8054AE4
:1026200092F83000B3EB900FDDD89B00591E82F872
:102630003110D8E70000002001207047394B93F893
:102640003110002965D011F0070C374A4FF0000314
:1026500031D0BCF1010F27D0BCF1020F1FD0BCF16B
:10266000030F17D0BCF1040F0FD0BCF1050F07D03A
:10267000BCF1060F51D132F802CB20F813C0013360
:1026800032F802CB20F813C0013332F802CB20F825
:1026900013C0013332F802CB20F813C0013332F8F3
:1026A00002CB20F813C0013332F802CB20F813C05C
:1026B00001338B422DD030B5944603F1010E3CF826
:1026C000024B20F81340558820F81E509C1CBCF883
:1026D000025020F81450DC1CD58820F814501C1D22
:1026E000158920F814505C1D558920F814509C1D44
:1026F000958920F81450DC1D0833B2F80EE020F85C
:1027000014E08B4202F11002D6D1490001F0FE0024
:1027100030BD480000F0FE00704732F8023B0380F5
:102720000123A8E700000020EC07012000207047EB
:10273000002070470020704700207047002070473D
:102740004379012B01D001207047807905289CBF77
:10275000024A82F832000120704700BF00000020CA
:10276000034B0B2193F8E42702704170022070475D
:10277000480001204379012B01D001207047807966
:102780000A289CBF024A82F8E4070120704700BF74
:1027900048000120012070472DE9F04181FB0141F3
:1027A000A50B5B0045EA8146B6FBF2F7C11B4FEA79
:1027B000E07060F10008A1FB030403FB0841002363
:1027C00004F0E4FD00296BDBB0F1004F0A4671F123
:1027D000000106464FF001010CDBB30843EA8276A4
:1027E000B6F1004F4FEAA2024FEA410572F1000034
:1027F000E9B2F2DA970347EA9645B40300234FF0B3
:10280000804E980840EA8E739C424FEAAE0E75EBFC
:102810000E02F6DB53EA0E0242D00022164698184A
:102820004EEB060C844275EB0C084FEA93070ADB6B
:10283000B4EB000865EB0C05DB184EEB0E049A18A0
:1028400046EB04064446500847EA8E734FEAAE0E44
:1028500040EAC67253EA0E004FEA6606DFD182FBF9
:102860000171FD1941EB0104EB1941EB0400420138
:102870005D015C1942EAD36640EB0600E71941EBC3
:10288000000100290CDB17F5005341F100029E0BFB
:1028900046EA8245FF2D28BFFF25E8B2BDE8F0815A
:1028A0000020BDE8F08100BF2DE9F0410027144D64
:1028B00082B080464FF400743E46D5F85C25D5F8CA
:1028C00060359A420DF10600F7D0FFF7BFFBBDF966
:1028D0000600013C00FB00F1A4B206EBA136074460
:1028E000002CEAD1394601234FF400723046FFF73D
:1028F00053FF0746012088F8007002B0BDE8F08160
:102900004800012010B5334A002102F1100C538811
:10291000034013F00F0302F1020E0CD05A0851D0FD
:102920005A4082EA930484EAD3049B0814BF2346E6
:10293000134603F00103BEF80220024012F00F021A
:1029400043EA41030BD054083ED05440910884EA36
:10295000920181EAD20208BF224602F00102BEF8CB
:102960000440044014F00F0142EA43020BD04C082B
:102970002CD04C408B0884EA910383EAD10108BF34
:10298000214601F00101BEF80640044014F00F0397
:1029900041EA42010EF106020DD05FEA530E17D054
:1029A00083EA0E0E9C088EEA930484EAD30308BFE0
:1029B000734603F0010343EA41049445A1B2A6D152
:1029C000084610BD0123B4E70122C6E70121D8E77C
:1029D0000123EEE746A90008224910B5044601F19B
:1029E000200E002031F8023F2340C3F30A038BB3CB
:1029F0005A0835D05FEA930C82EA030228D08CEAA9
:102A000002025FEAD30C23D082EA0C025FEA131CB5
:102A10001ED082EA0C025FEA531C19D082EA0C0233
:102A20005FEA931C14D082EA0C025FEAD31C0FD039
:102A300082EA0C025FEA132C0AD082EA0C0282EAD4
:102A4000532C8CEA932C1FFA8CFC5B0A18BF62464D
:102A500002F0010343EA40008E4580B2C2D110BDAE
:102A60000122F5E756A90008F0B53A4C0F46164684
:102A700004F108014FF0000E31F8023D03404FEA27
:102A80004E0213F0FF031FFA82FE20D05D0883EA96
:102A9000050C29D09A0816D0DD088CEA020C12D059
:102AA0001A098CEA050C0ED08CEA020C5D098CEA3E
:102AB000050585EA931282EAD31292B203D09B09EC
:102AC00014BF9446AC460CF001034EEA030E8C4250
:102AD000D2D1BEF1000F2DD0BEF1070F07D84FF6AF
:102AE000FF7030800020F0BD4FF0010CEBE7AEF13D
:102AF0000804E1B2C1F108054FF0010E0EFA05F22B
:102B000042401FFA82FC002908BF8446CCF34013E0
:102B1000CCF3C000CCF3800140EA430441EA440511
:102B2000CCF3400242EA450CA6F800E0A7F800C04A
:102B30000120F0BDC0F34014C0F3C003C0F3800512
:102B400043EA440145EA4102C0F3400040EA420C36
:102B5000EAE700BF78A900082DE9F041654E8646F6
:102B60008846174696E8070084B001AB1C4603C3AD
:102B70000DF10E0C00251A803CF8020D6A001EEAC9
:102B8000000695B23DD0730848D0B10883EA060329
:102B900034D0F00883EA010330D0320983EA00031D
:102BA0002CD0710983EA020328D0B00983EA01031B
:102BB00024D0F20983EA000320D0310A83EA020319
:102BC0001CD0700A83EA010318D0B20A83EA00031A
:102BD00014D0F10A83EA020310D0300B83EA010318
:102BE0000CD0710B83EA000308D0594081EA963378
:102BF000B20B83EAD636B3B208BF0B4603F001022C
:102C000015436445B8D1002D49D00F2D08D84FF693
:102C1000FF7500203D8004B0BDE8F0810123EDE7A1
:102C2000A5F11004E0B2C0F11001012505FA01FC84
:102C30008EEA0C039EB2002808BF7646C6F34034E5
:102C4000C6F3C02242EA4400C6F3802141EA4003B1
:102C5000C6F3402444EA430CC6F3C01242EA4C00D7
:102C6000C6F3801141EA4003C6F3401444EA43002E
:102C7000C6F3001C4CEA4002C6F3C00141EA42031D
:102C8000C6F3800444EA4300C6F3400646EA400225
:102C900001203D80A8F8002004B0BDE8F081CEF30B
:102CA0004031CEF3C02343EA4104CEF3802040EA12
:102CB0004406CEF3402C4CEA4602CEF3C01141EA62
:102CC0004203CEF3801444EA4300CEF3401646EAB2
:102CD0004001CEF3001C4CEA4102CEF3C00343EAAC
:102CE0004204CEF3800040EA4406CEF3400141EABC
:102CF0004602CDE780A900081849194A4B6992F8A5
:102D0000EDC783F0400343F480038B6192F8EC1726
:102D10008C4502D092F8183803B9704792F8EEC784
:102D2000D2F8E81741F82C0092F8EE1792F8EC0769
:102D300092F8EDC7013B0131DBB2C9B2884298BFBE
:102D4000002102EB83000CF1010CD0F8F00782F8AF
:102D5000EE1782F8EDC782F818387047000002407D
:102D60004800012010B5324B324CD3F81C18626B6E
:102D7000A1EB020CBCF1880F0DD94FF0000C10280C
:102D8000C3F81C2883F820C883F821C802D1012188
:102D900083F8211810BD93F821E8BEF1000F3CD054
:102DA000022893F820E80ED0032817D0102830D13D
:102DB000BEF1000FEED000244A1C83F82148C3F86E
:102DC0001C28087010BDBEF1000F1AD1012083F835
:102DD00021E883F82008C3F81C2810BDBEF1000FBD
:102DE000D8D0BCF1050F0CD95079ACF1060188425E
:102DF00007D1D3F8241821B1104688470C4B6063E3
:102E000002460024C3F81C2883F8204883F8214890
:102E100010BDBEF1000FF4D1BCE71028B7D093F875
:102E20002028002AB6D04C1CC3F81C48087010BDDE
:102E30004800012000000020264A116803E01368C2
:102E40005B1A642B35D892F83D30212BF7D01168EE
:102E500092F83CC082F8280892F83D00202814D14E
:102E6000BCF1010F03D01C480121FDF735BD1368EB
:102E7000581A64280DD892F83D301368581A6428FF
:102E800007D892F83D30202BF1D01068431A642BFC
:102E9000E2D9124B4FF400624FF0080EC3F818E06D
:102EA00040209A6180214FF48052986199619A6123
:102EB000FEE70A4B4FF400624FF0080CC3F818C04D
:102EC00040209A6180214FF48052986199619A6103
:102ED000FEE700BF4800012070080120000002400A
:102EE0000B4AD2F82C38D2F83018012003440340A2
:102EF00002EB832CC2F82C38C2F83408054A064B82
:102F00008CF83818C8B232F8101043F8C01C70475B
:102F1000480001208CA90008401101202DE9F84348
:102F2000DFF83CE149499EF838C051F8C03CBCF19B
:102F3000000F22D083EA0028454C464AC8F30727F1
:102F40004FF0000332F817508EF83830D4F82C3890
:102F5000D4F8347804EB832CBC4485EA0826B2B25A
:102F60000137C0F3032941F8C02C8CF83808C4F8A5
:102F7000347801F8BC9CBDE8F883354C11F8BC2CC2
:102F8000D4F82C68D4F82C78050942EA0012D4F859
:102F9000340801F8BC5C04EB8626B046064483EA9C
:102FA0000223BF0286F83828B946C3F30722294F07
:102FB00037F8122082EA032383EA0522C2F30723AB
:102FC000023037F8137086F8395840F2FD3387EA3B
:102FD0000225AEB20122984241F8C06CC4F8340810
:102FE0008EF83820C7D111F8BB7C88F8366C300ACF
:102FF00040F2FF3588F8350CC4F83458D7B111F8D1
:10300000BB6C01F8BBCC4FF4806188F8376CC4F816
:10301000341894F83D20202A0ED00F4908278F61DC
:10302000D4F83058013505F03F06C4F83068BDE8E3
:10303000F84355E72946ECE794F83C30012BECD0F7
:1030400006484844FDF748FCEAE700BF401101206C
:10305000480001208CA900080000024080080120DF
:10306000000000202DE9F043C24A92F83D3087B0BD
:10307000002B00F033825368D568242082F83D008D
:10308000DC6824F40056DE601F69116927F44050A3
:10309000084318615469DE689769116A25433D4306
:1030A00026F4164828F00C000D430543DD605D69E9
:1030B000D469B14F9068396825F4407626435E6143
:1030C000156AB5F5004F00F06381AC4CAC4DA342DE
:1030D0004FEA800C00F0B680AA4EB34200F0B280F6
:1030E000AF6804974FF4E05999FAA9F0AC680294DC
:1030F000B0FA80F799FAA9F6B6FA86F00390AC68B0
:10310000019499FAA9F6B6FA86FEAC6899FAA9F084
:10311000B0FA80F60096AD6899FAA9F8019800F423
:10312000E05929FA0EF6B8FA88F805F4E055019648
:1031300025FA08F0029E0590039806F4E055009EDB
:1031400025FA00FE04F4E054049824FA06F50295EA
:1031500000F4E055FD408C48019F059EC419871975
:1031600094F86894029E97F8688400EB0E0400942B
:1031700087192844009D019021FA09FE95F86804FA
:1031800097F8689421FA08F80EEB8E0408EB880E85
:1031900021FA00F604EB84070EEB8E04B7FBFCF576
:1031A000B4FBFCF7019C06EB860000EB8006B6FB47
:1031B000FCF094F8686421FA09F9F14009EB8908F8
:1031C00001EB810108EB880E01EB8104BEFBFCF9E9
:1031D000B4FBFCF8DFF8B4C1ACFB05656E096424F0
:1031E000ACFB075704FB16004FEA571EACFB085117
:1031F000060104FB1E954F09323629013231ACFB22
:1032000006504409ACFB01C904F0F005C9F34316AC
:10321000354305EB07179F601C6924F490461E6137
:103220005F6927F02A015961DC680020202544F4F9
:103230000056DE60106482F83D5082F83E5007B0C0
:10324000BDE8F083AC6803944FF4604090FAA0F6B8
:10325000AC680194B6FA86F790FAA0F6B6FA86F44E
:103260000294AE68009690FAA0FEAC68BEFA8EF9A1
:1032700090FAA0F6D5F80880B6FA86F690FAA0F093
:10328000009D05F4604E2EFA09F50495B0FA80F021
:1032900008F46045C540019804F4604400F46049B6
:1032A0000298F440039E019429FA00F0364C0090F5
:1032B00006F46040F840009E049F254404EB070894
:1032C000A61995F86894019D98F868E496F86864E2
:1032D000671921FA0EF8201821FA09FE21FA06F9D9
:1032E000009008EB88050EEB8E0609EB890097F835
:1032F000684405EB850706EB860500EB8006009821
:10330000B7FBFCF821FA04F404EB840E90F868444F
:10331000B5FBFCF7E1401D4CB6FBFCF901EB81016C
:103320000EEB8E0501EB8100B5FBFCF6A4FB08510A
:10333000A4FB07574909B0FBFCF04FF0640CA4FB59
:1033400000504FEA571E0CFB119529010CFB1E661D
:103350004709323130013230A4FB0156A4FB00454D
:10336000740904F0F001C5F34310014301EB0717A2
:103370009F6051E74800012000000020001001403C
:10338000003802400014014024A700081F85EB51BB
:1033900005F1804808F51046B342DFF888E24FEAAD
:1033A000400C00F0A0809C4DAB4200F09C80DEF809
:1033B00008604FF4E05999FAA9F4DEF80880B4FAED
:1033C00084F799FAA9F0B0FA80F50295DEF8084082
:1033D000009499FAA9F0B0FA80F50195DEF808504A
:1033E00099FAA9F4DEF808E0B4FA84F499FAA9F994
:1033F000B9FA89F00EF4E05E2EFA00F9009805F4AF
:10340000E05500F4E05EE5400198029C08F4E058C5
:103410002EFA00FE28FA04F00090804C06F4E056E4
:1034200026FA07F7009EA14404EB0E08A6192544CE
:10343000E71999F868E498F8680495F8684497F8EB
:10344000687496F8685421FA0EF921FA00F809EB2D
:10345000890E21FA04F421FA05F5F94008EB8800F9
:103460000EEB8E0601EB8101B6FBFCF804EB840E3B
:1034700005EB850606EB86050EEB8E04B5FBFCF727
:1034800001EB810600EB8009B9FBFCF0B4FBFCF911
:10349000B6FBFCF4DFF888C1ACFB0851ACFB005074
:1034A00046094FEA511E4FF06408ACFB045408FB78
:1034B000167708FB1E95E900F80032313230ACFB7C
:1034C0000156ACFB00C56409C6F342192F0909EB8C
:1034D000041407F4F87C64449C609DE603F0FF014B
:1034E00082F83C10C7E5DEF808604FF4604090FABF
:1034F000A0F5DEF80880B5FA85F790FAA0F4B4FAE2
:1035000084F50295DEF80840009490FAA0F9B9FA23
:1035100089F50195DEF8085090FAA0F4DEF808E08D
:10352000B4FA84F490FAA0F0B0FA80F90EF4604096
:1035300020FA09F9009805F4604500F4604EE54072
:103540000198029C08F460482EFA00FE28FA04F064
:10355000324C0090254406F46046009895F8685473
:103560000095FE4004EB0E07A14497F8688499F893
:1035700068E42718A619009897F8689496F8686484
:1035800021FA08F421FA00F704EB840521FA0EFE73
:1035900021FA09F905EB850421FA06F507EB870105
:1035A00009EB890001EB81070EEB8E08B7FBFCF9F4
:1035B0001B4FB4FBFCF408EB880EBEFBFCF805EBDC
:1035C000850E0EEB8E0500EB8006B5FBFCF1B6FB1D
:1035D000FCF0A7FB0454A7FB08564FEA561E4FF019
:1035E00064086609A7FB015108FB160008FB1E953D
:1035F000EC00C60032343236A7FB0449A7FB06476D
:103600004FEA511C3809C9F3421101EB0C1500F4C3
:10361000F87C65449D60FFE50014014024A7000884
:103620001F85EB5100380240F0B5444D95F88130CC
:10363000202B83B02CD1002200922F6895F8813086
:103640003F4C497804F8B82C0226202B84F84860B7
:1036500004F8B71C1CD13B4C3B4A2168CE08A2FBA6
:1036600006231C0A04EB840C0CEB8C02696C0092A0
:1036700003E08C6914F002040DD0009E731E0093C9
:10368000002EF6D120276E6785F8806085F881705E
:10369000002003B0F0BD95F88020012AF8D006463E
:1036A0004FF0010085F880000B68DFF8A4E0DFF838
:1036B000A4C023F400620A60A86F6A6CC0F84CE0F2
:1036C0004FF0210E85F881E04FF0100E85F882E072
:1036D0000223C5F884401D490465C0E90FC4C0E950
:1036E0001144DFF874C0A5F86E301032A966A5F851
:1036F0006C30C5F870C0FCF75FFE710088B23A46C6
:103700002321FDF71BFA074620B1D5F8843085F850
:103710008040BDE76C6C019066690196A0690190DC
:103720000199636843F480726260616841F40066E5
:103730006660012085F88070ABE700BF480001207B
:10374000401101200000002089B5F81488100120E4
:10375000790A0008F90900080000FFFF70B53C4B2A
:103760003C4C082282B09A61D4F84865FDF708FD08
:1037700072B6394D3948686062B672B60021C4F835
:103780004013C4F8441362B6354B4FF48032022024
:103790009A619861D4F84815D4F848355A1AB2F5A8
:1037A000407F0BD22F48036923F00402026130BF2F
:1037B000D4F848355A1AB2F5407FF4D394F8E4C7E8
:1037C00029496144002091F878E48DF8040001A9AA
:1037D0002D208DF805E0FFF727FFD4F8E4201168CD
:1037E00041F002001060D4F8E420012384F84E3543
:1037F000136843F001011160FDF7C2FC72B61B486B
:10380000686062B6D4F84855AA1BB2F5106F15D29D
:1038100006F51066701B11D0D4F84815D4F8483559
:103820005D1AA8420AD90F4A166926F004031361EB
:1038300030BFD4F848556E1AB042F5D8084C044948
:1038400004204FF40022A0618A6102B070BD00BF65
:10385000000802404800012000000020951F0008D9
:103860000000024000ED00E024A70008A91F0008A6
:10387000012803D820B9012914D9704700207047C6
:1038800000B5DFF838C083B00B46002201A92C2018
:103890008CF815308DF804208DF80530FFF7C4FE44
:1038A00003B000BD0548064B017521B94FF48032C5
:1038B0009A610120704701219961FAE70000002018
:1038C00000080240012800D970470B4A02EBC002F1
:1038D000537F8B42F8D900B50B46116A83B011F8BB
:1038E000331001920093FFF7C3FFDDE9003200B10E
:1038F000137703B000BD00BF0000002008B5134BD4
:10390000134901229A61D1F84805D1F848351A1AAD
:10391000B2F5C07F0BD20F4A136923F00403136181
:1039200030BFD1F848351B1AB3F5C07FF4D391F8F6
:103930004F0550B90849097FFFF7C4FF064ABDE8A3
:10394000084092F824100120BCE708BD00000240A6
:103950004800012000ED00E0000000204379012B29
:1039600001D0012070478279122AFAD810B50B498C
:1039700001EB420482B094F8841401930020009279
:10398000FFF7A0FF019894F88514FFF79BFF044808
:10399000009B0376012002B010BD00BF24A70008E1
:1039A00000000020144A92F84930112B00D97047CA
:1039B00010B5DFF850C01148DCF814100133DBB249
:1039C00000EB430481F4807E82B04EF08070CCF82E
:1039D000180094F8841482F8493000200193FFF70E
:1039E00071FF94F885140120FFF76CFF044A0199D8
:1039F000117602B010BD00BF4011012024A70008BD
:103A00000000002000080240154A92F8493003B92E
:103A100070471448416903F1FF3C5FFA8CF381F46D
:103A2000007C4CF00071122B82F849308161EFD894
:103A300000B50D4A02EB430283B092F8841401935F
:103A400000200092FFF73EFF009B012093F88514B1
:103A5000FFF738FF05480199017603B000BD00BFAC
:103A6000401101200008024024A7000800000020A7
:103A700070B5224E96F84F3582B083B9204D21485B
:103A8000214940F2012440230022C5E91401A5F890
:103A90004A40A5F84C30C6F8502502B070BD184A0F
:103AA00092F84940BCB94FF0010E184E82F849E037
:103AB00071467546744600200192FFF703FF06EB3E
:103AC0004503012093F885140C4EFFF7FBFE104AC6
:103AD000019D1476D3E7112C08D94FF0110C0B4E31
:103AE00082F849C0644665460121E4E7074901EBD5
:103AF00044000E46254690F88414DCE74800012077
:103B000040110120DB1B0400B9A2010024A700081A
:103B10000000002030B5524B082283B09A6172B683
:103B2000504C0020C4F85C05C4F8600562B694F8F7
:103B30004E1500296DD0D4F84815D4F84805D4F8AE
:103B40004825131A5F2B0AD8474D2A6922F004032F
:103B50002B6130BFD4F84825131A5F2BF5D9404D9F
:103B6000424B4FF400204FF48022A8619A61D4F8B0
:103B70004855D4F84835581B5F280AD83A4A136983
:103B800023F00400106130BFD4F84835581B5F287B
:103B9000F5D9334D0191FFF7B1FE34490822AA61EE
:103BA0004FF4003300204FF480258B6184F84E05DC
:103BB0008D61FDF7E5FA72B62D4D2E49696062B64A
:103BC0002D4B2E484FF080629A61FDF7DDF9D4F855
:103BD00048050199431AB3F5106F28D394F84F059F
:103BE00010BBD4F8E420116841F002031360D4F84C
:103BF000E440206820F001022260FDF7C1FA72B6AD
:103C00001F49696062B6164D4FF40023AB6103B0E3
:103C100030BD164D4FF48023AB61FFF76FFE94F873
:103C20004F05134D0028DCD0FFF722FFD9E701F53F
:103C30001062B2EB000CD1D0D4F84805D4F8481586
:103C40000B1A9C45CAD9084A116921F00403136173
:103C500030BFD4F848150B1A9C45F5D8BEE700BF15
:103C6000000802404800012000ED00E00000024092
:103C700000000020951F0008000402402EA7000845
:103C8000514800084379022B70D170B58479302CEB
:103C90006ED8C579002D74D0642D6BD9404E4FF489
:103CA000804506EB8404FFF759FDD4F8F866B41E8E
:103CB00006F2FE36B4F9020005FB00F040F38F3047
:103CC000FEF7EEF8B4F9041005FB01F141F38F3073
:103CD000FEF7E6F8B4F9063005FB03F343F38F3043
:103CE000FEF7DEF8B4F9082005FB02F242F38F304C
:103CF000FEF7D6F8B4F90A0005FB00F040F38F3068
:103D0000FEF7CEF8B4F90C1005FB01F141F38F304A
:103D1000FEF7C6F8B4F90E3005FB03F343F38F301A
:103D2000FEF7BEF834F9102F05FB02F242F38F3094
:103D3000FEF7B6F8A642BDD11A4DFEF7F5F8D5F854
:103D40004043D5F84463B44208D0174B1020986123
:103D5000D5F84013D5F844239142F8D1124D4FF4D1
:103D60008014AC61FFF7D6FE012070BD00207047C3
:103D7000002070BD0D4A0A4EA803A2FB00214D0988
:103D80008FE70B4B064E93F83250C5EBC502C2EBE2
:103D9000C20CA44406EB4C0EBEF9AC5481E700BF44
:103DA00024A7000848000120000802401F85EB51AD
:103DB000000000204379012B53D12DE9F041807997
:103DC000C0EB0011CA0102F58074B4F5006F4FEA30
:103DD000542548D24FF00408FFF7C0FC254E0027B9
:103DE000254CB4F90200FEF75BF8B4F90400FEF7C5
:103DF00057F8B4F90600FEF753F8B4F90800FEF7D7
:103E00004FF8B4F90A00FEF74BF8B4F90C00FEF7CE
:103E100047F8B4F90E00FEF743F834F9100FFEF737
:103E20003FF8A642DDD101374745D9D1FEF77CF8EE
:103E3000124BD3F84003D3F84413884208D0104DF6
:103E40001024AC61D3F84063D3F844239642F8D1F0
:103E50000B4F4FF48013BB61FFF75CFE0120BDE800
:103E6000F0810020704740F2AA384545B4D81FFAC7
:103E700085F8B1E7DEB20008DEAE00084800012098
:103E8000000802402DE9F84F4379022B02D00020B0
:103E9000BDE8F88F0546714EDFF8D091FFF75EFC64
:103EA000A979D6F800B000273846A6F5DF680029C2
:103EB0006AD1FDF7F5FF0424BBF9020033E0FDF7FA
:103EC000EFFFB4F5806F47D0A9793BF90400D6F82D
:103ED00000B00234002940F09780FDF7E1FFA97996
:103EE0003BF90400D6F800A004F1020B00297BD1B5
:103EF000FDF7D6FFAA793AF90B00D6F800A004F135
:103F0000040B002A60D1FDF7CBFFAB793AF90B0027
:103F1000D6F800A004F1060B002B45D1FDF7C0FF39
:103F20003AF90B000834AB79D6F800B0002BC6D0B4
:103F300099F83210C1EBC102C2EBC20ABA4408EBD5
:103F40004A0CBCF8ACE41EFB00F040F38F30FDF7E8
:103F5000A7FFB4F5806FB7D1EB7900243BB1FDF733
:103F6000E3FF0134E979A4B2B4EB412FF7DB3C4A1B
:103F7000964259D056F8043FA979B3F90000D6F813
:103F800000B00137002994D099F83220C2EBC20466
:103F9000C4EBC40ABA4408EB4A0CBCF8ACE41EFB00
:103FA00000F040F38F3084E799F83210C1EBC10282
:103FB000C2EBC20CBC4408EB4C0EBEF8AC3413FB95
:103FC00000F040F38F30A9E799F832C0CCEBCC0E6B
:103FD000CEEBCE033B4408EB4301B1F8AC2412FB1B
:103FE00000F040F38F308EE799F83220C2EBC20C1C
:103FF000CCEBCC0EBE4408EB4E03B3F8AC1411FB73
:1040000000F040F38F3073E799F83220C2EBC20A18
:10401000CAEBCA0CBC4408EB4C0EBEF8AC3413FB24
:1040200000F040F38F3058E70E4DD5F84063D5F8D7
:104030004473B74208D00C4B10219961D5F8404326
:10404000D5F844038442F8D1074D4FF48012AA6199
:10405000FFF760FD0120BDE8F88F00BF1CAE00082F
:10406000DCAE0008480001200008024000000020EB
:104070002DE9F04FC279ADF20C4D0346002A00F055
:10408000DA801446197A09B9012018729D79002D39
:1040900000F0CB806A4A6B4D92F832104FF0000B63
:1040A000C1EBC1085F46C8EBC800C61905EB46095D
:1040B0002744B9F9ACA4BFB2302FD344F5D9624E2E
:1040C00001930DF5816CCCF5806E4FEAEB790EF122
:1040D000020A06F2FE380DF106070020A6F6BC35EE
:1040E000302C0DD80AEB0701234605EB830223444D
:1040F000D2F8F8269BB232F901C0302B6044F4D9D3
:10410000C1178B0343EA90415A4680034B4603F0A4
:104110003DF9464527F8020F02D036F9020FDFE7D6
:10412000FFF71CFB0198047A002C61D000250DF2EA
:10413000064607460DF10602B11A8B1E58080130DB
:1041400010F007020DF106082BD0012A23D0022A15
:104150001DD0032A17D0042A11D0052A0BD0062A15
:1041600005D0BDF908000DF10808FDF799FE38F9F2
:10417000020FFDF795FE38F9020FFDF791FE38F9B1
:10418000020FFDF78DFE38F9020FFDF789FE38F9B1
:10419000020FFDF785FE38F9020FFDF781FE464557
:1041A00021D0B8F90200FDF77BFEB8F90400FDF755
:1041B00077FEB8F90600FDF773FEB8F90800FDF7C1
:1041C0006FFEB8F90A00FDF76BFEB8F90C00FDF7B9
:1041D00067FEB8F90E00FDF763FE38F9100FFDF722
:1041E0005FFE4645DDD13C7A0135A9B28C42A1D8AB
:1041F000164DFDF799FED5F84063D5F84473BE42DD
:1042000008D0134B10209861D5F84043D5F84423CB
:104210009442F8D10E494FF480158D61FFF77AFC76
:1042200001200DF20C4DBDE8F08F3126B6FBF2F700
:104230004FEA873B43E701221446C27122E700BFE1
:104240000000002024A70008E0B200084800012078
:10425000000802404379032B00D109E70020704792
:1042600008B54379012B01D0012008BD82794AB1FC
:1042700009490A4A8020886182F84F35FFF7F8FB28
:10428000012008BD0548044B80F84F254FF400017C
:104290009961012008BD00BF0000024048000120D4
:1042A0004379022B01D0012070478379012BFAD882
:1042B00010B50C4AC07902EBC30282B0517F814233
:1042C000044602D8012002B010BD116A01921846BE
:1042D00011F83410FFF7CCFA019B0028F2D01C77BC
:1042E000F0E700BF000000202DE98048A84C61687D
:1042F000C86820F0200287B0CA600023266894F8BE
:104300003C00C4F87C3294F83E50202D40F0D6801A
:10431000012800F0C580A06BDFF894E29D4EDFF825
:1043200094829D4AE6620025C0E9132525644FF07A
:10433000010CC0E90F8E4FF400533246222704319E
:1043400084F83CC0238684F83E70FCF735F8636837
:10435000924AD96884F84E5541F48071D960596900
:1043600041F00101596159694FF4803041F0400139
:104370004FF400394FF480275961C2F818909761C3
:10438000906184F83C50FCF7FBFE72B6844FDFF876
:104390002882C7F8048062B6824D834BEB654FF0EC
:1043A000020A2A2085F858A0FEF746FD226804E09C
:1043B0002068811A642900F2DC8094F83D002028EE
:1043C000F6D17A49A160FEF74DFE744B4FF40062BE
:1043D0009A61D4F8E00241681FFA81FBCBF5005ED8
:1043E000B5F860B0F34500F03581DFF8D0A133E0D7
:1043F000B5F864C0581E8CEA0B2983B2C9F30721B3
:10440000A5F862303AF811E08EEA092290B2012B49
:10441000A5F864004FEA0B2963D863B9002840F07F
:10442000978095F86A0030B195F85830002B00F06D
:104430009380FEF701FDD4F8E012B5F860304A68C9
:10444000013390B2C3F30C09C0F500518945CB4646
:10445000A5F8609000F0FE80B5F8623016F80BB059
:10446000002BC5D1BBF1100F00F0B9811BF0800FFC
:104470000BF040004FD100286CD0B5F8642082EAE0
:104480000B21C1F307233AF8130085F86AB080EADC
:10449000012240F2FE31A5F86420A5F86210CAE7B7
:1044A0002568AF1B642F0ED894F83E3023689A1B02
:1044B000642A08D894F83E50202DF1D02768BB1B01
:1044C000642B7FF620AF354E08244FF40062402065
:1044D00080214FF48055B461B261B061B161B561C2
:1044E000FEE795F85830012B04D0FFF737F901218A
:1044F00085F8581095F86620012A00F0D180022A2C
:1045000000F0BE80002A96D14FF0010EA5F868B0E9
:1045100085F866E08FE71BF0200F51D11BF0080FE4
:1045200018D01BF0040F0BF0010940F08680B9F1A0
:10453000000F00F0DE8095F85830002840F05181DF
:10454000002B40F015812BF0030349EA03006BE7D1
:10455000A5F86430802067E7226803E02368991A91
:10456000642955D815F8BB1C0029F7D105F8BB0CF8
:1045700061E70A4D08244FF40066402780234FF47A
:104580008052AC61AE61AF61AB61AA61FEE700BF72
:10459000480001203C4D0120650800080000024051
:1045A00000000020401101201D2F0008C0C62D0072
:1045B0006108000829080008951F00088CA9000858
:1045C0000BF01F0190BB12291BD8874ACDF808B009
:1045D000A2F63839019209EB410983460391019B08
:1045E00013F8010B01930128CC4609F101096BD99D
:1045F0000BF1010002284FF0010BF0D1DDE902B10F
:1046000039763A7E2BF01F0002F01F0318430BE7A8
:10461000764D08244FF40062402080264FF48057E6
:10462000AC61AA61A861AE61AF61FEE70A2998BFDB
:1046300084F8E41794F8E427E4E7B9F1000F40F0B8
:104640008E806A4984F84F954FF400038B6194F88B
:104650004F9578E794F84F25D4F84835002A3FF471
:10466000B8AED4F8500500283FF4B3AED4F85415D2
:104670005A1A132A00D880470023C4F85035A8E6F8
:10468000B5F868C04CEA0B13D900A1F5804210B20E
:10469000A5F86830FDF704FC002085F86600CAE63E
:1046A000B5F8683009F470601843C100A1F5804284
:1046B00010B2FDF7F5FB4FEA1B104FF0020BA5F807
:1046C000680085F866B0B6E607EBC0039CF80020EA
:1046D00093F81DE096458BD9196A059311F83210AD
:1046E0000492FFF7C5F8DDE90423002880D01A778B
:1046F0007EE720683E4A102104E0916123681B1A7E
:10470000642B50D8D4F840C3D4F844339C45F4D13A
:10471000374A36484FF4801191614FF400334FF41B
:1047200080224FF48031836182618161002084F8AE
:104730004E05FCF725FD72B6C7F8048062B6022369
:1047400085F8583015F8BB0C00283FF4FCAE15F87E
:10475000BB0CFEF771FB002105F8BB1CF3E62348F8
:1047600080228261012184F84F15FFF781F96EE7FD
:1047700020681F4A102104E0916123681B1A642BF2
:104780001FD8D4F840E3D4F844339E45F4D11848F8
:104790004FF480128261FEF7A3FBFFF7BBF9002103
:1047A00085F85810CFE6114E08244FF400654027D5
:1047B00080214FF48052B461B561B761B161B261DB
:1047C000FEE70A4E08244FF40065402780204FF48E
:1047D0008052B461B561B761B061B261FEE7FBF7C9
:1047E0000FFD002BAED1AEE6E0B60008000002409F
:1047F000000802404379022B01D0012070478179E3
:104800000129FAD8C27949B9012AF6D80E480F4BC6
:104810000275B2B94FF480329A61EEE700B5DFF865
:1048200028C083B04FF0000E01A92C208CF8152071
:104830008DF804E08DF80520FEF7F6FE012003B0A8
:1048400000BD01219961D8E7000000200008024066
:1048500010B56248624A4369624983F0800444F4B7
:10486000000384B08361D2F84805CC6D0130C2F8F2
:104870004805B2F83C3198B224B10190A047584A9B
:1048800058490198C000C0F58044A0F5804C91F8CB
:104890006B000FFA8CFE23B213EA2E0338BF734667
:1048A00001EB400E013000F03F04BEF96C0081F8CE
:1048B0006B40D1F8EC40AEF86C301B1A486D2344C5
:1048C0008342D2F84845C1F8EC304FDAB1F84A00DB
:1048D0002123A1F84C30431E98B2A1F84A000028C9
:1048E00064D0D2F85C05D2F86015431AB3F5807F26
:1048F0002FD13A4C606980F4806141F08063A361FC
:1049000039483A493A4B4FF0007484611068C2F854
:104910001411C2F81C31D2F8E41003E013681C1A19
:10492000642C4DD88C68A307F8D54AF6AA2200203B
:10493000CA600390CB6803938C680394039B4A6816
:1049400042F0400048600B6843F040040C6004B043
:1049500010BDD2F85C45E0B202EB4001A1F864C59D
:10496000D2F85C350133C2F85C35C9E7086D834283
:1049700014DDB1F84C3040F20120A1F84A00581E75
:1049800083B2A1F84C30002BABD11A48C2F8544581
:104990002124C2F85005A1F84C40A2E7212440F29E
:1049A0000123A1F84C40A1F84A309AE7124BC2F813
:1049B000544540F20124C2F85035A1F84A4090E72E
:1049C0000E4B08249C614FF40062402080214FF47C
:1049D00080549A61986199619C61FEE700080240E9
:1049E000480001204011012000040240E2B6000806
:1049F00084010120093A0008A5390008000002409E
:104A00004379012B01D0012070476D4B82796D49AC
:104A100083F86B2731F812C0B3F8692762454FF06D
:104A20000000F0D030B5FF2493F8815089B083F8AE
:104A30006847A3F869C7D3F868178DF80C00202DD4
:104A4000CDF80D1010D1DDE90324DFF884C14CF856
:104A5000B82C1A6893F881000CF8B44C4FF0050E8E
:104A600020288CF848E002D0012009B030BDD3F8EE
:104A700044C003E01D68A81A19282BD8DCF8185088
:104A8000E94311F00204F5D093F880000128EBD03F
:104A9000012183F88010DCF800504B48019225F486
:104AA00000642125CCF8004083F8815010240025B3
:104AB00083F88240C3F884501867A020FCF73EF8C2
:104AC000019A3F4B70B14FF00001D3F8842083F876
:104AD0008010C9E74FF0200C5C6783F8804083F8B2
:104AE00081C0C1E7596C0290486902908C690294B8
:104AF0000298364D4FF0050E486910F080042AD117
:104B0000D1F814C01CF4806C19D11C68A01A0128BB
:104B1000F2D9D3F8842020252A43C3F88420C3F88F
:104B200074C083F88150D3F884400025042C83F8A6
:104B3000805099D10B6843F40070086094E76FF4DB
:104B4000806C04202022C1F814C0C3F884005C6784
:104B500083F88120E7E7AC460EF1FF34A0B21CF8E1
:104B6000014B0C614C69640726D528B36C780C6145
:104B7000AEF102001FFA80FE0235486910F004040D
:104B800009D1D1F814C01CF4806CD8D11C68A01ACB
:104B90000128F2D9BDE7BEF1000FADD10A6842F499
:104BA000007008602025012083F8815083F880E0A0
:104BB00083F882E009B030BD86466546DDE700BF78
:104BC0004800012048A700080000FFFF88100120CE
:104BD00040110120DFF824C000B58646BCE80F0074
:104BE000CEF80000BCF80000AEF81000CEF80410BB
:104BF000CEF80820CEF80C30122000BDC401030806
:104C00002E4A2F49DFF8D8C0034610682D4A10B548
:104C10000C68186003CAC3F803402B4CC3F80600A5
:104C2000C3F80A1003CC18615961BCE8030014886A
:104C3000264A98611068264AD9614FF03A0E2549F4
:104C4000C3F8220083F820E01068DFF898E0C3F88A
:104C5000250092880868DC814FF0310C83F821C070
:104C6000C3F82B00A3F82920BEE80700DFF878C0BE
:104C7000C3F82E00C3F83210BCE80300C3F8362096
:104C8000154AC3F83B002C2483F83A4083F845408A
:104C9000C3F83F10114CBCF800C02488A3F843C0EF
:104CA00003CAC3F84A10A3F84D4093F84D10C3F857
:104CB00046002C2914BF4E204D2010BDDC010308F6
:104CC000E0010308E4010308F001030808020308F7
:104CD0000C02030814020308340203083C02030810
:104CE000FC0103081802030828020308074B0022EE
:104CF000C3F86C27C3F87027C3F87427C3F8782764
:104D0000C3F87C27A3F880270120704748000120C2
:104D10002DE9F04FAA4AAB49AB4BAC4CAC4DB1B00E
:104D2000824602F5006001F5006603F50067CDE9F3
:104D30000D130C9209908022002110A80A960B975F
:104D400008940F9505F0ACF9A24E4FF40077D6F811
:104D50005C25D6F860158A42F9D00DF11E00FDF7EA
:104D600075F9DDE908C06446BDF91EB0BCF8021053
:104D700034F8043B0894DDE90A52119CB0F8029023
:104D800011FB0BF141F38F38444430F8041B1194AC
:104D90006C88099011FB0BF035F8041B0A9519FB80
:104DA0000BFC159D14FB0BF949F38F3440F38F383E
:104DB00011FB0BF0518813FB0BF3254443F38F3E9B
:104DC00015954CF38F3311FB0BF540F38F3C109985
:104DD00032F8040B0B92714410FB0BF2DDE913E087
:104DE00042F38F399E44DDE9163245F38F34129D2C
:104DF0001091A84484444B442244CDE9128ECDF84E
:104E000050C0CDE91632DDF830800F99B8F8025065
:104E100038F8043BCDF83080DDE90D4013FB0BF989
:104E200015FB0BF5209B49F38F3245F38F3C219DF9
:104E3000B0F802901A4463882092AC4434F8045BC2
:104E40000D9413FB0BF343F38F3E15FB0BF34C88D0
:104E5000CDF884C019FB0BF243F38F3830F8043BD4
:104E60000E9042F38F3931F8042B0F9113FB0BF0A6
:104E700014FB0BF5279B45F38F3412FB0BFB40F320
:104E80008F3C4BF38F312344DDE9242BDDE92240B5
:104E9000269D2793013F0D44444470446244CB4413
:104EA000BFB2CDE92240CDE9242B2695002F7FF417
:104EB0004EAF5046CAF8007040F8047F4FF06409C6
:104EC000B8460DF1400AA0F1040C5346C6465546BB
:104ED000CDE9043C61460CF102069846F346824651
:104EE000AC46D8E9007484FB042E87FB0737900B8F
:104EF0009C0B40EA8E4544EA8742A8185AD487148E
:104F0000840300234FF080409D0845EA80739C4253
:104F10004FEAA00077EB0002F6DB53EA000249D02B
:104F2000CDE9018100229646CDF80CB0991840EBEE
:104F30000E058C4277EB050B4FEA930808DB641AE9
:104F400067EB0507DB1840EB000B9A184EEB0B0ED6
:104F5000510848EA8073801041EACE7253EA00019A
:104F60004FEA6E0EE2D11C4CDDF80CB009FB02F5E5
:104F70002F19DDE9018117EA250738BF2F46BB1538
:104F800001F8013BB14208F10808AAD1049B514540
:104F9000DE465046654603F1100301D08C4697E784
:104FA000059E0CF1400AB01DBBF1000F04D14FF07B
:104FB000020888E70023E3E7082031B0BDE8F08F5E
:104FC000E4BE0008E4CE0008E4DE0008E4B6000811
:104FD000E4EE000848000120FFFF3F00054B0022DF
:104FE000C3F89427C3F89827C3F89C27A3F8A027F1
:104FF000012070474800012008B5402200210248E6
:1050000005F04EF8012008BDEC07012070B5A6B0F0
:1050100006469822144C0021684605F041F8FE220D
:10502000012325688DF802208DF805308DF8066083
:1050300003E02068411B642907D807216846FCF774
:10504000E1F80028F5D026B070BD084E08234FF4D3
:105050000062402480254FF48050B361B261B46196
:10506000B561B061FEE700BF4800012000000240CA
:105070002DE9F0477B4D95F8F47095F8F530BB427B
:1050800086B004463ED0784E96F81808002839D0ED
:10509000E17801F00303012B00F09180022B00F076
:1050A000AC80A1787F2931D095F8F690D5F8F03012
:1050B00096F8828743F8294095F8F64095F8F50070
:1050C00095F8F4200134E1B28A4298BF0021471CD0
:1050D00085F8F61085F8F570B8F1010F05D1634D2C
:1050E00086F883874FF40063AB6196F818484CB19B
:1050F00004F1FF3C5FFA8CFA06EB8A0986F818A8DF
:10510000D9F8F047204606B0BDE8F0876379002B58
:10511000CAD0607896F86B97814501D0FF28C3D13B
:10512000D4F806200192D4F89030D5F89411504864
:105130005A1A99468A460023A2FB00014D4A02F002
:1051400075F9019BC11A01EBD17096F882174210D4
:10515000A2F12208022928EAE873884677D0029350
:10516000D6F848354248434A0093A3EB0A0EAEFBFB
:105170000001002302F05AF900993D4A0390A1EB87
:105180000903A3FB02013B4A002302F04FF90199F6
:10519000CDE904010DF1080CBCE80F004FF0100E32
:1051A00084F805E0C4F8060095F8F500C4F80A1084
:1051B000B842C4F80E20C4F812308DD074E794F8C9
:1051C00001C096F86B078445E0467FF46AAF9822E9
:1051D000002105F1FC0085F8F83004F061FF85F846
:1051E000FC8094F800A094F8048085F8FDA07F2747
:1051F00085F8FE7085F8008156E796F86B27607891
:105200009042904602D0FF287FF44BAF96F8A21749
:1052100000297FF446AF98221748012785F8F870D7
:1052200004F03EFF85F8FC8094F8009094F804A008
:1052300085F8FD907F21042385F8FE1085F800A1F4
:1052400085F80131D4F89420C5F802212CE70748ED
:10525000426982F4006141F000628261D4F890906A
:105260007DE700BF401101204800012000080240F6
:1052700040420F0000EE02003C1201202DE9F04FE9
:10528000DFF8508398F8993100229FB088F8982170
:10529000002B00F0ED82DFF84093DFF840B3CA48FE
:1052A00098F8A011047E98F8A161D8F89C51A14209
:1052B00028BF2146A64238BF264688F8A0112F19DC
:1052C000402200210EA8C8F89C7188F8A16104F062
:1052D000E7FE98F8A23198F8A3A10133DBB29A4512
:1052E00088F8A23100F0AB82B848C41894F8E8CA34
:1052F00094F8F4EA0CEB4C020244724492F8C45B5A
:1053000092F8D06B00EB850100EB8607D1F8000B1B
:10531000D7F8005BAD4C07952344069093F8EBAAB1
:1053200093F8F7CA0AEB4A0EA644E64493F8EEAAAD
:105330009EF8D06B9EF8C42B93F8FACA0AEB4A0E7B
:10534000A644E64493F8F1AA93F8FDCA04EB86015B
:105350000AEB4A039EF8D06BD1F8005B0995234411
:1053600004EB8601634404EB8207D1F8005B9EF8EE
:10537000C42B93F8D06B93F8C41BD7F8000B08909C
:1053800004EB820704EB860E04EB8104D7F8000BD4
:10539000DEF8002BD4F8007B0A90CDE90C720B9557
:1053A0004FF40076D9F85C55D9F86005854200F0D5
:1053B00016820DF11600FCF749FE069FBDF9163066
:1053C000D8F8A811D8F8A4413A4603FB03FA32F8FA
:1053D000040B0692194404EBAA35C8F8A81110FB77
:1053E00003F40E99C8F8A45144F38F350D440E957B
:1053F0007F880F9A17FB03FA079F4AF38F303C46CA
:1054000010440F9034F8041B109A079411FB03F416
:1054100044F38F31114410917F88119C17FB03FADC
:105420004AF38F32089F2244119201923A46013E7C
:1054300032F804AB08921AFB03F4129A44F38F3447
:10544000144412947F8817FB03FA4AF38F32139F98
:10545000DDF824A03A44D6461392149F3EF804CBBC
:10546000CDF824E01CFB03FC4CF38F3C67441497FD
:10547000BAF80270DDF828E017FB03F747F38F3A1C
:10548000159F574415977746B6B237F804CB0A975D
:105490001CFB03F747F38F3A169F57441697BEF845
:1054A0000270DDF82CE017FB03F747F38F3C179FE2
:1054B00067441797774637F804AB0B971AFB03F747
:1054C00047F38F3C189F67441897BEF80270DDF8C9
:1054D00030E017FB03F747F38F3A199F57441997AA
:1054E000774637F804CB0C971CFB03F747F38F3A4A
:1054F0001A9F57441A97BEF80270DDF834A017FBC4
:1055000003F747F38F3E1B9F7744D6461B971C9F9C
:105510003EF804CBCDF834E01CFB03FC4CF38F3C8D
:1055200067441C97BAF802A01AFB03F343F38F37C2
:105530001D9B3B441D93002E7FF434AF244F98F8FD
:10554000AC610823BB6198F89871002E00F086804A
:1055500080FB000C830B85FB050543EA8C4A830B1B
:1055600081FB010143EA854C850B019845EA8143A3
:10557000E24480FB001C8D0B45EA8C40034408EBA1
:105580004711012EC1E96CA368D082FB0232980B4F
:1055900040EA8243DDE914A584FB0424900B40EA31
:1055A000844C634485FB0552C1F8B831AB0B8AFBD0
:1055B0000A5AA80B43EA824440EA8A4C6444022E09
:1055C000C1F8BC414AD00BE000000020FCFB000801
:1055D00000080240401101204800012000ED00E0D9
:1055E000DDE9164282FB020584FB044C820BDDE9F7
:1055F00018A342EA8540A50B45EA8C421044C1F845
:10560000C00183FB03309C0B8AFB0A2344EA8045DC
:10561000900B40EA834A5544032EC1F8C4511DD073
:10562000DDE91AC484FB0425940B44EA85428CFB13
:105630000C4AA50BDDE91C3045EA8A4C6244C1F8EE
:10564000C82183FB03329C0B80FB003044EA824577
:105650009A0B42EA804A5544C1F8CC5198F89941D6
:10566000854B0137FDB24FF40021AC42996188F8B7
:1056700098513FF614AE804810228261002E00F04F
:10568000D780DFF808E2B8F8B8429EF80C70DFF86F
:105690000092D8F8B002D8F8B4C20297013403944B
:1056A0000025DEF83C40019509EB471702990029D7
:1056B00000F0CB8009EBC502A7EB020BABF1200396
:1056C0004FEA531A0AF1010B00211BF0030A0B46A3
:1056D00068D0BAF1010F28D0BAF1020F12D059F8F0
:1056E00035B0D2F804A0DA45ABBFAAEB0B0AABEB9E
:1056F0000A0A4FF0010B8B46BAF1000FC4BF59469E
:1057000053462032D2E900BADA45ABBFAAEB0B0A06
:10571000ABEB0A0A4FF0010B4FF0000B9A45C8BFE4
:10572000594620329A45C8BF5346D2E900BADA45F5
:10573000ABBFAAEB0B0AABEB0A0A4FF0010B4FF021
:10574000000B20329A45C8BF59469A45C8BF5346F8
:10575000BA4227D14BE0A3EB0B034FF0000B5345AC
:10576000DCBF53468B46D2E908A15145ABBFA1EB44
:105770000A0AAAEB010A012100219A45D4BF9A46E0
:105780008B46D2E910319942ABBFCB1A5B1A01218B
:10579000002160325345D8BF59465345D8BF5346C0
:1057A000BA4224D0D2E900BADA45B5BFABEB0A0A57
:1057B000AAEB0B0A4FF0000B4FF0010B9A45D8BF34
:1057C0009A4602F120021368C8BF5946D2F804B0C5
:1057D0009B45C0DBABEB03034FF0010BBFE7DBF8EE
:1057E000101021F00403CBF8103030BFDAE51818A0
:1057F0004CEBE37C227841EA42030399237029446D
:105800004A0707D11D4A0134A31AB3F5897F1ED276
:10581000012201920135AE4207F108077FF446AF3D
:10582000019DA8F8B8120DB1CEF83C40C8E9AC0C07
:10583000114C4FF48016A6611FB0BDE8F08F002315
:105840000F4D104888F8A23164E50299D2E70E4F57
:10585000C8F8B002B7F88007A8F8B8120130CEF83F
:105860003C40C8F8B4C2A7F880071FB0BDE8F08F6D
:1058700098F8AC61FFE600BF00080240FC1301206D
:10588000E4F60008E4FE00084800012000000020C3
:10589000F01201202DE9F04FDFF828A0084BDAF8CC
:1058A00040402022ADF2B44D9A61657965B94FF45C
:1058B000001401209C610DF2B44DBDE8F08F00BFD3
:1058C0000008024000000020E378854AC3F380010D
:1058D00001EB4100A2F10C0808EB80090C2D43F309
:1058E000800699F80CB006F00C0799F80D608CBF93
:1058F0004FF002094FF001094D440BEBC50C0CF1C0
:10590000FF3EBEFBFBF50DF52A7B174400216A0024
:105910005846CAF81070009704F0C2FB009B002E96
:1059200000F09E80002D00F07383691E1FFA81FC39
:105930000DF2AA2E6B490EEB4C0780224FF0000CA3
:10594000A7EB0B08A8F102004008013010F003009B
:10595000DE4637D0012823D0022810D091F80090DD
:10596000BBF8000012EA090F4FEA400018BF40F0F0
:1059700001002EF8020B520804BF0131802291F879
:105980000080BEF8000012EA080F4FEA400018BF7E
:1059900040F001002EF8020B520804BF01318022B2
:1059A000BEF8000091F80090400012EA090F18BFFD
:1059B00040F0010052082EF8020B01D10131802283
:1059C000BE4548D091F80090BEF80080704612EABB
:1059D000090F4FEA480E18BF4EF0010E20F802EBF7
:1059E0005208804608BF013138F802EB91F8009068
:1059F00008BF802212EA090F4FEA4E0918BF49F08A
:105A00000109520828F8029C01D18022013191F845
:105A100000E0B0F8028012EA0E0F4FEA480918BF02
:105A200049F00109520808BF0131A0F8029091F82D
:105A3000008000F1060E808808BF802212EA080F5D
:105A40004FEA400018BF40F0010052082EF8020C47
:105A5000B4D0BE45B6D10CF1010CB4457FF470AFA3
:105A6000002D00F01F836C1EA5B20DF2AA2E0EEBC6
:105A7000450928AC19F0020F00951B4FDFF86C8028
:105A800025460DF11A0600F0D0819B68BBF8000096
:105A9000324621469847002800F0CF8130880DF229
:105AA000AA2BA0B1DAF84010B7F87C2791F888C08B
:105AB00052FA80F5604481F88800A7F87C57D8F83E
:105AC000143083F0400040F48001C8F81810D94524
:105AD000DAF8103004F1020540F0A78108E000BFB9
:105AE00030A700080A1401204800012000080240E5
:105AF0000DF11C09822200214846019304F0D0FADE
:105B0000019F009897F80080012508F1FF36B54005
:105B1000A61C06EB400BA8B2002800F0D382A9B265
:105B2000B1FA81F2C2F11F0301930709002345096D
:105B300019464A464FEA500C4FEA900E03970495D7
:105B4000CDF808B0CDF814904FEAD008B4F8009022
:105B500001F0070710EA090F4FEA430318BF43F0AB
:105B60000103072F009701F1010500F078811FFA6A
:105B70008CF7BCF1000F00F00E8117EA090F4FEA15
:105B8000430305F0070718BF43F00103072F08BFC1
:105B900002F8013B01F1020B08BF0023BEF1000F28
:105BA00000F0F980B4F800905B001EEA090F0BF0DA
:105BB000070718BF43F00103072F04BF02F8013B9A
:105BC0000023B8F1000F00F0E68027885B0018EA98
:105BD000070F4FEA417718BF43F00103B7F1004FB9
:105BE000039F04BF02F8013B0023002F00F0D38085
:105BF000B4F800B05B0017EA0B0F01F0070718BFFD
:105C000043F00103032F049F04BF02F8013B00236C
:105C1000002F00F0C080B4F800905B0017EA090F75
:105C20004FEA417718BF43F00103B7F1804F04BF3B
:105C300002F8013B0023870900F0AD80B4F800B002
:105C40005B0017EA0B0F4FEA417718BF43F00103DF
:105C5000B7F1005F04BF02F8013B0023C70900F061
:105C60009A80B4F800905B0017EA090F18BF43F060
:105C700001035FEA417904BF02F8013B0023070AF0
:105C800000F08980B4F800B017EA0B0F009F4FEACC
:105C9000430318BF43F00103072F00F0EF805FEAD2
:105CA000502978D019EA0B0F4FEA43034FEA417BA2
:105CB00018BF43F00103BBF1404F08BF02F8013B9E
:105CC00001F10A0708BF00235FEA902963D0B4F806
:105CD00000B007F0070719EA0B0F4FEA430318BF9C
:105CE00043F00103072F04BF02F8013B0023C70A5A
:105CF00051D0B4F800905B0017EA090F4FEA4177E2
:105D000018BF43F00103B7F1004F04BF02F8013B95
:105D100000235FEA103B3ED027885B001BEA070F99
:105D200001F0070718BF43F00103032F04BF02F877
:105D3000013B00235FEA503B2DD027885B001BEA24
:105D4000070F4FEA417718BF43F00103B7F1804FC7
:105D500004BF02F8013B00235FEA903B1BD0278879
:105D60005B001BEA070F4FEA417718BF43F00103BE
:105D7000B7F1005F04BF02F8013B0023C70B0AD054
:105D8000248804F0010747EA430949070ABF02F8DB
:105D9000019B4B46002301996918029DB542344688
:105DA00078D00236D2E633880235324629460BF1E6
:105DB000020BA3B1B7F87CC7DAF840E05CFA83F0D5
:105DC0009EF888C0A7F87C0763448EF88830D8F81E
:105DD000143083F0400040F48003C8F81830DAF83B
:105DE00010008368BBF80000984730B33088023554
:105DF0000BF1020BA0B1DAF84010B7F87C2791F84C
:105E000088E052FA80F3704481F88800A7F87C3764
:105E1000D8F8140080F0400141F48002C8F818203E
:105E2000D945DAF810303FF463AE9B68BBF8000048
:105E30003246294698470028B5D19E4D9E486F6945
:105E4000B0F87E6787F0800141F400030136AB6152
:105E5000A0F87E6700200DF2B44DBDE8F08F02F887
:105E6000013B1FFA8CF3BCF1000F94D027883B4212
:105E700014BF0123002301F1020B8FE602F8013B5E
:105E8000430A88D027883B4214BF0123002301F135
:105E90000A0719E7DDF81490DAF8404062790C2A15
:105EA0005BD8002A57D0854D99F8006099F80170A9
:105EB000AB5D501CC1B27B400229EB5C3FD099F82E
:105EC000026073400329EB5C39D099F8030043402A
:105ED0000429EB5C33D099F804707B400529EB5C16
:105EE0002DD099F8056073400629EB5C27D099F80E
:105EF000060043400729EB5C21D099F807707B40EE
:105F00000829EB5C1BD099F8086073400929EB5C09
:105F100015D099F8090043400A29EB5C0FD099F895
:105F20000A707B400B29EB5C09D099F80B60734039
:105F30000D29EB5C03D199F80C104B40EB5C33B1AD
:105F40005D4AB2F87A470134A2F87A4782E74946B7
:105F5000A01D01F085FA574BA9E40DF11E0A9244E9
:105F60001AF00307564E48464FF0000322D0012F87
:105F700013D0022F07D099F800C036F81C800DF11D
:105F80001D0088EA0C4310F801BB83EA0B23C3F31E
:105F9000072136F8115085EA032310F8017B83EAC4
:105FA000072CCCF30723504536F8138088EA0C21E0
:105FB0008BB2C4D0834645781BF8017B83EA072C5B
:105FC000CCF307219BF8018036F8113083EA0C27C7
:105FD00087EA0525C5F30721043036F811B010F81B
:105FE000011C8BEA052C8CEA0828C8F307235045CE
:105FF00036F8137087EA082585EA0127C7F3072BCF
:1060000036F81BC08CEA07281FFA88F3D2D196E72E
:10601000711E11F00E0FC1F3420320D00225AE42D3
:1060200040D0012B1BD0AB4216D0032B11D0042B38
:106030000CD0052B07D0062B02D02D44AE4231D018
:106040000235AE422ED00235AE422BD00235AE42E2
:1060500028D00235AE4225D00235AE4222D06B1C8C
:106060009E4205F1020205F1040A05F1060805F158
:10607000080905F10A0705F10C0005F10E0B11D016
:10608000964205F110050DD056450BD0464509D076
:106090004E4507D0BE4205D0864203D05E4501D0B2
:1060A000AE42DCD10DF11C0982220021484603F0EA
:1060B000F7FFF3E60008024048000120D807010876
:1060C00048A70008ABEB040CACF1040111F01C0F65
:1060D000C1F382022FD05E453FF4DEAE0434012AC4
:1060E00004F1020627D0022A20D0032A19D0042A5C
:1060F00012D0052A0BD0062A04D05E453FF4CCAE60
:10610000A61D04345E453FF4C7AEA61D04345E45AB
:106110003FF4C2AEA61D04345E453FF4BDAEA61DDD
:1061200004345E453FF4B8AEA61D04345E453FF42A
:10613000B3AE0434A61C5E4504F1040304F1060E5C
:1061400004F10A0804F10E0704F1120504F1160027
:1061500004F11A0C3FF4A0AE9B4504F11E063FF477
:106160009BAEDE4504F120043FF496AED8453FF4E3
:1061700093AE5F453FF490AE5D453FF48DAE58451C
:106180003FF48AAEDC453FF487AE5E453FF484AE13
:10619000A61CD0E72DE9F04FC178DFF8E8924479EA
:1061A000DFF8E4B2ADF2AC4D41F3800303F00C0232
:1061B00009F10C0505AF15440646C1F380082246D7
:1061C000811D3846CBF8105001F04AF90C2C4FD8FD
:1061D000002C00F0438297F800C0A848012C10F86A
:1061E0000C3034D079784B40022CC35C2FD0BA7875
:1061F0005340032CC35C2AD0F9784B40042CC35C79
:1062000025D03A795340052CC35C20D079794B4096
:10621000062CC35C1BD0BA795340072CC35C16D044
:10622000F9794B40082CC35C11D03A7A5340092CC1
:10623000C35C0CD0797A4B400A2CC35C07D0BA7A85
:1062400053400C2CC35C02D1F97A4B40C35C3B55E4
:1062500026A84FF402720021019003F021FF08EB01
:10626000480209EB820898F80CC04FF0010864E07E
:10627000601E0DF1150111FA80FC1CF0030180482D
:106280003A464FF000031AD001290CD0022940F001
:10629000DC8112F8011B83EA012ACAF3072330F8D4
:1062A000131081EA0A2312F801EB83EA0E2ACAF3DB
:1062B0000723944530F8131081EA0A232AD01146A7
:1062C00092F801A011F801EB83EA0E23C3F3072E25
:1062D000497830F81EE08EEA032383EA0A2ACAF3DB
:1062E000072E043230F81E3083EA0A2A8AEA012E89
:1062F000CEF3072130F8113012F8011C83EA0E2A80
:106300008AEA012ACAF30723944530F8131081EA78
:106310000A23D4D13A19190A395526A853700021F5
:106320004FF40272019003F0BBFE08EB480009EB4A
:1063300080094FF0020899F80CC0387808EB040186
:106340008E46CB0063445A1E92FBFCFABAF1000F52
:1063500040F39E80019900220A800DF19A09BCF158
:10636000000F00F05D81CDE90245802390460024B6
:106370001CF00305214633D0012D1FD0022D0DD076
:10638000184214BF012400245B0806D10132D2B2A6
:1063900096458CBFB85C18468023012118424FEA0D
:1063A000440418BF44F001045B0806D10132D2B2A4
:1063B00096458CBFB85C18468023013118424FEADD
:1063C000440418BF44F001045B0806D10132D2B284
:1063D00096458CBFB85C1846802301318C4540D06F
:1063E00018424FEA440418BF44F001045B0806D188
:1063F0000132D2B296458CBFB85C18468023184251
:106400004FEA440518BF45F001055B0801F10101A1
:1064100006D10132D2B296458CBFB85C18468023B3
:1064200018424FEA450418BF44F001045D0806D144
:106430000132D2B296458CBFB85C284680252842EE
:106440004FEA440418BF44F001046B0806D101323E
:10645000D2B296458CBFB85C1846802303318C4578
:10646000BED108F101011FFA81F8C24529F8024C9A
:106470000CDD4FF0000429F8024B78E7D80701083B
:1064800048A7000824A7000800000020DDE9024515
:10649000A8AF4FF402720021384603F001FEDDF888
:1064A00004A0B9464FF000082CB10C2C8CBF02237D
:1064B00001231C44E4002A781319581E90FBF2F1C2
:1064C00041450BDD6A683AF8020B904708F1010874
:1064D00029F8020B7479DBF81050E5E76E78012596
:1064E000741EA540A8B2002800F08F808AB2002A4E
:1064F00000F0878002F1FF3BBB1C1FFA8BFC604A57
:1065000003EB4C040023E11B8E1E7108013111F0D6
:1065100003063D4638D0012E23D0022E10D011782C
:1065200035F8029B013310EA090FDBB24FEA41064E
:1065300018BF46F00106082B167004BF0023013275
:10654000117835F802AB013310EA0A0FDBB24FEADB
:10655000410618BF46F00106082B167004BF002341
:106560000132117835F802EB4E0010EA0E0F03F1FC
:106570000103DBB218BF46F00106082B167004BFFA
:1065800000230132AC4244D02946157831F8028B01
:106590000133DBB210EA080F4FEA450618BF46F098
:1065A0000106082B167004BF013200231578B1F8DC
:1065B00000B0013310EA0B0F4FEA4506DBB218BFFB
:1065C00046F00106082B167001D100230132157820
:1065D000B1F802C0B1F8049001336E0010EA0C0F5C
:1065E000DBB218BF46F00106082B167008BF013257
:1065F00001F10605117808BF00234E0010EA090FCB
:10660000B5E7430801D08008FBD10DF2AC4DBDE8E1
:10661000F08F40087FF477AF0DF2AC4DBDE8F08FFE
:106620000CF101071FFA87FE0CF10200F2451FFA78
:1066300080FC7FF72DAFE245A9F800207FF728AF57
:10664000A9F8022009F10409EAE797F800A030F858
:106650001AE00DF115028EEA0A431AE626A84FF455
:10666000027221463C70019003F01AFD08EB4802CB
:1066700009EB8209204699F80CC02346A64661E63C
:106680001E1501202DE9F04F354D364EB5F86C370B
:10669000354A364F04464FF40061A1B00133916191
:1066A00006F574704FF489720021A5F86C3703F079
:1066B000F7FCFDF753F820681090A588ADF844501A
:1066C00000225FFA80F8A6F8E22417F808309DF857
:1066D00041109DF842004B409DF84310FD5C454041
:1066E0009DF844007B5D4B409DF84510FD5C4540A6
:1066F00046467B5D4B400DF16205FB5C8DF84630F4
:10670000CDE91922CDE91B22CDE91D221F920DF101
:106710007E0BA84680273E4214BF012300235FEA78
:10672000570A28F8023F62D10132D2B2062A14D8A1
:106730000DEB020C9CF940109CF84060C80F40EA39
:106740004300C6F38013C6F3401743EA400947EA03
:106750004903A8F8003010276AE058005646F0E7D1
:10676000480001204011012000000240D807010824
:1067700016EA090F4FEA430318BF43F001035FEA2B
:106780009C07A8F8003053D10132D2B2062A40F259
:106790003F85D8454FD028F8027F3B464FF0200C6C
:1067A0003E4616EA0C0F4FEA430318BF43F00103BD
:1067B0005FEA5C09A8F80030DAD10132D2B2062AC9
:1067C0004FEA430000F22A820DEB020ED8459EF9F3
:1067D00040109EF8409040EAD176A8F800602AD098
:1067E000C9F3801328F8023F4E464FF0200A16EAFC
:1067F0000A0F4FEA430318BF43F001035FEA5A0C44
:10680000A8F80030CDD10132D2B2062A00F20082BF
:106810000DEB020E20279EF940109EF84060C80F35
:1068200040EA4303C6F3801141EA4303A8F800306D
:10683000D8457FF470AF0022CDE91222CDE91422B1
:10684000CDE91622A84E18920DF1460A35F8020F2E
:10685000A649002731F8028F00EA080E1EF00F0348
:106860000ED05A0882EA030282EA930C8CEAD3091A
:1068700000F0DD819B0814BF4B46134603F0010373
:10688000B14243EA4707E5D1AB452AF8027FDDD1A3
:10689000974B0820002280211D78BDF848B06E007B
:1068A00011EA0B0F18BF46F001061E70BDF84AA092
:1068B000F7B2951C7E0011EA0A0FEFB218BF46F03E
:1068C0000106082F1E7040F0B4815A78BDF84C7054
:1068D0005500394218BF45F0010501225D7013448F
:1068E000BDF84E701E78551C39424FEA4606EFB28D
:1068F00018BF46F00106082F1E7040F0D6815A7866
:10690000BDF850705500394218BF45F0010501220D
:106910005D701344BDF852701E78551C39424FEA21
:106920004606EFB218BF46F00106082F1E7040F071
:10693000B0815A78BDF854705500394218BF45F0FF
:10694000010501225D701344BDF856701E78551C78
:1069500039424FEA4606EFB218BF46F00106082F4B
:106960001E7040F08A815A78BDF85870550039423F
:1069700018BF45F0010501225D701344BDF85A703F
:106980001E78551C39424FEA4606EFB218BF46F052
:106990000106082F1E7040F064815A78BDF85C70C3
:1069A0005500394218BF45F0010501225D701344BE
:1069B000BDF85E701E78551C39424FEA4606EFB2AC
:1069C00018BF46F00106082F1E7040F03E815A782D
:1069D000BDF860705500394218BF45F0010501222D
:1069E0005D7013441F78BDF86280013211EA080F10
:1069F000D2B24FEA470618BF46F00106082A1E70B9
:106A000004BF0022013301384FEA51017FF444AF43
:106A1000A3787F2B00F01982677957B12046FFF7E2
:106A2000B9FB67792FB10C2F8CBF022401242744B6
:106A3000FF00DFF8CC902F48D9F8105099F830605B
:106A400095F800E06978049677447A1E92FBFEFC84
:106A500011FB0CF370331FFA83FE99F83270A0F823
:106A6000E2E4002E00F0D083C7EBC706CDE906E7CD
:106A70004FF00008C6EBC6011F4C204ADFF884A087
:106A80000591F8000294039220210123C346CDF81A
:106A900004800890059FFD180AEB450E7B180AEB51
:106AA000430CBEF9AC64BCF9AC44F11735198A0348
:106AB00042EA9641EB172A46B00300F067FC07460E
:106AC000E0178603EB1746EA94412A46A00300F03C
:106AD0005DFC0299039BCDF808A00646C2469D1EA8
:106AE0008C1E01F2FE380FE056A9000846A90008E6
:106AF0001015012040110120D80C0108D808010808
:106B00000000002024A70008B5F90200B4F902E053
:106B100006FB00F007FB0E0242F38F30FBF7C0F9D3
:106B2000B5F90430B4F9041006FB03F307FB013098
:106B300040F38F30FBF7B4F9B5F90630B4F906200D
:106B400006FB03F307FB023141F38F30FBF7A8F993
:106B5000B5F90800B4F9083006FB00F007FB0302A2
:106B600042F38F30FBF79CF9B5F90A10B4F90A002B
:106B700006FB01F107FB001343F38F30FBF790F99D
:106B8000B5F90C10B4F90C2006FB01F107FB02105B
:106B900040F38F30FBF784F9B5F90E30B4F90E10DD
:106BA00006FB03F307FB013242F38F30FBF778F962
:106BB00035F9100F34F9103F06FB00F007FB030115
:106BC00041F38F30FBF76CF944459DD1D446DDE9A4
:106BD000017A002F75D1049C0CF101080126A04513
:106BE000019677D0A64D019A05EB820EDEF8E46B94
:106BF00006EB0B0416F80B30A1780AEB830C0AEBBA
:106C00008107DCF8F806D7F8F8560290039541E7BB
:106C10009B00A8F800306646202709E6D845A8F86A
:106C200000003FF408AE28F8029F4B46DCE5012344
:106C300024E61D78BDF84C806E0011EA080F18BFDD
:106C400046F001061E7003324AE61D78BDF860A0CA
:106C50006E0011EA0A0F18BF46F001061E700232DC
:106C6000C0E61D78BDF85CB06E0011EA0B0F18BFCE
:106C700046F001061E7002329AE61D78BDF8589063
:106C80006E0011EA090F18BF46F001061E700232AD
:106C900074E61D78BDF854C06E0011EA0C0F18BFE1
:106CA00046F001061E7002324EE61D78BDF850E037
:106CB0006E0011EA0E0F18BF46F001061E70023278
:106CC00028E6049C0CF101080025A0458BF0010B7F
:106CD000019587D1DDE906E70898DFF8B8810790CC
:106CE000C31BCDE905E7C3EBC3010022A8F581660C
:106CF00004910292A8F6080B0E2103961323019229
:106D0000049D6C180AEB440C2B440AEB430EBCF9AF
:106D1000AC74BEF9AC64F817BD19820342EA97411E
:106D2000EB172A46B80300F031FBF1178C03EB1781
:106D300044EA96412A460746B00300F027FB039B2E
:106D4000ABF1020406469D1E0BF2FE3BB4F90200B5
:106D5000B5F9022007FB00F006FB020141F38F307A
:106D6000FBF79EF8B4F90400B5F9043007FB00F016
:106D700006FB030242F38F30FBF792F8B4F90610DA
:106D8000B5F9060007FB01F106FB001343F38F3052
:106D9000FBF786F8B4F90820B5F9081007FB02F2F2
:106DA00006FB012040F38F30FBF77AF8B4F90A2094
:106DB000B5F90A3007FB02F206FB032141F38F30DD
:106DC000FBF76EF8B4F90C00B5F90C2007FB00F0E6
:106DD00006FB020343F38F30FBF762F8B4F90E10A1
:106DE000B5F90E0007FB01F106FB001242F38F30EC
:106DF000FBF756F834F9101F35F9103F07FB01F186
:106E000006FB031040F38F30FBF74AF8A3459DD1F2
:106E1000029F002F40D11B4901268845029644D08D
:106E200018F8017F164A019E02EB870EDEF8E45B3C
:106E3000AC19A95DA3780AEB83000AEB810CD0F8AA
:106E4000F876DCF8F8B603975AE76779002F3FF435
:106E5000F0AD0D4F2046D7F84855FFF79BF9D7F80E
:106E60004865D4F806200948C5EB46018B1AA3FBF8
:106E70000001074A002300F0D9FAC4F80600CBE568
:106E8000F40C0108E31801084800012040420F00FB
:106E900000EE0200E0180108019DD24985F00104CE
:106EA0000022884501940292BAD1DDE90553079882
:106EB000002D00F06B8199F80C600696C71ACA4E37
:106EC0004FF0800BC7EBC704CBF3470300270197B4
:106ED000B8460B94574696F800A0002B40F033813B
:106EE00096F801E04FF0100C01364FEADE19CEF3B0
:106EF0008011CEF34013069808F104041FFA84F8B9
:106F0000002800F01681B94A1BEA0A0F02EB830A37
:106F100002EB8101DAF8F00B0A9014BF0120002087
:106F200002EB890B02EB800ECDE90C58CDE90E6C1B
:106F3000D1F8F04BDBF8F03BDEF8F02B08930021A2
:106F4000099407920591019DA94E079B089C0998F9
:106F50000A992E4496F8E88A96F8EB9A96F8EEAAE3
:106F600096F8F12A96F8F45A08EB480C9C4409EB81
:106F7000490B96F8F73A1CF8055096F8FACA96F8B5
:106F8000FD6AA3440AEB4A0E864402EB42081BF852
:106F900003400B9A049488441EF80C1018F80660FD
:106FA00003915019131907EB430B541807EB4009D1
:106FB00007EB440E9119BBF9ACA4B9F9AC04BEF9C6
:106FC000AC84029607EB410C0AEB0002BCF9AC64FE
:106FD0004244C317B41899032246E31741EA90418B
:106FE000800300F0D3F983464FEAEA70820342EA55
:106FF0009A41E31722464FEA8A3000F0C7F94FEA78
:10700000E87399032246E31741EA984182464FEA22
:10701000883000F0BBF92246E317F4178146A0033D
:1070200040EA9641B00300F0B1F9049E039A029B36
:1070300007EB820407EB850507EB860807EB830166
:10704000D5F8F826D8F8F866D4F8F856D1F8F84606
:107050000297023E023D023CA2F1020802F2FE3318
:107060000746B8F902E0B6F90200B5F90210039339
:107070000BFB0EFC0AFB00C2B4F9020009FB012362
:1070800007FB003242F38F30FAF70AFFB8F9041019
:10709000B6F904000BFB01F3B5F904100AFB00324A
:1070A000B4F9040009FB012307FB003242F38F30DF
:1070B000FAF7F6FEB8F90610B6F906000BFB01F375
:1070C000B5F906100AFB0032B4F9060009FB0123EA
:1070D00007FB003242F38F30FAF7E2FE38F9081F5F
:1070E00036F9080F0BFB01F335F9081F0AFB0032D4
:1070F00034F9080F09FB012307FB003242F38F30FC
:10710000FAF7CEFE039B9845ABD1DDE90167059CFC
:10711000069B0136F5B2032D04F1010408BF0025DA
:107120009C42059401957FF40EAFDDE90C58DDE932
:107130000E6C45452AD9E346CBF3470396F800A0E9
:10714000002B3FF4CDAE13EA0A0F14BF4FF0010934
:107150004FF000091BF47F7FCBF3870007D17078D5
:107160004FF0200C0136C109C0F38013C3E610EACA
:107170000A0FCBF3C70314BF01210021002B59D103
:1071800074784FF0400C0136E309B4E6FAF7CCFE10
:107190001849D1F84003D1F8442382420FD0164F4A
:1071A000164D1026BE612C6924F004032B6130BFFC
:1071B0001049D1F84003D1F844239042F2D10E4F48
:1071C0000C4B0F4D0F484FF48016BE61D3F8481595
:1071D0004FF00064AC61C0F8941121B0BDE8F04FED
:1071E000FCF798BCE318010810150120F40C010805
:1071F000FCFB0008480001200008024000ED00E010
:107200000000024040110120DFF848A0F80064E5CA
:10721000D8453FF410AB0DEB020999F8407099F98D
:107220004060C7F3801AF30F4AEA430328F8023F8D
:10723000FFF7B4BA13EA0A0F14BF012300231BF4AB
:107240007F6FCBF3071C7FF456AE01364FF0800CF6
:1072500051E600BF24A700082DE9F843364A374C11
:107260005369374FDFF8F090054683F0020040F491
:107270000031916104F2E4404FF42A72002102F0DF
:107280000FFF4FF0000C2F492F4B304A84F88CC76A
:10729000A4F890C704F2947004F2A47E4668D0F873
:1072A000008003EB850302EB8502B342026040D00D
:1072B00043600022CEE90022CEE90222A1F500536C
:1072C000C3E90022C3E90422C3E90822C3E90C226E
:1072D000C3E91022C3E91422C3E91822C3E91C221E
:1072E00080338B42ECD1BCF1000F13D157F8046FFF
:1072F00096F80080B37809EB880209EB8306D2F890
:10730000002BD6F8003B083008310EF1100E4FF07C
:10731000010CC3E7084E0E4D0E4A0420B06171699E
:10732000C4E9145281F0020747F40033B361BDE8A9
:10733000F8834245D7D0BCE7000802404011012045
:10734000D81801083C4D0120E4D60008E4B6000836
:10735000DB1B0400B9A20100FCFB000808B5094BC7
:10736000094993F8322000F8012B01EB820C7E22B0
:10737000DCF8101C02F0D8FE00F022F90130C0B297
:1073800008BD00BF00000020F40C01087BB972B9F1
:107390000029BEBF00204FF0004106E008BF0028D2
:1073A0001CBF6FF000414FF0FF3000F057B8ADF157
:1073B000080C6DE904CE002909DB002B1ADB02F072
:1073C000DFFCDDF804E0DDE9022304B07047404251
:1073D00061EB4101002B1BDB02F0D2FCDDF804E085
:1073E000DDE9022304B0404261EB4101524263EB0C
:1073F00043037047524263EB430302F0C1FCDDF8E4
:1074000004E0DDE9022304B0404261EB4101704732
:10741000524263EB430302F0B3FCDDF804E0DDE924
:10742000022304B0524263EB4303704753B94AB995
:10743000002908BF00281CBF4FF0FF314FF0FF307C
:1074400000F00CB8ADF1080C6DE904CE02F098FC28
:10745000DDF804E0DDE9022304B07047704700BFA7
:10746000844641EA000313F003036DD1403A41D34F
:1074700051F8043B40F8043B51F8043B40F8043B0E
:1074800051F8043B40F8043B51F8043B40F8043BFE
:1074900051F8043B40F8043B51F8043B40F8043BEE
:1074A00051F8043B40F8043B51F8043B40F8043BDE
:1074B00051F8043B40F8043B51F8043B40F8043BCE
:1074C00051F8043B40F8043B51F8043B40F8043BBE
:1074D00051F8043B40F8043B51F8043B40F8043BAE
:1074E00051F8043B40F8043B51F8043B40F8043B9E
:1074F000403ABDD2303211D351F8043B40F8043B3E
:1075000051F8043B40F8043B51F8043B40F8043B7D
:1075100051F8043B40F8043B103AEDD20C3205D34D
:1075200051F8043B40F8043B043AF9D2043208D045
:10753000D2071CBF11F8013B00F8013B01D30B88B7
:1075400003806046704700BF082A13D38B078DD095
:1075500010F003038AD0C3F10403D21ADB071CBF67
:1075600011F8013B00F8013B80D331F8023B20F8D1
:10757000023B7BE7043AD9D3013A11F8013B00F80A
:10758000013BF9D20B7803704B7843708B78837092
:10759000604670470000000000000000000000008E
:1075A00000000000000000000000000000000000DB
:1075B00000000000000000000000000000000000CB
:1075C00030B490F800F020F007016FF0000C10F0DC
:1075D000070491F820F040F048804FF000046FF06D
:1075E0000700D1E9002391F840F000F1080082FA89
:1075F0004CF2A4FA8CF283FA4CF3A2FA8CF34BBB54
:10760000D1E9022382FA4CF200F10800A4FA8CF2CC
:1076100083FA4CF3A2FA8CF3E3B9D1E9042382FA9A
:107620004CF200F10800A4FA8CF283FA4CF3A2FAAF
:107630008CF37BB9D1E9062301F1200182FA4CF2E7
:1076400000F10800A4FA8CF283FA4CF3A2FA8CF34E
:10765000002BC6D0002A04BF04301A4612BAB2FA70
:1076600082F200EBD20030BC7047D1E9002304F075
:107670000305C4F100004FEAC50514F0040F91F8AA
:1076800040F00CFA05F562EA05021CBF63EA050347
:1076900062464FF00004AAE72DE98048D5B072B6E3
:1076A0000025CB4C1595236B43F001002063216B23
:1076B00001F001021592159B1495266B46F0020706
:1076C0002763236B03F002001490149A1395216B27
:1076D000C04841F004022263266B309506F004078F
:1076E0002EA901261397139B31952F962E96F8F706
:1076F000A5FF4FF48033022283614FF400372E92AE
:107700004FF0040BF8F79AFF87614FF40069CDF84A
:10771000B8B0F8F793FF4FF48023836148444FF0EB
:107720000068CDE92F653195CDF8B8904FF0080A83
:10773000F8F784FFC0F81880A0F50060CDE92F6548
:107740003195CDF8B8A0F8F779FF4FF400228261A7
:10775000CDF8B890F8F772FF4FF04009C0F81880E4
:10776000CDF8B890F8F76AFF4FF4800383614FF0CB
:107770008008CDF8B880F8F761FF4FF4000282610D
:107780004FF4805CCDF8B8C0F8F758FF4FF0805345
:1077900083611295D4F830C04CEA0B0CC4F830C0A9
:1077A000D4F830C032950CEA0B0CCDF848C01298D2
:1077B0002F964FF4806000F180422E9002F5013048
:1077C000CDE93056F8F73AFF02232E93F8F736FF4B
:1077D000CDF8B8B0F8F732FFCDF8B8A0F8F72EFF23
:1077E00010222E92F8F72AFF20232E93F8F726FF77
:1077F000CDF8B890F8F722FFDFF8E491CDF8B88023
:10780000F8F71CFF4FF480722E92F8F717FF4FF431
:1078100000732E93F8F712FFC9F85051C9F8485178
:107820004FF0806585614FF4802187614FF48012AD
:107830004FF4002781614FF4001387614FF48005F6
:1078400082614FF400014FF080774FF00072836146
:10785000856181618761826199F879314FF080405B
:1078600011251821C9F84001C9F84C51C9F8441133
:10787000002B00F05B855849022589F87951F9F70A
:107880000DFA5648C9F8F45001264AF6C8734FF469
:10789000FA7189F879618362C162C660066000246A
:1078A00000F550534FF4827799F83501C9F8EC4050
:1078B000C9E94144C9F8F840C9F80C41C9F8E87071
:1078C0004FF40064082207214FF40077C9F8F04014
:1078D000C9F8E430C9F80021C9F81011C9F8FC70E2
:1078E00000F0FF04002801F057824FF0020889F8E9
:1078F0003581186820F040011960D9E93A75D9F846
:10790000F060D9F8F440D9F8F830D9F80001D9F886
:107910000411D9F8E4202F43374327431F43D9F8F4
:107920000C51D9F8FC6007430F4306F400742F4351
:1079300027431760B9F8FE70D9F80801D9F8E42098
:10794000234C07F0040303435360D16921F400651D
:10795000D56101260025C9F8385189F8356111959E
:10796000276B37432763206B30401190119A109595
:10797000226B32432263236B33401093109B0F958D
:10798000616C41F010076764606C00F010020F92A8
:107990000F9B0E95236B43F480012163276BCDF879
:1079A000BC8007F480004FF400720E90072709484E
:1079B0002E922EA94FF4806B4FF0120A0E9B329735
:1079C000CDE93056F8F73AFECDE930560AE000BF6F
:1079D00000380240000002408C01012000040040F9
:1079E00048000120CDE92EBA3297F8F727FED04B98
:1079F000D048C9F89C52C9E9A35B4FF000614FF42D
:107A000080374FF0400BC9E9A031C9E9A555C9F845
:107A1000A452C9F8A072C9F888B2F8F731FC4FF047
:107A20000062C549C9F8E4224FF480634FF48072C4
:107A3000C9F80073C9F83400A0F51F776030C9E9B0
:107A4000BC35C9F8E012C9F8FC22C9E9BA55C9F831
:107A5000F852C9F80453C9F8B872F8F711FCDFF806
:107A600048C3C9F838000C234FF4E130C9F8183086
:107A7000C9E901C0C9E90355C9E90755C9F818732F
:107A8000C9F81450AD4FFBF7EDFA2A460321252023
:107A9000F8F7C8FB20212A46796046202946F8F7E6
:107AA000C1FB2A4629464420C7F808B0F8F7BAFBBC
:107AB000C9E91855C9F858501025BD604FF48042E7
:107AC00099F881109E4B9F48C9F854205E25C9F84B
:107AD0004C20FE22C9F85050C9E91130C9F85C2089
:107AE00001F0FF05002901F08780974E01962427B9
:107AF00089F881701C6824F001021A60934B4FF4DE
:107B0000E0509D6890FAA0F1914C924B924AB1FAE4
:107B100081F605F4E057F74027441E6897F868049B
:107B2000C640A2FB0615D9F844008C49AF0C47604B
:107B3000D9F848408C4200F2CF830137076240F603
:107B4000FC776500B6FBF5F33B4208BF0423C36135
:107B5000D9E9186426430660D9E91412D9F844001B
:107B60000A438260D9E916352B43C36007687C4914
:107B700047F00106066000242020C9F8844089F8F7
:107B80008100C9F8744089F8824004F1804CD9F82A
:107B9000D850C9F8A0400CF590364FF48032012738
:107BA000C9F8A840C9F8B040C9F8B840C9F8C440FD
:107BB000C9F8A440C9F8C840C9F89860C9F8C0100D
:107BC000C9F89C20C9F8AC70002D01F05F81D9F88C
:107BD000D870FC0640F1CA8600230127219389F85A
:107BE000D4703069019C20F0E06535613169C4F8DA
:107BF000887841F000723261706B20F01F05756368
:107C0000716B41F00802726389F8D430554B082635
:107C10000220C4F88468C4F88C0880259E614FF463
:107C2000006440264FF480519C619E619D61996182
:107C300099F88120202A00F063874B4C20460025CC
:107C4000FF26012189F86B5789F86867FAF7B4FABB
:107C5000A9F86907434C4FF480014FF00060A1611F
:107C6000A061F9F78DFA72B63A4A404B536062B69A
:107C70004FF480374FF400354FF480264FF4002145
:107C80004FF400004FF08053A761A561A661A16188
:107C9000A061A361019C94F894784FF0000A89F8E0
:107CA000E4A789F84EA5002F00F0E886304C019A31
:107CB0003048C2F8B00E04F1980CC9F8F4C704F5C6
:107CC000987CC9F8F8C704F5E47CC9F8FCC704F54A
:107CD000187CC9F800C804F53E7CC9F804C8264FD2
:107CE000264E274B27492848C2F8BC7E04F5647C01
:107CF000C2F8C06EC2F8C43EC2F8C81EC2F8CC0EAC
:107D0000C9F808C8214F224E224B23492348C2F804
:107D1000D07E04F5856CC2F8D46EC2F8003FC2F87C
:107D2000041FC2F8080FC9F80CC81D4F1D4E3DE0D6
:107D3000B8640240C80201208864024000E100E00B
:107D400000540040801A0600401101200038024013
:107D500024A700080000002083DE1B43A08601004A
:107D60000100000F00000240B3070120951F00082A
:107D7000001A0120952700085D210008014A00082B
:107D80001121000849210008D123000869250008B5
:107D9000352300083D24000825210008F547000888
:107DA000E125000861420008001001408A4B8B4920
:107DB0008B48C2F80C7F04F5986CC2F8106FC2F8BB
:107DC000143FC2F8181FC2F81C0FC9F810C8854F1D
:107DD000854E864B86498748C2F8207F04F5AB6CF8
:107DE000C2F8246FC2F8283FC2F8301FC2F8340F1F
:107DF000C9F814C8804F814E81488249824B834D17
:107E0000DFF8BCE2DFF8BC82DFF8BCA2DFF8BCB26E
:107E1000C9F8F0474FF00A0C89F818C8C2F8387F43
:107E2000C2F8506FC2F8780FC2F87C1FC2F8903FBA
:107E30001046774F774E7849784BC2F8747FC2F876
:107E4000806FC2F894EFC2F8B08FC2F8B41FC2F8C6
:107E5000B8AFC2F8BCBFC2F8C03F714F714A724E92
:107E60007249734BC0F8C42F45F8487C45F83C6C08
:107E700045F8381C45F8343C6E4A6F4F6F4E7049D8
:107E8000704B45F8302C45F82C7C45F8286C45F8AB
:107E9000241CAB606C4A6D4F6D4E6E496E4BEA60B0
:107EA0002F616E61A961EB616C4A6D4F6D4E6E4939
:107EB0006E4B2A626F62AE62E9622B63D9F804707E
:107EC0006B4AF9686B4EAA6341F02003FB606A4A73
:107ED0006A4F6B496B4BEE632A646B4E6B4AAF651E
:107EE0006B4FEE67C5F880106A4E6B49C5F8843059
:107EF000C5F88820694B6A4AC5F89870694FC5F87B
:107F00009C60C5F8B810684E6849C5F8BC30C5F823
:107F1000C020674B674AC5F8C470674FC5F8C86092
:107F2000C5F8CC10C5F8B831C9F87C22C9F8247856
:107F300062B6624EDFF898B18021B1614FF0000E59
:107F40000127A4F2046480F849E089F84F750DF127
:107F50003608FBF78DFDFBF7DDFD89F83E710B94CC
:107F600095F8BC61002E00F0D281012E00F0B6829F
:107F7000022E01F00D8099F88907002800F0528147
:107F8000D9F88C27D9F86437B9F890779C1AA0B241
:107F9000B842C0F04781B9F892673A44941BC21BBB
:107FA000B118B1F5004F00F29482982200212EA85A
:107FB00002F076F84FF0A00A99F88807ADF8C17082
:107FC0000523D9F80070ADF8BF608DF8BD308DF88D
:107FD000BE008DF8BAA085E0A14200087527000810
:107FE000ED22000841270008852100085D390008BE
:107FF0006D24000871250008E94200089923000853
:10800000853E0008554200087123000838220120EF
:10801000853C0008B53D0008ED4C0008F12400083F
:10802000D54B0008DD4F0008014C0008A9210008CD
:108030000121000845210008CD2300086D25000816
:1080400025230008152400081521000889210008AF
:10805000B5250008F1200008ED230008612700087D
:10806000C12200085D73000861210008D9230008BF
:10807000ED24000899250008B125000875230008A3
:108080003D27000835270008312700083927000858
:10809000A9280008114D00086D220008BD22000823
:1080A0003D2600082D270008F52400086525000856
:1080B00071500008652D0008F92C000800000240EE
:1080C00011240008B922000839260008F94F0008D9
:1080D00000ED00E0D9F80000C11B642900F2D08156
:1080E0009DF8BD300633D9B22EA8F9F78BF80028D9
:1080F000F0D0002E00F08880C4F30E0A00272EAACC
:1081000000230AF10101B74207F101041FFA81FCC3
:1081100062D2BD4F11F4004F37F81A00D07108BF7A
:10812000E246A7B218BF4FF0000A4FEA102EB7423E
:108130000AF1010007F1010482F806E01FFA80FC51
:1081400003F1020348D2B04910F4004F31F81A107D
:10815000517208BFE246A7B218BF4FF0000A4FEABB
:10816000112E0AF10100B74207F1010482F808E07C
:108170001FFA80FC03F102032ED2A34F10F4004F2C
:1081800037F81A10D17208BFE246A7B218BF4FF0F5
:10819000000A4FEA112E0AF101000233B74282F8B9
:1081A0000AE007F101041FFA80FC03F1020E13D26A
:1081B000954B33F81A70577310F4004F1FFA8EF373
:1081C0004FEA17210CBFE2464FF0000A802B1173D3
:1081D000A7B202F1080294D1D9B2D9F800408DF8C3
:1081E000BD1007E0D9F80020101B642800F2F684C7
:1081F0009DF8BD100631C9B22EA8F9F703F8002882
:10820000F0D0B742FFF47BAF804E7F4AB468A01A2B
:1082100000234110C9F8641789F88937C9F88C37E9
:1082200089F88837019E96F8F510002940F0CA8039
:10823000019991F8F870002F40F0A38099F8ED278C
:10824000002A3FF48DAE99F8EF6799F8EC07D9F85A
:10825000E817731CDCB2A04298BF3C4602F1FF3A1B
:1082600089F8EDA789F8EF4751F8264094F90220E4
:10827000A078BA42C0F23386394698222EA801F07F
:108280000FFFFF2799F86B678DF8B8608DF8BA700B
:1082900060788DF8B90094F804A0D9F800608DF8E2
:1082A000BCA005E0D9F80000831B642B01F24D85CA
:1082B0009DF8BD3006332EA8D9B2F8F7A3FF0028E9
:1082C000F0D099F86B17524F21702046FEF7DAF97B
:1082D0008022BA6101F0F8BC4FF49672D9F84C30A4
:1082E00002FB07F74FF47A7EB7FBFEF50135056216
:1082F000002B00F0E180192707FB04F4B6FBF4F62D
:10830000C6F30B04002C40F0EA8601231FE44FF46F
:10831000006231463F4801F0C3FE01273046C5F8F0
:10832000C069FEF799FF85F8BC7124E603F0FF07EA
:10833000179789F87871206C30432064226C3240A2
:10834000179231463A461C20179BF7F76BFF3246CF
:10835000314E4FF0805333601697256C45F0020183
:108360002164246C04F0020716971D200921169B36
:10837000F7F758FF4FF00052D9F840013260FFF78D
:108380007ABA019AD9F884474FF0000A82F8F8A027
:108390008CB1D9F84805D9F848351E1AB4420AD923
:1083A0001E490F6927F004020A6130BFD9F8483529
:1083B0001E1AB442F5D81A48154CFEF763F980200E
:1083C000A061CDE596F8F72096F8F440D6F8F000D5
:1083D000531CDFB2BC4298BF002701F1FF3C86F876
:1083E000F77086F8F5C050F8224094F805E0D4F80C
:1083F0008660A644CEF80660B4F88A10D9F80070FA
:10840000AEF80A1013E000BF440000200000002076
:1084100000080240F823012000E100E000ED00E048
:108420003C120120D9F80010CA1B642A36D86279A0
:108430000C322046D1B2F8F7E5FE0028F2D099F8C8
:108440001838092B06D809EB830A0133CAF8F0471C
:1084500089F81838019C94F8F570002F7FF4E8AE85
:1084600099F8820701287FF4E3AE07F1804C0CF500
:10847000023E4FF0006689F88377CEF81860D7E6A1
:10848000C34D08264FF40062402480274FF48050EB
:10849000AE61AA61AC61AF61A861FEE7BC4D082383
:1084A0004FF40066402080244FF48057AB61AE61EA
:1084B000A861AC61AF61FEE704EB4401B6FBF1F8E3
:1084C000C8F30B02002A3FF420AF48F40043FFF743
:1084D0003EBB1444A9F89007074666E5AD48C26A5A
:1084E00090F83130C78A069302F57F563F3616EA78
:1084F000220638BF1646B413019E04940597002443
:10850000D9F85C15D9F8600581423FF434AD2EA846
:10851000F9F79CFD96F88C27D9F85835B5F8C8A915
:1085200002935AB102EB820706EB870C0299DCF842
:10853000DC040B1AB3F5806F00F21282D6F8943780
:10854000954F981C07EB0A111F46C6F8940737F899
:1085500004EBC6F89477B3F802C0BDF9B8301EFB3F
:1085600003F040F38F301CFB03F70390B1F90200D6
:1085700047F38F374F804FEA0A1CA7EB000E864F58
:1085800037F90C000790039827F80C00079FA0EB21
:10859000070CD6F8A407D6F898776044C6F8A40765
:1085A000D6F8A8077044C6F8A80707F1020E3846A7
:1085B000C6F898E730F804CBC6F898071CFB03F020
:1085C0007F8840F38F3EB1F90400A1F804E017FB67
:1085D00003FCAEEB000EB1F906004CF38F37CF80F1
:1085E0003F1AD6F8AC07D6F89CC77044C6F8AC075B
:1085F000D6F8B00707446046C6F8B0770CF102071A
:10860000C6F89C7730F804EBC6F89C07BCF802006B
:108610001EFB03FC10FB03F7B1F908004CF38F3E7F
:10862000A1F808E0AEEB000EB1F90A00D6F8A0C739
:1086300047F38F374F813F1AD6F8B4077044C6F816
:10864000B407D6F8B8070744C6F8B87760460CF107
:108650000207C6F8A07730F804EBC6F8A007BCF80C
:1086600002C01EFB03F71CFB03F083FB033C9B0BC8
:1086700005EB8A0E43EA8C43B1F90CC047F38F3700
:1086800040F38F308F81A7EB0C0CB1F90E70C881CD
:10869000DEF8C011CEF8C0315B1AD6F8C017C01B87
:1086A0000844D6F8BC77C6F8C007D5F8C0096744B7
:1086B0000344C6F8BC77C5F8C039571C03F580736E
:1086C000CDE9082A07930397134692460CE0DCF89D
:1086D000EC340133CCF8EC3403980AF101011FFAB1
:1086E00081FA5045534659DB0AF0010206EB021E9F
:1086F00003EB8301DEF8AC77DEF8A407DEF8B027E1
:10870000CDF828A006EB810CDEF8A81787FB077EC2
:10871000BF0B47EA8E4782FB022E920B42EA8E4E37
:10872000774481FB011E8A0B42EA8E4280FB000ED9
:10873000810B41EA8E400244DCF8E4041744079AB6
:1087400097FBF2F181424FEA8307C0DD10B9029A2C
:10875000CCF8F4243B4406EB830C039FCCF8E414E0
:108760000AF10101CAB20298CCF8F004BA428CF8BE
:10877000E844CCF8EC44AFDC02EB820E013206EBAD
:108780008E03D2B29742C3F8E444F5DAA4E700BFFF
:1087900000000240000000203C2D0120DDE9082CF3
:1087A00002EB820706EB870E049BDEF8E4148B4293
:1087B00031DD0CF10100C0F30800A5F8C80900285C
:1087C0007FF49EAEC24B96F890A796F891E7C14809
:1087D0009A449E449AF8F81B9AF8FA7B00EB810CB5
:1087E00000EB870A9EF8FC1B9EF8FE7BDCF8002B52
:1087F000DAF8003BC6F8942700EB810E00EB870007
:10880000DEF8002BC6F89837D0F8003BC6F89C2756
:10881000C6F8A03774E6DEF8EC340599AE48AF4FE1
:108820008B42C6E914070BD2002AC2D0D6F8F03426
:1088300002984FF0800AC71A0AEB42239F42B8D928
:1088400012F00107A64914BF04234FF480238B6163
:10885000F1199F4B0CF1010003EB870C91F8903755
:10886000DCF8E4EB0133DBB2022B08BF002381F814
:1088700090371EF803A0974901EB8A0C73440293CA
:10888000DCF8003B0299C0F3080C06EBC70A03EBC7
:108890008C0ECAF894E78B788E4901EB830EDEF8D4
:1088A000003B03EB8C018F4BCAF8981703EBC7030F
:1088B00003F5005C0CF1100A10339E4643E90444B2
:1088C0004EF8104B4EF80C4C4EF8104B4EF80C4C2A
:1088D000C3E90844C3E90C44C3E91044C3E91444A0
:1088E000C3E9184480335345E7D17F4901EB0713AF
:1088F0003F011F2ACC51C3E90144DC6006D809EBD3
:108900004202B2F8A4170131A2F8A4179DF80C3066
:10891000069A86F88C37142707FB036C9342CCF831
:10892000EC44FFF448AF019C0022D4F8F0046F4CF3
:10893000924602E0E668311A8A440132D6B2B34266
:1089400004F11404F6D8BAFBF3FC013300EB032165
:1089500061440227C5F8C41985F8BC71FFF70BBB49
:108960005046FEF779FC96F88C27E7E5D9F8D83021
:108970005F4DD9F89C2023F4885424F0020040F085
:108980000201C9F8D8106F6827F440336B606C6837
:1089900014436C60706820F4807171607568D9F858
:1089A000A82045EA02277760736823F0407474605A
:1089B0007068D9F8A0104F4C08437060B56825F472
:1089C0000062B260B768D9F8A4301F43B760B168DD
:1089D000D9F8C00021F07065B560A042B26800F01F
:1089E000D382D9F8C0301A43B260B46824F0405042
:1089F000B060B568D9F8C4100D43B560B26822F014
:108A00000207B760B368D9F8B04043EA4400B060E9
:108A1000D9F8B850002D40F0A182716821F40062AD
:108A20007260F46AD9F8B45024F47000F062F16A0C
:108A300005F1FF3E41EA0E52F262B76827F4007377
:108A4000B360B468D9F8C80044EA4025B560B1689D
:108A500021F48062B260B768D9F8AC30002047EAF0
:108A60008324B460C9F8DC00D9F8D85025F003019C
:108A700041F00102C9F8D820FFF7AEB81E4AC9F884
:108A8000E8270125052684F89458C9F8EC673B4689
:108A9000D9F8E81741F82730013799F8ECC7F8B250
:108AA0008445F5D8019F154CC7F8F04005220025F4
:108AB000C7F8F4202E46D7F8F03043F8256001358A
:108AC00097F8F4105FFA85FB5945F4D8FFF7EEB834
:108AD000F40C0108FCFB0008DB1B0400B9A2010038
:108AE000000802403C2D0120E4180120241601203A
:108AF000002301400100000FD8190120EC190120CA
:108B0000D9F8005099F88130202B7FF496A8394687
:108B100098482B461922F7F73DFF014600287FF4BD
:108B20008CA899F8800001283FF487A8D9F8444020
:108B300089F880702268904822F400632360D9F895
:108B40004440222289F8812089F88260C9F8841083
:108B5000C9F87000266846F480602060D9F8444067
:108B6000226842F480762B4626603A464FF0011088
:108B7000F7F710FF58BBD9F844108048A0230B61C9
:108B80002A463946F7F7A0FF002841F05080D9F86F
:108B90004440249062692492A66924962846249B26
:108BA000F8F718F848B9D9F8441008612846F8F7DA
:108BB00011F80146002801F02180D9F88410042919
:108BC00005D1D9F84400036843F40072026000271D
:108BD000D9F8842089F88070FFF72FB8684D0827EE
:108BE0004FF40063402480264FF48052AF61AB61A4
:108BF000AC61AE61AA61FEE7209589F88050216BD7
:108C000041EA08032363206B00EA08022092209ABD
:108C10001F95216B41EA08032363206B00EA0802D9
:108C20001F921F9A1E95216C41F400132364206C3F
:108C300000F400121E921E9A1D95216B41F4001340
:108C40002363246BCDF8B8B004F400101D90042405
:108C50004C481D9A31962EA9CDE92FA53294F7F7ED
:108C6000EDFC8022CDE93056CDF8BCA032942E9296
:108C7000F7F7E4FC444B454CC3F8CCB79A464FF4A5
:108C800080614FF000720AF2C470C3F8D057C3F885
:108C9000D417C3F8D857C3F8DC57C3F8E057C3F864
:108CA000E457C3F8E857C3F8C447C3F8C8274FF4DC
:108CB000001403234FF4000BCAF8EC37CAF8F4474A
:108CC000CAF8F0B7CDF804A0F7F7DAFA019BC9F8B3
:108CD00078009A464FF000714FF48062C3F828186C
:108CE000C3F8342803232A4ACAF84C3860304FF4BA
:108CF0000033CAF85448274CCAF84438CAF82C58EC
:108D0000CAF83058CAF83858CAF83C58CAF8405817
:108D1000CAF84858CAF82428CAF850B8CAF8FC4714
:108D2000F7F7AEFAC9F87C0001983246C0F85C4803
:108D300041462F20F7F776FA2A464FF40045414680
:108D40000B207D60F7F76EFA4FF400613246202069
:108D500039604146F7F766FA7E60424641461F2079
:108D60004FF00046F7F75EFA3E60D9F84430FEF760
:108D7000BEBE00BF020010000000FFFF02000100A5
:108D8000000002400004024040110120B86002408F
:108D9000106002408C00012003F5003E1C9489F80D
:108DA0003441DEF830302B43CEF83030DEF830007E
:108DB00028401C901C9A1B94DEF830202A43CEF8E1
:108DC0003020DEF8301029401B911B9A1A94DEF8EF
:108DD00030302B43CEF83030DEF8300028401A9087
:108DE0001A9A1994DEF830202A43CEF83020DEF8A3
:108DF000301029401991199A1894DEF8403043F444
:108E00008040CEF84000DEF84020B7482E9702F4AC
:108E1000804118912EA9189BCDE92F643196F7F760
:108E20000DFC87614FF480672E97F7F707FC876189
:108E30004FF480572E97F7F701FC87614FF40053EA
:108E400005272E93CDE92F5431963297F7F7F6FB8D
:108E50004FF40042CDE930462E922F953297F7F726
:108E6000EDFBCDE931672F95A04E30944FF480454E
:108E70002E95F7F7E3FB2246214624201024F7F72E
:108E8000D1F9D9F8E4307460FEF72FBD06F58C3ABD
:108E9000C9F8DC5089F8D4502295DAF8443043F40C
:108EA0008074CAF84440DAF844002E9700F48071C8
:108EB00022918D48229B03262EA9CDE930572F966B
:108EC000F7F7BCFB2A460921884D1220F7F7AAF9CB
:108ED0004FF480222A60D9F89860FEF778BE019B93
:108EE00080F0800A03EB8A0CDCF8B02E002A00F038
:108EF000298720469047002800F0E38639469822CB
:108F00002EA801F0CDF805EB8A00A17850F8487C36
:108F10008DF8BA100DF1BE00B847D9F800708DF881
:108F2000BD009DF8BD3006332EA8D9B2F8F76AF916
:108F3000002840F0C986D9F80020D01B6428F0D959
:108F40006B4D08244FF40063402680214FF4805776
:108F5000AC61AB61AE61A961AF61FEE7776847F4D0
:108F600000637360746824F4604070604FF460457F
:108F700095FAA5FBD9F8BC207368BBFA8BF1571E94
:108F80008F401F4377604CE522F04057B76035E5CE
:108F9000D9F85C05D9F86035984202D02EA8F9F7C7
:108FA00055F8D5F8C429D9F858158A427EF4E3AFAC
:108FB000B9F86E7799F888474E4B013700264FF481
:108FC0000000022CA9F86E7785F8BC61986100F06A
:108FD0001D81494C474894F8316094F830A04749C6
:108FE0000136BAEB060248BF0332C2F387070223F9
:108FF000FF2F8361259100F0FE803F4CE36A03F56B
:109000007F5000263F30B342A8BF18468213059216
:109010003B483C4ABE464FF0000A4FF0010CCDE9F8
:1090200002CACDE9066E25AF04970026CDE92E666B
:10903000CDE93066C5F8C069CDE927204FF4007648
:1090400039E04046F9F702F82799B8F900302E9A2E
:109050000C46013E34F8040B279410FB03F747F34A
:109060008F3010442E904988289F2F9A11FB03F4CB
:1090700044F38F3111443C462F9134F8042B28944B
:1090800012FB03F444F38F32309C224430927F88E9
:1090900017FB03F444F38F3783FB03349B0B43EA42
:1090A0008443D5F8C0492344319CC5F8C0392744CE
:1090B000B6B2319746B3D9F85C15D9F860458C4201
:1090C000BFD1DBF8103023F00400CBF8100030BF24
:1090D000D9F85C25D9F86075BA42B2D1F1E746F407
:1090E0004043FEF734BD00BF0004024000E100E051
:1090F00000000240000802400000002001000001C2
:10910000E4DE0008E4BE000887FB0774BF0B47EAF3
:10911000844E82FB0224970B47EA844C81FB0114A6
:109120008A0B42EA844780FB0004810BE64441EA53
:10913000844C6744029ABE44059F03F580739EFBEE
:10914000F3F39F42CCBF002202F001020292BAF177
:10915000000F1CD104990DF197068E424FF0010AC1
:109160001FD011F8017F824A039B049102EB870C08
:109170008049DCF8E40BC618C45CB77801EB840EB8
:1091800001EB870CDEF8002BDCF8000B4DE70398B1
:109190000499B2460DF1970680F001048E420394C3
:1091A000DFD1029BDDE9066E002B3CD1B64522D013
:1091B0009DF894A06E4A6F4902EB8A0C0136DCF8E8
:1091C000E47B3878BC7801EB800301EB840AD3F8A8
:1091D000002BDAF8000B1EE7B9F87807664A013071
:1091E000A9F87807536983F0800646F40004946177
:1091F000614902278F61019A6048614B5E4C4FF4D0
:109200000036C2E91403A661FEF7B5BE99F88927B6
:10921000002A7FF4DEAED9F86417C9F88C1701274D
:1092200089F88977D5E6B9F87077F4B20137062C5A
:10923000A9F8707706D809EB4606B6F894170131FD
:10924000A6F89417D9F84805D9F85C25D9F86035FF
:10925000494C4C4903449F1A4FF40036C5F8CC7969
:10926000A6618A46086C9822002100F019FF4FF48D
:1092700089720021444800F013FF019A0B989AF874
:109280000C70CAF83C00FF2682F8A0619FED367B87
:10929000D9F85865C5F8D0690023019EA2F8B83204
:1092A000042103204FF0020AC2E96933C2F89C315D
:1092B00082F8A13182F8997182F8AC1182F8A30189
:1092C00082F8A2A14FF480104FF400114FF48002F5
:1092D0004FF400034FF4002786EDAC7BA761A0613B
:1092E000A161A261A361FBF7C9FF1B24093CA4B2E1
:1092F000FBF7C4FFFBF7C2FFFBF7C0FFFBF7BEFFA6
:10930000FBF7BCFFFBF7BAFFFBF7B8FFFBF7B6FFB5
:10931000FBF7B4FF002CE9D1174F1B4A4FF0000EAA
:1093200020200821B8618023CDE92744CDE92944D4
:10933000CDE92B442D940991ADF828402746764677
:10934000ADF808407046A246ADF80CE0ADF810400C
:10935000ADF814E0ADF81840ADF81CE0ADF820E031
:10936000C1E000BFAFF3008000000000000000007B
:10937000F40C0108FCFB000800080240DB1B0400A1
:10938000B9A2010000000020FC13012092F9013075
:109390000899DB0F43EA410C0132ADF89EC0ADF8ED
:1093A00020C0402311787F000B4218BF47F001070F
:1093B0005FEA530EADF8A07040F0C18092F901E071
:1093C000760046EADE76ADF8A260013240230299CB
:1093D00092F800C0490013EA0C0F18BF41F00101D8
:1093E0005B08ADF8A410ADF8081040F0C18092F908
:1093F00001C0400040EADC70ADF8A60001324FF039
:10940000400E13784FEA4A0A1EEA030F18BF4AF0CB
:10941000010A5FEA5E03ADF8A8A040F0BF80039B9D
:10942000590092F9013041EAD371ADF8AA10ADF8B4
:109430000C1001324023049992F800E0490013EA2D
:109440000E0F18BF41F001015B08ADF8AC10ADF88C
:10945000101040F0BF8092F901300599DB0F43EA0C
:10946000410C0132ADF8AEC0ADF814C040230699EE
:1094700092F800E0490013EA0E0F18BF41F0010115
:109480005B08ADF8B010ADF8181040F0BF80079938
:109490004B0092F9011043EAD17CADF8B2C0ADF8AF
:1094A0001CC001324FF0400E137864001EEA030F17
:1094B00018BF44F001045FEA5E01ADF8B44040F02B
:1094C000BF80BDF8B61092F901C0490041EADC7EC8
:1094D000013240230999ADF8B6E0013911F0FF01DE
:1094E000099100F0BB8092F800C00A9913EA0C0FB2
:1094F0004FEA410118BF41F001015FEA530CADF89A
:109500009C10ADF828103FF441AF089992F800E0A4
:1095100049001CEA0E0F18BF41F001019B08ADF88D
:109520009E10ADF820107FF43DAF92F901107F003E
:1095300047EAD177ADF8A07001324FF0400E1378B2
:1095400076001EEA030F18BF46F001065FEA5E03CD
:10955000ADF8A2607FF43BAF02994B0092F9011085
:1095600043EAD17CADF8A4C0ADF808C00132402375
:10957000117840000B4218BF40F001005FEA530E23
:10958000ADF8A6007FF43DAF4FEA4A0192F901A081
:1095900041EADA7AADF8A8A001324023039992F8A3
:1095A00000E0490013EA0E0F18BF41F001015B080B
:1095B000ADF8AA10ADF80C107FF43DAF92F9011090
:1095C000CB0F049943EA410C0132ADF8ACC0ADF8C1
:1095D00010C04023059992F800C0490013EA0C0F0F
:1095E00018BF41F001015B08ADF8AE10ADF81410E2
:1095F0007FF43DAF92F90110CB0F069943EA410E7B
:109600000132ADF8B0E0ADF818E04023079992F8C8
:1096100000C0490013EA0C0F18BF41F001015FEAD6
:10962000530EADF8B210ADF81C107FF43DAF92F9B7
:109630000130640044EAD374ADF8B44001324021F3
:1096400013781942BDF8B6304FEA430E18BF4EF0FA
:10965000010E4B0804BF013280233BE7BDF89C009C
:10966000954C42462EA9F9F7FFF900283FF4B4AD16
:10967000B8F8002092B1914FB9F876073E6C96F891
:1096800088E050FA82FA9644A9F876A786F888E02E
:10969000636983F0400141F48002A261BDF89E003D
:1096A00042460DF1BA01F9F7DFF900283FF494AD15
:1096B000B8F8006028AF96B18048B9F876C7016C59
:1096C00091F888E05CFA86FAB644A9F876A781F8A2
:1096D00088E0636983F0400242F48006A6612FAE01
:1096E000388842463146F9F7BFF900283FF474AD97
:1096F000B8F80000023790B17049B9F876C70A6C23
:1097000092F888E05CFA80FA8644A9F876A782F895
:1097100088E0636983F0400040F48001A161023673
:10972000388842463146F9F79FF900283FF454AD96
:10973000B8F8002092B1614BB9F87617186C90F820
:1097400088A051FA82FC9244A9F876C780F888A0D4
:10975000626982F0400E4EF48003A361788842462D
:10976000B11CF9F781F900283FF436ADB8F80000D4
:1097700090B15249B9F876C70A6C92F888E05CFA61
:1097800080FA8644A9F876A782F888E0636983F0B6
:10979000400040F48001A161B8884246311DF9F7CC
:1097A00063F900283FF418ADB8F80020063792B1ED
:1097B000424BB9F87617186C90F888A051FA82FCE1
:1097C0009244A9F876C780F888A0626982F0400EBA
:1097D0004EF48003A3612EA8B84206F106067FF47A
:1097E0007FAF002025900DF1B606CDF89700024618
:1097F0000DF1940CB1787388C1F3C00747EA4000BB
:10980000C1F3800444EA4007C1F3400A50074AEA22
:10981000470E03F00101B0F1004F41EA4E0306F19B
:10982000020640D01C4696F802A07388CAF3C0070F
:1098300047EA4401CAF3800040EA410ECAF34004FB
:1098400044EA4E0A03F00103171D520743EA4A0196
:1098500006F102062BD008463A1D92B2382AC9D129
:10986000174C9DF894609DF89570A35D9DF8960047
:109870009DF897207B409DF89870E15C41409DF8F1
:109880009900665C56409DF89A20A35D7B40E15CA0
:109890004140665C5640A45DA4B1B9F874770137C5
:1098A000A9F87477A4E40CF8013B0024BBE70CF89A
:1098B000011B0020D0E700BF00080240000000208C
:1098C000D8070108C74B25991F6CC7483960BDF8F8
:1098D0009860BE804FF4001282617C79002C00F009
:1098E0007E810C2C8CBF022001200444E700BD4B7C
:1098F000186990F800C0417867447E1E96FBFCFE14
:1099000011FB0EF270321FFA82FABAF5096F3FF6B8
:109910006FAC019C94F8AC71BA440AF1FF3393FB2D
:10992000F7F0A0F11C018EB2002E41D0721E01246E
:1099300002F00707FBF7A2FCA64239D93BB21FB3DE
:10994000012B1BD0022B16D0032B11D0042B0CD0D3
:10995000052B07D0062B02D0FBF790FC0224FBF767
:109960008DFC0134FBF78AFC0134FBF787FC0134E2
:10997000FBF784FC0134FBF781FC01340134FBF775
:109980007DFCA0B2864213D90834FBF777FCFBF7C5
:1099900075FCFBF773FCFBF771FCFBF76FFCFBF747
:1099A0006DFCFBF76BFCFBF769FCA1B28E42EBD8B8
:1099B000FBF770FF00283FF41BAC019ED5F8D039AF
:1099C00096F8AC71D9F85825864CD21AD6E96901B7
:1099D0003B46F8F7E1FE246CB6F8B82284F886001E
:1099E0000023D6E9AC010292FDF7D0FC0029024623
:1099F0000B46C0F2FF80B0F1004F71F100014FF053
:109A000001060ADB900840EA837271009B10B2F1F4
:109A1000004FCEB273F10001F4DA980340EA924CA1
:109A20004FEA823E00234FF080419A0842EA817358
:109A30009E454FEAA1017CEB0102F6DB53EA0102ED
:109A400028D0CDE904741A4600231846B246D61829
:109A50004FEA9207039741EB0007B6457CEB0704FA
:109A600009DBBEEB060E6CEB070C941841EB01060C
:109A7000E31846EB0000039A42EA817289105F08FE
:109A800052EA010647EAC0734FEA6000DFD1DDE920
:109A90000474564686FB03AEA7FB0A2CC82007FBBE
:109AA0000EC1A2FB00236FF4FF7600FB0130B2422F
:109AB00070F1FF31C0F29C80002804DA40F2FF11FF
:109AC000521840F10000530A43EAC05A1AF50056F2
:109AD0004FEA602141F10002B00B40EA8243414E5F
:109AE000D5F8CC2996F83010019EC4F88C20FF2BB5
:109AF00001F10401A2EB412028BFFF2396F8991140
:109B000084F88730C4F89000D6F89C31029896F813
:109B1000A0E196F8A1C184F88AE007FB03F301FBFA
:109B200000F0B3FBF0F0637984F8890084F88BC00F
:109B30003BB10C2B8CBF4FF0020C4FF0010C634477
:109B4000DB00284E366930787678034403F1FF3E17
:109B50009EFBF0F306FB03F307F1FF3A7033D5F8F1
:109B6000B86101FB03A1B1FBF7F702EB4722C4F890
:109B7000942056B120461D4C636983F0080141F4DE
:109B80000027A761B047174A1064B9F8720799F81F
:109B90008847154E01304FF40023A9F872074FF49F
:109BA0008011B3614FF400174FF480024FF40000AE
:109BB0000223032CB161B761B261B061B3617FF47C
:109BC0001AAB99F88967002E7FF415ABD9F8644772
:109BD000C9F88C47012189F88917FFF70CBB274684
:109BE00085E600BF0000002000080240000002409F
:109BF000002374E74FF0FF3AD6464DE7D9F844000A
:109C0000046844F4807202602B463A464FF001101B
:109C1000F6F7C0FE00287EF4DAAF3946D9F8447072
:109C20005148A1233B612A46F6F74EFF18B1D9F8F7
:109C30008430FEF7CCBFD9F844602390706923903C
:109C4000B46923942846239BF6F7F8FF01460028C1
:109C500071D1D9F844201769536989F8687713F0EE
:109C6000040842D01469414889F869472B4601220B
:109C70003F4CF6F78FFEA8BBD9F84450296841F451
:109C800000702860D9F844301E6926701A69627025
:109C900099F8685700242027FF2D89F8817089F8EA
:109CA000804089F882407DF4C8AF324CB9F86967CA
:109CB00001212046F8F780FA86427DF4BFAFFDF718
:109CC000C9BFA078FBF7A2F999F81868092E3EF6EB
:109CD00047A909EB860E0136CEF8F04789F81868D7
:109CE000FEF73EB90134FDF7A9BF41461F48224C9B
:109CF0002B460122F6F74EFE014600BB2B46D9F853
:109D000044501A482E6826F480622A60D9F84470BC
:109D10003D6925700122F6F73DFE80B9D9F844105F
:109D2000086840F400730B60D9F8446032696270CF
:109D30003769A770ACE7D9F88430FDF77EBF0234ED
:109D4000FDF77CBFFBF762F9BEE70C4D08274FF427
:109D50000062402480214FF48056AF61AA61AC615B
:109D6000A961AE61FEE700BF02000100040001002E
:109D7000B2070120B3070120B10701200000024013
:109D80002DE9F04782B00646DDF828E00846B446E3
:109D90000D46002B4ED18A4214466DD9B2FA82F29A
:109DA00042B1C2F12003954026FA03F394401D43CB
:109DB00006FA02FC260CA7B2B5FBF6F14FEA1C43EB
:109DC00006FB115543EA054301FB07F0984209D908
:109DD000E31801F1FF3580F00381984240F20081E1
:109DE000023923441B1A1FFA8CFCB3FBF6F006FB66
:109DF00010334CEA034C00FB07F363450AD914EB1C
:109E00000C0C00F1FF3580F0ED80634540F2EA80F4
:109E1000A444023840EA0140ACEB030C0021BEF13F
:109E2000000F04D02CFA02F30022CEE9003202B077
:109E3000BDE8F0878B4209D9BEF1000F01D0CEE911
:109E400000610021084602B0BDE8F087B3FA83F153
:109E5000174600294DD1834202D3B24200F20F814E
:109E6000B6EB070C60EB030301201D46BEF1000FAB
:109E7000DDD0CEE900C5DAE7002A00F098801A4666
:109E8000B4FA84F3002B40F0AF800B1B270CA6B272
:109E90000121B3FBF7F54FEA1C4007FB153340EAFD
:109EA000034306FB05F8984507D9E31805F1FF3091
:109EB00002D2984500F2E8800546A3EB08031FFA9A
:109EC0008CFCB3FBF7F007FB10334CEA034C06FBAA
:109ED00000F3634508D914EB0C0C00F1FF3602D2F5
:109EE000634500F2CE803046ACEB030C40EA0540FF
:109EF00095E7C1F120058B4022FA05FC4CEA030CE2
:109F000000FA01F426FA05F3E84002FA01F943EAFF
:109F100004084FEA1C4206FA01FAB0FBF2F71FFAF6
:109F20008CF602FB17004FEA184444EA004407FB92
:109F300006F0A0420AD91CEB040407F1FF3380F0BD
:109F40009C80A04240F29980023F6444241A1FFA88
:109F500088F3B4FBF2F002FB104443EA044300FB35
:109F600006F69E4209D91CEB030300F1FF3480F092
:109F700082809E427FD90238634440EA0740A0FBBA
:109F800009749B1BA3423E46A04664D361D0BEF138
:109F9000000F0AD0BAEB060263EB080303FA05F5DB
:109FA000CA401543CB40CEE9005300213FE7730878
:109FB00043EAC1734A08190C41EA02414FEAC67CE0
:109FC0009BB2B2FBF4F02646A04627461F2243EA86
:109FD0000143B1FBF4F1A3EB080341EA004158E768
:109FE0002946FFE6284615E71A46C3F120019C40A2
:109FF00026FA01F320FA01F190400343270C06FAF8
:10A0000002FCB1FBF7F0A6B207FB1015190C41EAF0
:10A01000054100FB06F58D423BD9611801D28D4206
:10A0200020D8491B0138B1FBF7F5019505FB06F86F
:10A03000019D9BB207FB151143EA0143434526D21C
:10A04000E31805F1FF31C6D24345C4D2A91E23440B
:10A05000C1E7BA459BD2B7EB090664EB0C040138A3
:10A06000A04694E7651B29440238B1FBF7F501953A
:10A0700005FB06F8DCE720467FE71F4666E7084653
:10A08000F4E6A44402382FE7023D234415E7019982
:10A09000A1E7491BB1FBF7F5019505FB06F8C7E7FA
:10A0A00030B584078646034606D0A2B303F8011BE9
:10A0B000980702F1FF32F8D1032A26D95FFA81FC12
:10A0C0000CEB0C2C0F2A0CEB0C402AD922F00F0CB5
:10A0D0009C44C3E90000C3E9020010336345F8D192
:10A0E00012F00C0F02F00F0417D04FEA940C0CF191
:10A0F000FF351A4603EB8C0C42F8040B6245FBD18A
:10A10000043304F0030203EB850322B11A4403F87D
:10A11000011B9A42FBD1704630BD2246002AF5D180
:10A12000F9E71446E1E700BF10B50446084383078A
:10A1300001D1032A19D8A44601F1FF3E07E01EF819
:10A14000011F03F8011B501E31B19C4602466346B5
:10A15000002AF4D1204610BD94440028FAD003F818
:10A16000011B6345FBD1204610BD0B46A446186871
:10A170001946A0F1013323EA000313F0803F01F1F7
:10A180000403D9D1043A032A4CF8040BEFD819463A
:04A19000D2E700BF53
:10A1940008B5F6F733F800BF024A136801331360B9
:10A1A400704700BF4800012080B5704B704A84B0EE
:10A1B4001968914200AF0AD16E4D6F4E1D6086F34F
:10A1C4000888A3F5303CDCF80440A047FEE76B4860
:10A1D4006B4ED0F8884044F47005C0F8885032685B
:10A1E400684C002342F001013160B360356825F00A
:10A1F400847828F48032326074603168624C21F4CF
:10A2040080224FF000653260F36085608460D0F88E
:10A2140088605E4B46F47001C0F888105C48984230
:10A2240008D25B485B495C1E221A22F00302043206
:10A23400FDF714F9584D594EAE4208D25748691EDD
:10A244000B1A23F0030204320021FFF727FF544DB9
:10A254004A4E2A6842F400712960286840F48063F9
:10A264002B602A6842F480712960F5684FF6FF0478
:10A2740025404C4C45EA0400F060F6F767FB404E7D
:10A28400494B0021F960326C42F080553564346CDE
:10A2940004F08050F860FA68B9601A68434942F4DF
:10A2A40040451D601B6803F44040B8600124BB684E
:10A2B400CC64B26802F00C01042927D0B56805F01B
:10A2C4000C03082B1FD02E4CA06800F00C020C2AA3
:10A2D40000F01D822A4A364801259570046803E07F
:10A2E4000668311B64296CD813689E03F8D5244A88
:10A2F400936803F00C04082C63D02C4E2C490020E6
:10A3040030660E6809E076687202DCD51C4D2B6855
:10A31400EDE70C68A51B022D53D81568AD01F8D4E0
:10A3240047F6C07393FAA3FC4FF44036BCFA8CF49E
:10A3340096FAA6F34FF0706E9EFAAEF84FF0E04531
:10A34400B8FA88F095FAA5F307264FF4D873A3401A
:10A3540006FA00F42343154D43F4800040F014033F
:10A36400012653602E660D68054A27E000C00120CF
:10A37400AD700DB0EFBEADDEF82A002000ED00E0B8
:10A38400003802401030002400000008440001207E
:10A39400000000208C0203083C6D012048000120CD
:10A3A400003C02400003FA050070004000004742F0
:10A3B400480001200868431B022B02D81468A4013A
:10A3C400F8D5A149086800F00F03042B00F2D280ED
:10A3D40005260E700A6802F00F04052C00F0CA80EE
:10A3E4009A4D9B4A916801F00C03082B00F01781E9
:10A3F400984E9749984B8C689848C4F30318434483
:10A40400974C93F8002CD6402E60051B002D52DD8E
:10A41400AE10711E54F8043B012501F0070898475B
:10A42400AE4248DDB8F1000F2CD0B8F1010F23D0B3
:10A43400B8F1020F1CD0B8F1030F15D0B8F1040F16
:10A444000ED0B8F1050F07D0B8F1060F40F05A81CD
:10A4540054F8042B9047013554F8041B8847013500
:10A4640054F8043B9847013554F8040B80470135F0
:10A4740054F8042B9047013554F8041B01358847E0
:10A48400AE4218DD2346083553F8040B7B60804741
:10A494006268904779684B689847E068804722690A
:10A4A400904761698847A3699847E0698047AE424D
:10A4B40004F12004E6DC6B4C6B4D661B002E57DD6B
:10A4C400B610721E55F8041B02F007048847012ECB
:10A4D4004FF001084CDD6CB3012C23D0022C1CD0AE
:10A4E400032C15D0042C0ED0052C07D0062C40F0DC
:10A4F400038155F8040B804708F1010855F8042B33
:10A50400904708F1010855F8041B884708F1010831
:10A5140055F8044BA04708F1010855F8043B984747
:10A5240008F1010855F8040B804708F1010296422E
:10A5340090461DDD2C46203554F8041B884755F8F9
:10A544001C3C98476068804755F8142C904755F890
:10A55400104CA04755F80C1C884755F8083C984700
:10A5640055F8040C804708F1080296429046E1DC55
:10A57400FDF790F8364B9D6825F0F0019960186856
:10A5840082017FF52DAF9E68384926F0030C4CF00C
:10A5940002029A600C6841F2883C04E00E68301BA9
:10A5A40060453FF61DAF9D6805F00C06082EF5D1F9
:10A5B400254C236803F00F01052907D905202070D5
:10A5C400226802F00F05052D7FF40AAF204EB4680F
:10A5D40024F4E05E4EF4A053B360B16821F460400B
:10A5E40040F40042B260B56805F00C04082C61D058
:10A5F4000C2C3FD0174C164DF020AA6890FAA0F608
:10A604001B4B124DB6FA86F102F0F000C840184414
:10A6140090F86824D4402C60F6F798F9E1E6506885
:10A624000B4E546852680B4804F03F0E7468B0FB3C
:10A63400FEF1C4F30140C2F38813013003FB01F1BE
:10A644004200B1FBF2F6D4E6003C024000000020D8
:10A65400003802400024F400F40C01088C020308C2
:10A664008C0203088C0203088C02030848000120B2
:10A6740024A70008756870682748766805F03F02CB
:10A6840047F6C073B0FBF2F493FAA3F8234DB8FA7B
:10A6940088F11E40CE406A6806FB04F44FF0E040A7
:10A6A40090FAA0F6B6FA86F302F0E041D940B4FB82
:10A6B400F1F4A0E77168184B7068766801F03F0008
:10A6C40047F6C072B3FBF0F592FAA2F4134BB4FA56
:10A6D40084F11640CE4006FB05F54FF440305E6829
:10A6E40090FAA0F2B2FA82F406F44031E14001316A
:10A6F4004B00B5FBF3F47EE755F8043B98474FF065
:10A704000208F6E654F8040B80470225A0E66168C7
:10A714004B027FF5DFADF9E50024F4000038024078
:10A724000006101600061016008000000408000041
:10A7340005290008692A00080B100000D92900081F
:10A74400592B00080000ADBAF7CF5A754325EE9F88
:10A75400B4EA1950864A2BF07185DC3FC56F68D581
:10A7640032A09F1A0C95A12FFB5A56E04FB0E20A73
:10A77400B87F15C58ADF27657D10D0AAC9FA644061
:10A784003E35938FB590182A425FEFE5F6B55B0F1F
:10A79400017AACC033DA9E60C41569AF70FFDD4541
:10A7A40087302A8AB90514BF4ECAE370FA20579A33
:10A7B4000DEFA0553F4F92F5C880653A7C6AD1D021
:10A7C4008BA5261FC79B6A2130549DEE84BE2904A5
:10A7D4007371DECB41D1EC6BB61E1BA402F4AF4EF9
:10A7E400F53B5881CB0E66B43CC1917B882B2591F7
:10A7F4007FE4D25E4D44E0FEBA8B17310E61A3DBD9
:10A80400F9AE5414720BDFB185C4287E312E9C94AA
:10A81400C6E16B5BF44159FB038EAE34B7641ADEB8
:10A8240040ABED117E9ED324895124EB3DBB9001B6
:10A83400CA7467CEF8D4556E0F1BA2A1BBF1164B98
:10A844004C3EE184238D8E37D44279F860A8CD1232
:10A8540097673ADDA5C7087D5208FFB2E6E24B5878
:10A86400112DBC972F1882A2D8D7756D6C3DC18766
:10A874009BF23648A95204E85E9DF327EA7747CD58
:10A884001DB8B002961D3BA761D2CC68D53878823A
:10A8940022F78F4D1057BDEDE7984A225372FEC838
:10A8A400A4BD09079A8837326D47C0FDD9AD741726
:10A8B4002E6283D81CC2B178EB0D46B75FE7F25D18
:10A8C400A8280592E41649AC13D9BE63A7330A89B4
:10A8D40050FCFD46625CCFE69593382921798CC300
:10A8E400D6B67B0CE88345391F4CB2F6ABA6061CE2
:10A8F4005C69F1D36EC9C373990634BC2DEC8056E0
:10A90400DA2377995186FC3CA6490BF312A3BF19AD
:10A91400E56C48D6D7CC7A7620038DB994E93953BF
:10A924006326CE9C5D13F0A9AADC07661E36B38CA1
:10A93400E9F94443DB5976E32C96812C987C35C69F
:10A944006FB3C2090D000B000800070004000200E9
:10A9540001000E00D506B30500048F0300020001B8
:10A9640080007F0040002000100008000400020066
:10A9740001006907AA0066001E00FF00AAAA666615
:10A984001E1EFE01FFFF0000000075D19F73EAA2A6
:10A994003EE74B36A194D445091F7CCE966CE3BDAB
:10A9A40037F84229A88BDD5A123E67EF8D4DF89C8B
:10A9B4002CD95908B3AAC67B1B216EF08452F183AB
:10A9C40025C65017BAB5CF64247C51ADBB0FCEDE7B
:10A9D4001A9B6F4A85E8F0392D6358B2B210C7C18B
:10A9E400138466558CF7F92636424393A931DCE08B
:10A9F40008A57D7497D6E2073F5D4A8CA02ED5FF4B
:10AA040001BA746B9EC9EB1848F83D29D78BA25A3A
:10AA1400761F03CEE96C9CBD41E73436DE94AB452A
:10AA24007F000AD1E07395A25AC62F17C5B5B0644A
:10AA3400642111F0FB528E8353D92608CCAAB97B2A
:10AA44006D3E18EFF24D879C6C841955F3F78626FA
:10AA5400526327B2CD10B8C1659B104AFAE88F390A
:10AA64005B7C2EADC40FB1DE7EBA0B6BE1C99418CA
:10AA7400405D358CDF2EAAFF77A50274E8D69D07CA
:10AA840049423C93D631A3E0E52190F07A520F83FA
:10AA9400DBC6AE1744B53164EC3E99EF734D069CAA
:10AAA400D2D9A7084DAA387BF71F82CE686C1DBD8A
:10AAB400C9F8BC29568B235AFE008BD1617314A2AA
:10AAC400C0E7B5365F942A45C15DB48C5E2E2BFF7A
:10AAD400FFBA8A6B60C91518C842BD93573122E08A
:10AAE400F6A5837469D61C07D363A6B24C1039C18A
:10AAF400ED84985572F70726DA7CAFAD450F30DE4A
:10AB0400E49B914A7BE80E39ADD9D80832AA477B39
:10AB1400933EE6EF0C4D799CA4C6D1173BB54E6429
:10AB24009A21EFF005527083BFE7CA362094554549
:10AB34008100F4D11E736BA2B6F8C329298B5C5A29
:10AB4400881FFDCE176C62BD89A5FC7416D66307F9
:10AB5400B742C29328315DE080BAF56B1FC96A1809
:10AB6400BE5DCB8C212E54FF9B9BEE4A04E87139C9
:10AB7400A57CD0AD3A0F4FDE9284E7550DF77826C9
:10AB8400AC63D9B2331046C10000000001020304D3
:10AB94000102030406070809055085ABC5D8E5EE94
:10ABA400F5FAFD00010001010102010301040105A0
:10ABB4000106010701080109010A010B010C010D3D
:10ABC400010E010F01100111011200000040853631
:10ABD400B02D0826C91F651A601675133E11A00F03
:10ABE4003E0EF70C2A0C9D0B440B0F0BCC0AAE0A3D
:10ABF4006C0A3A0A200A1F0A1F0A240A300A190A90
:10AC0400050AD2099C096C093309E7089B0847081F
:10AC1400DF077A071307C0068F067A0688069D06A3
:10AC2400CC06ED06200741074D076A07E5073537CF
:10AC34004C3327309B2D862BD02967283C2745266B
:10AC44007925D1244A24DD238A234C2322230B2370
:10AC540004230C2324234A237D23BD230A246424B0
:10AC6400CA243C25BC254826E02687273B28FD2806
:10AC7400CE29AF2AA12BA42CB92DE22E2030743179
:10AC8400DF3264340536C2379E399A3BBA3D004000
:10AC940000400040004000400040004000400040B0
:10ACA40000400040004000400040004000400040A0
:10ACB4000040004000400040004000400040004090
:10ACC4000040004000400040004000400040004080
:10ACD4000040004000400040004000400040004070
:10ACE4000040004000400040004000400040004060
:10ACF40000400040AD388732892D9A296426A42368
:10AD04003A211E1F451DA11B291AD4189B1783160F
:10AD14008D15AB14D8130F134E129711E81045106C
:10AD2400AD0F1E0F990E200EAE0D430DDF0C830CDC
:10AD3400360CF50BC50B930BFD0ABB0A8F0A660A8A
:10AD44002B0AF009B4097E094E0926090209E30811
:10AD5400C708AD08004000400040004000400040EB
:10AD640000400040004000400040004000400040DF
:10AD740000400040004000400040004000400040CF
:10AD840000400040004000400040004000400040BF
:10AD940000400040004000400040004000400040AF
:10ADA400004000400040004000400040004000409F
:10ADB400004000400040E90C9C0BE60A3C0A910963
:10ADC400BC08FB0744079606E4054705C304520480
:10ADD400F703A603640333030D03EA02CD02B402AE
:10ADE400A00294028F029602A802C702F0022E0368
:10ADF4007503CE033704B1044005EE05C806CE073B
:10AE04000209510ADF0BB30DFC0F10133017851C18
:10AE14003B23B42B17350040E0B20008D80C0108DE
:10AE24001CC501081CC101081CBD01081CB901088E
:10AE34001CB501081CB101081CAD01081CA90108BE
:10AE44001CA501081CA101081C9D01081C990108EE
:10AE5400D81001081C9501081C9101081C8D0108DB
:10AE64001C890108D81401081C8501081C810108EB
:10AE74001C7D01081C7901081C7501081C7101085E
:10AE84001C6D01081C6901081C6501081C6101088E
:10AE94001C5D01081C590108D80801081C5501084B
:10AEA4001C5101081C4D01081C4901081C450108DE
:10AEB4001C4101081C3D01081C3901081C3501080E
:10AEC4001C3101081C2D01081C2901081C2501083E
:10AED4001C2101081C1D01081C190108000064093B
:10AEE40094125D1B8E23FA2A7931E536203B143EF9
:10AEF400B13FEC3FC53E423C71386733412D1F26BC
:10AF04002B1E8F157C0C2303BBF974F083E719DF28
:10AF140067D795D0CACA26C6C2C2B2C000C0B2C0E2
:10AF2400C2C226C6CACA95D067D719DF83E774F0B0
:10AF3400BBF923037C0C8F152B1E1F26412D673371
:10AF44007138423CC53EEC3FB13F143E203BE536F0
:10AF54007931FA2A8E235D1B9412640900009CF651
:10AF64006CEDA3E472DC06D587CE1BC9E0C4ECC14A
:10AF74004FC014C03BC1BEC38FC799CCBFD2E1D967
:10AF8400D5E171EA84F3DDFC45068C0F7D18E720DA
:10AF940099286B2F3635DA393E3D4E3F00404E3FFF
:10AFA4003E3DDA3936356B2F9928E7207D188C0F12
:10AFB4004506DDFC84F371EAD5E1E1D9BFD299CC31
:10AFC4008FC7BEC33BC114C04FC0ECC1E0C41BC992
:10AFD40087CE06D572DCA3E46CED9CF60000640910
:10AFE40094125D1B8E23FA2A7931E536203B143EF8
:10AFF400B13FEC3FC53E423C71386733412D1F26BB
:10B004002B1E8F157C0C2303BBF974F083E719DF27
:10B0140067D795D0CACA26C6C2C2B2C000C0B2C0E1
:10B02400C2C226C6CACA95D067D719DF83E774F0AF
:10B03400BBF923037C0C8F152B1E1F26412D673370
:10B044007138423CC53EEC3FB13F143E203BE536EF
:10B054007931FA2A8E235D1B9412640900009CF650
:10B064006CEDA3E472DC06D587CE1BC9E0C4ECC149
:10B074004FC014C03BC1BEC38FC799CCBFD2E1D966
:10B08400D5E171EA84F3DDFC45068C0F7D18E720D9
:10B0940099286B2F3635DA393E3D4E3F00404E3FFE
:10B0A4003E3DDA3936356B2F9928E7207D188C0F11
:10B0B4004506DDFC84F371EAD5E1E1D9BFD299CC30
:10B0C4008FC7BEC33BC114C04FC0ECC1E0C41BC991
:10B0D40087CE06D572DCA3E46CED9CF6000064090F
:10B0E40094125D1B8E23FA2A7931E536203B143EF7
:10B0F400B13FEC3FC53E423C71386733412D1F26BA
:10B104002B1E8F157C0C2303BBF974F083E719DF26
:10B1140067D795D0CACA26C6C2C2B2C000C0B2C0E0
:10B12400C2C226C6CACA95D067D719DF83E774F0AE
:10B13400BBF923037C0C8F152B1E1F26412D67336F
:10B144007138423CC53EEC3FB13F143E203BE536EE
:10B154007931FA2A8E235D1B9412640900009CF64F
:10B164006CEDA3E472DC06D587CE1BC9E0C4ECC148
:10B174004FC014C03BC1BEC38FC799CCBFD2E1D965
:10B18400D5E171EA84F3DDFC45068C0F7D18E720D8
:10B1940099286B2F3635DA393E3D4E3F00404E3FFD
:10B1A4003E3DDA3936356B2F9928E7207D188C0F10
:10B1B4004506DDFC84F371EAD5E1E1D9BFD299CC2F
:10B1C4008FC7BEC33BC114C04FC0ECC1E0C41BC990
:10B1D40087CE06D572DCA3E46CED9CF6000064090E
:10B1E40094125D1B8E23FA2A7931E536203B143EF6
:10B1F400B13FEC3FC53E423C71386733412D1F26B9
:10B204002B1E8F157C0C2303BBF974F083E719DF25
:10B2140067D795D0CACA26C6C2C2B2C000C0B2C0DF
:10B22400C2C226C6CACA95D067D719DF83E774F0AD
:10B23400BBF923037C0C8F152B1E1F26412D67336E
:10B244007138423CC53EEC3FB13F143E203BE536ED
:10B254007931FA2A8E235D1B9412640900009CF64E
:10B264006CEDA3E472DC06D587CE1BC9E0C4ECC147
:10B274004FC014C03BC1BEC38FC799CCBFD2E1D964
:10B28400D5E171EA84F3DDFC45068C0F7D18E720D7
:10B2940099286B2F3635DA393E3D4E3F00404E3FFC
:10B2A4003E3DDA3936356B2F9928E7207D188C0F0F
:10B2B4004506DDFC84F371EAD5E1E1D9BFD299CC2E
:10B2C4008FC7BEC33BC114C04FC0ECC1E0C41BC98F
:10B2D40087CE06D572DCA3E46CED9CF60000412D0C
:10B2E4000040412D0000BFD200C0BFD20000412D5C
:10B2F4000040412D0000BFD200C0BFD20000412D4C
:10B304000040412D0000BFD200C0BFD20000412D3B
:10B314000040412D0000BFD200C0BFD20000412D2B
:10B324000040412D0000BFD200C0BFD20000412D1B
:10B334000040412D0000BFD200C0BFD20000412D0B
:10B344000040412D0000BFD200C0BFD20000412DFB
:10B354000040412D0000BFD200C0BFD20000412DEB
:10B364000040412D0000BFD200C0BFD20000412DDB
:10B374000040412D0000BFD200C0BFD20000412DCB
:10B384000040412D0000BFD200C0BFD20000412DBB
:10B394000040412D0000BFD200C0BFD20000412DAB
:10B3A4000040412D0000BFD200C0BFD20000412D9B
:10B3B4000040412D0000BFD200C0BFD20000412D8B
:10B3C4000040412D0000BFD200C0BFD20000412D7B
:10B3D4000040412D0000BFD200C0BFD20000412D6B
:10B3E4000040412D0000BFD200C0BFD20000412D5B
:10B3F4000040412D0000BFD200C0BFD20000412D4B
:10B404000040412D0000BFD200C0BFD20000412D3A
:10B414000040412D0000BFD200C0BFD20000412D2A
:10B424000040412D0000BFD200C0BFD20000412D1A
:10B434000040412D0000BFD200C0BFD20000412D0A
:10B444000040412D0000BFD200C0BFD20000412DFA
:10B454000040412D0000BFD200C0BFD20000412DEA
:10B464000040412D0000BFD200C0BFD20000412DDA
:10B474000040412D0000BFD200C0BFD20000412DCA
:10B484000040412D0000BFD200C0BFD20000412DBA
:10B494000040412D0000BFD200C0BFD20000412DAA
:10B4A4000040412D0000BFD200C0BFD20000412D9A
:10B4B4000040412D0000BFD200C0BFD20000412D8A
:10B4C4000040412D0000BFD200C0BFD20000412D7A
:10B4D4000040412D0000BFD200C0BFD20000412D6A
:10B4E4000040412D0000BFD200C0BFD20000412D5A
:10B4F4000040412D0000BFD200C0BFD20000412D4A
:10B504000040412D0000BFD200C0BFD20000412D39
:10B514000040412D0000BFD200C0BFD20000412D29
:10B524000040412D0000BFD200C0BFD20000412D19
:10B534000040412D0000BFD200C0BFD20000412D09
:10B544000040412D0000BFD200C0BFD20000412DF9
:10B554000040412D0000BFD200C0BFD20000412DE9
:10B564000040412D0000BFD200C0BFD20000412DD9
:10B574000040412D0000BFD200C0BFD20000412DC9
:10B584000040412D0000BFD200C0BFD20000412DB9
:10B594000040412D0000BFD200C0BFD20000412DA9
:10B5A4000040412D0000BFD200C0BFD20000412D99
:10B5B4000040412D0000BFD200C0BFD20000412D89
:10B5C4000040412D0000BFD200C0BFD20000412D79
:10B5D4000040412D0000BFD200C0BFD20000412D69
:10B5E4000040412D0000BFD200C0BFD20000412D59
:10B5F4000040412D0000BFD200C0BFD20000412D49
:10B604000040412D0000BFD200C0BFD20000412D38
:10B614000040412D0000BFD200C0BFD20000412D28
:10B624000040412D0000BFD200C0BFD20000412D18
:10B634000040412D0000BFD200C0BFD20000412D08
:10B644000040412D0000BFD200C0BFD20000412DF8
:10B654000040412D0000BFD200C0BFD20000412DE8
:10B664000040412D0000BFD200C0BFD20000412DD8
:10B674000040412D0000BFD200C0BFD20000412DC8
:10B684000040412D0000BFD200C0BFD20000412DB8
:10B694000040412D0000BFD200C0BFD20000412DA8
:10B6A4000040412D0000BFD200C0BFD20000412D98
:10B6B4000040412D0000BFD200C0BFD20000412D88
:10B6C4000040412D0000BFD200C0BFD20000412D78
:10B6D4000040412D0000BFD200C0BFD20001AAAA81
:10B6E400000000405A2E212CEC3FDDFCCD298ACFEE
:10B6F400BBF94FC08CCDA1D8B2C0640926DB53344A
:10B704007C0CC53E12363D22143E74F08B1F51C88A
:10B714006CEDC2C2D6C63AE3BEC38F1511E6823AB7
:10B724007D18203BB63B0817DA39A3E413143BC356
:10B73400D5E18FC752C2EFEE1BC9E720FBF1713E82
:10B744008E2336350E3FF10A6733E1D9D5077CC025
:10B7540067D787CE2DC04BFB95D0FA2A6EFEFB3FF0
:10B76400412D412DFB3F6EFEFA2A95D04BFB2DC097
:10B7740087CE67D77CC0D507E1D96733F10A0E3F7E
:10B7840036358E23713EFBF1E7201BC9EFEE52C222
:10B794008FC7D5E13BC31314A3E4DA390817B63BCA
:10B7A400203B7D18823A11E68F15BEC33AE3D6C614
:10B7B400C2C26CED51C88B1F74F0143E3D22123688
:10B7C400C53E7C0C533426DB6409B2C0A1D88CCDB1
:10B7D4004FC0BBF98ACFCD29DDFCEC3F212C5A2E7A
:10B7E40000400000212CA6D1DDFC14C08ACF33D642
:10B7F4004FC04506A1D8743264094E3F5334DA244D
:10B80400C53E84F33D22EEC974F0ECC151C875E025
:10B81400C2C294123AE32A398F15423C823AEF1994
:10B82400203B83E708174AC4A3E426C63BC3EDEBD9
:10B834008FC72B1EEFEEAE3DE720E536713E050EB9
:10B84400363572DCF10AF2C0E1D999CC7CC02BF810
:10B8540087CE99284BFBD33FFA2A6B2FFB3F9201EB
:10B86400412DBFD26EFE05C095D006D52DC0B504BE
:10B8740067D77931D507843F67331F260E3F0FF50D
:10B884008E23CACAFBF18FC11BC919DF52C2111121
:10B89400D5E171381314C53CDA395D1BB63BF8E8C1
:10B8A4007D18E0C411E67EC5BEC371EAD6C6C61CC7
:10B8B4006CED3E3D8B1FAF37143E8C0F1236C3DD4B
:10B8C4007C0C3BC126DBADCBB2C09CF68CCD5F2794
:10B8D400BBF9B13FCD297630EC3F23035A2EDFD399
:10B8E400000000C0A6D1DFD314C0230333D67630C2
:10B8F4004506B13F74325F274E3F9CF6DA24ADCB48
:10B9040084F33BC1EEC9C3DDECC18C0F75E0AF37E6
:10B9140094123E3D2A39C61C423C71EAEF197EC599
:10B9240083E7E0C44AC4F8E826C65D1BEDEBC53CDA
:10B934002B1E7138AE3D1111E53619DF050E8FC18E
:10B9440072DCCACAF2C00FF599CC1F262BF8843FCB
:10B9540099287931D33FB5046B2F06D5920105C0E0
:10B96400BFD2BFD205C0920106D56B2FB504D33F19
:10B9740079319928843F2BF81F2699CC0FF5F2C012
:10B98400CACA72DC8FC1050E19DFE5361111AE3D4E
:10B9940071382B1EC53CEDEB5D1B26C6F8E84AC486
:10B9A400E0C483E77EC5EF1971EA423CC61C2A391C
:10B9B4003E3D9412AF3775E08C0FECC1C3DDEEC988
:10B9C4003BC184F3ADCBDA249CF64E3F5F2774323F
:10B9D400B13F4506763033D6230314C0DFD3A6D156
:10B9E40000C00000DFD35A2E2303EC3F7630CD296C
:10B9F400B13FBBF95F278CCD9CF6B2C0ADCB26DB43
:10BA04003BC17C0CC3DD12368C0F143EAF378B1F49
:10BA14003E3D6CEDC61CD6C671EABEC37EC511E6BA
:10BA2400E0C47D18F8E8B63B5D1BDA39C53C131455
:10BA34007138D5E1111152C219DF1BC98FC1FBF155
:10BA4400CACA8E230FF50E3F1F266733843FD507DE
:10BA5400793167D7B5042DC006D595D005C06EFEE3
:10BA6400BFD2412D9201FB3F6B2FFA2AD33F4BFBF0
:10BA7400992887CE2BF87CC099CCE1D9F2C0F10A81
:10BA840072DC3635050E713EE536E720AE3DEFEE4D
:10BA94002B1E8FC7EDEB3BC326C6A3E44AC408178D
:10BAA40083E7203BEF19823A423C8F152A393AE367
:10BAB4009412C2C275E051C8ECC174F0EEC93D22C3
:10BAC40084F3C53EDA2453344E3F64097432A1D85A
:10BAD40045064FC033D68ACF14C0DDFCA6D1212C35
:10BAE400000000405A2E212CEC3FDDFCCD298ACFEA
:10BAF400BBF94FC08CCDA1D8B2C0640926DB533446
:10BB04007C0CC53E12363D22143E74F08B1F51C886
:10BB14006CEDC2C2D6C63AE3BEC38F1511E6823AB3
:10BB24007D18203BB63B0817DA39A3E413143BC352
:10BB3400D5E18FC752C2EFEE1BC9E720FBF1713E7E
:10BB44008E2336350E3FF10A6733E1D9D5077CC021
:10BB540067D787CE2DC04BFB95D0FA2A6EFEFB3FEC
:10BB6400412D412DFB3F6EFEFA2A95D04BFB2DC093
:10BB740087CE67D77CC0D507E1D96733F10A0E3F7A
:10BB840036358E23713EFBF1E7201BC9EFEE52C21E
:10BB94008FC7D5E13BC31314A3E4DA390817B63BC6
:10BBA400203B7D18823A11E68F15BEC33AE3D6C610
:10BBB400C2C26CED51C88B1F74F0143E3D22123684
:10BBC400C53E7C0C533426DB6409B2C0A1D88CCDAD
:10BBD4004FC0BBF98ACFCD29DDFCEC3F212C5A2E76
:10BBE40000400000212CA6D1DDFC14C08ACF33D63E
:10BBF4004FC04506A1D8743264094E3F5334DA2449
:10BC0400C53E84F33D22EEC974F0ECC151C875E021
:10BC1400C2C294123AE32A398F15423C823AEF1990
:10BC2400203B83E708174AC4A3E426C63BC3EDEBD5
:10BC34008FC72B1EEFEEAE3DE720E536713E050EB5
:10BC4400363572DCF10AF2C0E1D999CC7CC02BF80C
:10BC540087CE99284BFBD33FFA2A6B2FFB3F9201E7
:10BC6400412DBFD26EFE05C095D006D52DC0B504BA
:10BC740067D77931D507843F67331F260E3F0FF509
:10BC84008E23CACAFBF18FC11BC919DF52C211111D
:10BC9400D5E171381314C53CDA395D1BB63BF8E8BD
:10BCA4007D18E0C411E67EC5BEC371EAD6C6C61CC3
:10BCB4006CED3E3D8B1FAF37143E8C0F1236C3DD47
:10BCC4007C0C3BC126DBADCBB2C09CF68CCD5F2790
:10BCD400BBF9B13FCD297630EC3F23035A2EDFD395
:10BCE400000000C0A6D1DFD314C0230333D67630BE
:10BCF4004506B13F74325F274E3F9CF6DA24ADCB44
:10BD040084F33BC1EEC9C3DDECC18C0F75E0AF37E2
:10BD140094123E3D2A39C61C423C71EAEF197EC595
:10BD240083E7E0C44AC4F8E826C65D1BEDEBC53CD6
:10BD34002B1E7138AE3D1111E53619DF050E8FC18A
:10BD440072DCCACAF2C00FF599CC1F262BF8843FC7
:10BD540099287931D33FB5046B2F06D5920105C0DC
:10BD6400BFD2BFD205C0920106D56B2FB504D33F15
:10BD740079319928843F2BF81F2699CC0FF5F2C00E
:10BD8400CACA72DC8FC1050E19DFE5361111AE3D4A
:10BD940071382B1EC53CEDEB5D1B26C6F8E84AC482
:10BDA400E0C483E77EC5EF1971EA423CC61C2A3918
:10BDB4003E3D9412AF3775E08C0FECC1C3DDEEC984
:10BDC4003BC184F3ADCBDA249CF64E3F5F2774323B
:10BDD400B13F4506763033D6230314C0DFD3A6D152
:10BDE40000C00000DFD35A2E2303EC3F7630CD2968
:10BDF400B13FBBF95F278CCD9CF6B2C0ADCB26DB3F
:10BE04003BC17C0CC3DD12368C0F143EAF378B1F45
:10BE14003E3D6CEDC61CD6C671EABEC37EC511E6B6
:10BE2400E0C47D18F8E8B63B5D1BDA39C53C131451
:10BE34007138D5E1111152C219DF1BC98FC1FBF151
:10BE4400CACA8E230FF50E3F1F266733843FD507DA
:10BE5400793167D7B5042DC006D595D005C06EFEDF
:10BE6400BFD2412D9201FB3F6B2FFA2AD33F4BFBEC
:10BE7400992887CE2BF87CC099CCE1D9F2C0F10A7D
:10BE840072DC3635050E713EE536E720AE3DEFEE49
:10BE94002B1E8FC7EDEB3BC326C6A3E44AC4081789
:10BEA40083E7203BEF19823A423C8F152A393AE363
:10BEB4009412C2C275E051C8ECC174F0EEC93D22BF
:10BEC40084F3C53EDA2453344E3F64097432A1D856
:10BED40045064FC033D68ACF14C0DDFCA6D1212C31
:10BEE40000000040DA395D1B793167D774F0ECC18A
:10BEF4003BC184F3E1D967332B1E7138EC3FDDFC81
:10BF04007D18E0C406D595D0C2C294129CF64E3F6B
:10BF140036358E23E53619DFBBF94FC0BEC371EA4F
:10BF2400BFD2412D8F15423CB13F4506E7201BC9C6
:10BF340072DCCACAB2C064096CED3E3D6B2FFA2AAA
:10BF4400203B83E7230314C08FC7D5E199CC1F2678
:10BF54007C0CC53E143E8C0F992887CEA3E426C6DC
:10BF640000C00000A3E4DA3999287931143E74F052
:10BF74007C0C3BC199CCE1D98FC72B1E2303EC3F2A
:10BF8400203B7D186B2F06D56CEDC2C2B2C09CF667
:10BF940072DC3635E720E536B13FBBF98F15BEC3F9
:10BFA400BFD2BFD2BEC38F15BBF9B13FE536E72080
:10BFB400363572DC9CF6B2C0C2C26CED06D56B2F6E
:10BFC4007D18203BEC3F23032B1E8FC7E1D999CC6E
:10BFD4003BC17C0C74F0143E79319928DA39A3E41E
:10BFE400000000C026C6A3E487CE99288C0F143E17
:10BFF400C53E7C0C1F2699CCD5E18FC714C0230302
:10C0040083E7203BFA2A6B2F3E3D6CED6409B2C0F6
:10C01400CACA72DC1BC9E7204506B13F423C8F15F2
:10C02400412DBFD271EABEC34FC0BBF919DFE5365B
:10C034008E2336354E3F9CF69412C2C295D006D557
:10C04400E0C47D18DDFCEC3F71382B1E6733E1D969
:10C0540084F33BC1ECC174F067D779315D1BDA39E5
:10C06400004000005D1B26C667D787CEECC18C0F4D
:10C0740084F3C53E67331F267138D5E1DDFC14C057
:10C08400E0C483E795D0FA2A94123E3D4E3F6409FA
:10C094008E23CACA19DF1BC94FC0450671EA423C48
:10C0A400412D412D423C71EA45064FC01BC919DFA1
:10C0B400CACA8E2364094E3F3E3D9412FA2A95D093
:10C0C40083E7E0C414C0DDFCD5E171381F26673373
:10C0D400C53E84F38C0FECC187CE67D726C65D1BA3
:10C0E40000000040DA395D1B793167D774F0ECC188
:10C0F4003BC184F3E1D967332B1E7138EC3FDDFC7F
:10C104007D18E0C406D595D0C2C294129CF64E3F69
:10C1140036358E23E53619DFBBF94FC0BEC371EA4D
:10C12400BFD2412D8F15423CB13F4506E7201BC9C4
:10C1340072DCCACAB2C064096CED3E3D6B2FFA2AA8
:10C14400203B83E7230314C08FC7D5E199CC1F2676
:10C154007C0CC53E143E8C0F992887CEA3E426C6DA
:10C1640000C00000A3E4DA3999287931143E74F050
:10C174007C0C3BC199CCE1D98FC72B1E2303EC3F28
:10C18400203B7D186B2F06D56CEDC2C2B2C09CF665
:10C1940072DC3635E720E536B13FBBF98F15BEC3F7
:10C1A400BFD2BFD2BEC38F15BBF9B13FE536E7207E
:10C1B400363572DC9CF6B2C0C2C26CED06D56B2F6C
:10C1C4007D18203BEC3F23032B1E8FC7E1D999CC6C
:10C1D4003BC17C0C74F0143E79319928DA39A3E41C
:10C1E400000000C026C6A3E487CE99288C0F143E15
:10C1F400C53E7C0C1F2699CCD5E18FC714C0230300
:10C2040083E7203BFA2A6B2F3E3D6CED6409B2C0F4
:10C21400CACA72DC1BC9E7204506B13F423C8F15F0
:10C22400412DBFD271EABEC34FC0BBF919DFE53659
:10C234008E2336354E3F9CF69412C2C295D006D555
:10C24400E0C47D18DDFCEC3F71382B1E6733E1D967
:10C2540084F33BC1ECC174F067D779315D1BDA39E3
:10C26400004000005D1B26C667D787CEECC18C0F4B
:10C2740084F3C53E67331F267138D5E1DDFC14C055
:10C28400E0C483E795D0FA2A94123E3D4E3F6409F8
:10C294008E23CACA19DF1BC94FC0450671EA423C46
:10C2A400412D412D423C71EA45064FC01BC919DF9F
:10C2B400CACA8E2364094E3F3E3D9412FA2A95D091
:10C2C40083E7E0C414C0DDFCD5E171381F26673371
:10C2D400C53E84F38C0FECC187CE67D726C65D1BA1
:10C2E40000000040DA395D1B793167D774F0ECC186
:10C2F4003BC184F3E1D967332B1E7138EC3FDDFC7D
:10C304007D18E0C406D595D0C2C294129CF64E3F67
:10C3140036358E23E53619DFBBF94FC0BEC371EA4B
:10C32400BFD2412D8F15423CB13F4506E7201BC9C2
:10C3340072DCCACAB2C064096CED3E3D6B2FFA2AA6
:10C34400203B83E7230314C08FC7D5E199CC1F2674
:10C354007C0CC53E143E8C0F992887CEA3E426C6D8
:10C3640000C00000A3E4DA3999287931143E74F04E
:10C374007C0C3BC199CCE1D98FC72B1E2303EC3F26
:10C38400203B7D186B2F06D56CEDC2C2B2C09CF663
:10C3940072DC3635E720E536B13FBBF98F15BEC3F5
:10C3A400BFD2BFD2BEC38F15BBF9B13FE536E7207C
:10C3B400363572DC9CF6B2C0C2C26CED06D56B2F6A
:10C3C4007D18203BEC3F23032B1E8FC7E1D999CC6A
:10C3D4003BC17C0C74F0143E79319928DA39A3E41A
:10C3E400000000C026C6A3E487CE99288C0F143E13
:10C3F400C53E7C0C1F2699CCD5E18FC714C02303FE
:10C4040083E7203BFA2A6B2F3E3D6CED6409B2C0F2
:10C41400CACA72DC1BC9E7204506B13F423C8F15EE
:10C42400412DBFD271EABEC34FC0BBF919DFE53657
:10C434008E2336354E3F9CF69412C2C295D006D553
:10C44400E0C47D18DDFCEC3F71382B1E6733E1D965
:10C4540084F33BC1ECC174F067D779315D1BDA39E1
:10C46400004000005D1B26C667D787CEECC18C0F49
:10C4740084F3C53E67331F267138D5E1DDFC14C053
:10C48400E0C483E795D0FA2A94123E3D4E3F6409F6
:10C494008E23CACA19DF1BC94FC0450671EA423C44
:10C4A400412D412D423C71EA45064FC01BC919DF9D
:10C4B400CACA8E2364094E3F3E3D9412FA2A95D08F
:10C4C40083E7E0C414C0DDFCD5E171381F2667336F
:10C4D400C53E84F38C0FECC187CE67D726C65D1B9F
:10C4E40000000040DA395D1B793167D774F0ECC184
:10C4F4003BC184F3E1D967332B1E7138EC3FDDFC7B
:10C504007D18E0C406D595D0C2C294129CF64E3F65
:10C5140036358E23E53619DFBBF94FC0BEC371EA49
:10C52400BFD2412D8F15423CB13F4506E7201BC9C0
:10C5340072DCCACAB2C064096CED3E3D6B2FFA2AA4
:10C54400203B83E7230314C08FC7D5E199CC1F2672
:10C554007C0CC53E143E8C0F992887CEA3E426C6D6
:10C5640000C00000A3E4DA3999287931143E74F04C
:10C574007C0C3BC199CCE1D98FC72B1E2303EC3F24
:10C58400203B7D186B2F06D56CEDC2C2B2C09CF661
:10C5940072DC3635E720E536B13FBBF98F15BEC3F3
:10C5A400BFD2BFD2BEC38F15BBF9B13FE536E7207A
:10C5B400363572DC9CF6B2C0C2C26CED06D56B2F68
:10C5C4007D18203BEC3F23032B1E8FC7E1D999CC68
:10C5D4003BC17C0C74F0143E79319928DA39A3E418
:10C5E400000000C026C6A3E487CE99288C0F143E11
:10C5F400C53E7C0C1F2699CCD5E18FC714C02303FC
:10C6040083E7203BFA2A6B2F3E3D6CED6409B2C0F0
:10C61400CACA72DC1BC9E7204506B13F423C8F15EC
:10C62400412DBFD271EABEC34FC0BBF919DFE53655
:10C634008E2336354E3F9CF69412C2C295D006D551
:10C64400E0C47D18DDFCEC3F71382B1E6733E1D963
:10C6540084F33BC1ECC174F067D779315D1BDA39DF
:10C66400004000005D1B26C667D787CEECC18C0F47
:10C6740084F3C53E67331F267138D5E1DDFC14C051
:10C68400E0C483E795D0FA2A94123E3D4E3F6409F4
:10C694008E23CACA19DF1BC94FC0450671EA423C42
:10C6A400412D412D423C71EA45064FC01BC919DF9B
:10C6B400CACA8E2364094E3F3E3D9412FA2A95D08D
:10C6C40083E7E0C414C0DDFCD5E171381F2667336D
:10C6D400C53E84F38C0FECC187CE67D726C65D1B9D
:10C6E4000000004079319928C53E84F32B1E8FC782
:10C6F40083E7E0C4C2C26CEDCACA8E23BBF9B13F62
:10C70400412D412DB13FBBF98E23CACA6CEDC2C283
:10C71400E0C483E78FC72B1E84F3C53E9928793183
:10C7240000400000992887CE84F33BC18FC7D5E130
:10C73400E0C47D186CED3E3D8E233635B13F450691
:10C74400412DBFD2BBF94FC0CACA72DCC2C2941217
:10C7540083E7203B2B1E7138C53E7C0C793167D7AB
:10C76400000000C087CE67D73BC17C0CD5E171388F
:10C774007D18203B3E3D9412363572DC45064FC091
:10C78400BFD2BFD24FC0450672DC363594123E3D4F
:10C79400203B7D187138D5E17C0C3BC167D787CE2F
:10C7A40000C0000067D779317C0CC53E71382B1E60
:10C7B400203B83E79412C2C272DCCACA4FC0BBF9E1
:10C7C400BFD2412D4506B13F36358E233E3D6CED3B
:10C7D4007D18E0C4D5E18FC73BC184F387CE992887
:10C7E4000000004079319928C53E84F32B1E8FC781
:10C7F40083E7E0C4C2C26CEDCACA8E23BBF9B13F61
:10C80400412D412DB13FBBF98E23CACA6CEDC2C282
:10C81400E0C483E78FC72B1E84F3C53E9928793182
:10C8240000400000992887CE84F33BC18FC7D5E12F
:10C83400E0C47D186CED3E3D8E233635B13F450690
:10C84400412DBFD2BBF94FC0CACA72DCC2C2941216
:10C8540083E7203B2B1E7138C53E7C0C793167D7AA
:10C86400000000C087CE67D73BC17C0CD5E171388E
:10C874007D18203B3E3D9412363572DC45064FC090
:10C88400BFD2BFD24FC0450672DC363594123E3D4E
:10C89400203B7D187138D5E17C0C3BC167D787CE2E
:10C8A40000C0000067D779317C0CC53E71382B1E5F
:10C8B400203B83E79412C2C272DCCACA4FC0BBF9E0
:10C8C400BFD2412D4506B13F36358E233E3D6CED3A
:10C8D4007D18E0C4D5E18FC73BC184F387CE992886
:10C8E4000000004079319928C53E84F32B1E8FC780
:10C8F40083E7E0C4C2C26CEDCACA8E23BBF9B13F60
:10C90400412D412DB13FBBF98E23CACA6CEDC2C281
:10C91400E0C483E78FC72B1E84F3C53E9928793181
:10C9240000400000992887CE84F33BC18FC7D5E12E
:10C93400E0C47D186CED3E3D8E233635B13F45068F
:10C94400412DBFD2BBF94FC0CACA72DCC2C2941215
:10C9540083E7203B2B1E7138C53E7C0C793167D7A9
:10C96400000000C087CE67D73BC17C0CD5E171388D
:10C974007D18203B3E3D9412363572DC45064FC08F
:10C98400BFD2BFD24FC0450672DC363594123E3D4D
:10C99400203B7D187138D5E17C0C3BC167D787CE2D
:10C9A40000C0000067D779317C0CC53E71382B1E5E
:10C9B400203B83E79412C2C272DCCACA4FC0BBF9DF
:10C9C400BFD2412D4506B13F36358E233E3D6CED39
:10C9D4007D18E0C4D5E18FC73BC184F387CE992885
:10C9E4000000004079319928C53E84F32B1E8FC77F
:10C9F40083E7E0C4C2C26CEDCACA8E23BBF9B13F5F
:10CA0400412D412DB13FBBF98E23CACA6CEDC2C280
:10CA1400E0C483E78FC72B1E84F3C53E9928793180
:10CA240000400000992887CE84F33BC18FC7D5E12D
:10CA3400E0C47D186CED3E3D8E233635B13F45068E
:10CA4400412DBFD2BBF94FC0CACA72DCC2C2941214
:10CA540083E7203B2B1E7138C53E7C0C793167D7A8
:10CA6400000000C087CE67D73BC17C0CD5E171388C
:10CA74007D18203B3E3D9412363572DC45064FC08E
:10CA8400BFD2BFD24FC0450672DC363594123E3D4C
:10CA9400203B7D187138D5E17C0C3BC167D787CE2C
:10CAA40000C0000067D779317C0CC53E71382B1E5D
:10CAB400203B83E79412C2C272DCCACA4FC0BBF9DE
:10CAC400BFD2412D4506B13F36358E233E3D6CED38
:10CAD4007D18E0C4D5E18FC73BC184F387CE992884
:10CAE4000000004079319928C53E84F32B1E8FC77E
:10CAF40083E7E0C4C2C26CEDCACA8E23BBF9B13F5E
:10CB0400412D412DB13FBBF98E23CACA6CEDC2C27F
:10CB1400E0C483E78FC72B1E84F3C53E992879317F
:10CB240000400000992887CE84F33BC18FC7D5E12C
:10CB3400E0C47D186CED3E3D8E233635B13F45068D
:10CB4400412DBFD2BBF94FC0CACA72DCC2C2941213
:10CB540083E7203B2B1E7138C53E7C0C793167D7A7
:10CB6400000000C087CE67D73BC17C0CD5E171388B
:10CB74007D18203B3E3D9412363572DC45064FC08D
:10CB8400BFD2BFD24FC0450672DC363594123E3D4B
:10CB9400203B7D187138D5E17C0C3BC167D787CE2B
:10CBA40000C0000067D779317C0CC53E71382B1E5C
:10CBB400203B83E79412C2C272DCCACA4FC0BBF9DD
:10CBC400BFD2412D4506B13F36358E233E3D6CED37
:10CBD4007D18E0C4D5E18FC73BC184F387CE992883
:10CBE4000000004079319928C53E84F32B1E8FC77D
:10CBF40083E7E0C4C2C26CEDCACA8E23BBF9B13F5D
:10CC0400412D412DB13FBBF98E23CACA6CEDC2C27E
:10CC1400E0C483E78FC72B1E84F3C53E992879317E
:10CC240000400000992887CE84F33BC18FC7D5E12B
:10CC3400E0C47D186CED3E3D8E233635B13F45068C
:10CC4400412DBFD2BBF94FC0CACA72DCC2C2941212
:10CC540083E7203B2B1E7138C53E7C0C793167D7A6
:10CC6400000000C087CE67D73BC17C0CD5E171388A
:10CC74007D18203B3E3D9412363572DC45064FC08C
:10CC8400BFD2BFD24FC0450672DC363594123E3D4A
:10CC9400203B7D187138D5E17C0C3BC167D787CE2A
:10CCA40000C0000067D779317C0CC53E71382B1E5B
:10CCB400203B83E79412C2C272DCCACA4FC0BBF9DC
:10CCC400BFD2412D4506B13F36358E233E3D6CED36
:10CCD4007D18E0C4D5E18FC73BC184F387CE992882
:10CCE4000000004079319928C53E84F32B1E8FC77C
:10CCF40083E7E0C4C2C26CEDCACA8E23BBF9B13F5C
:10CD0400412D412DB13FBBF98E23CACA6CEDC2C27D
:10CD1400E0C483E78FC72B1E84F3C53E992879317D
:10CD240000400000992887CE84F33BC18FC7D5E12A
:10CD3400E0C47D186CED3E3D8E233635B13F45068B
:10CD4400412DBFD2BBF94FC0CACA72DCC2C2941211
:10CD540083E7203B2B1E7138C53E7C0C793167D7A5
:10CD6400000000C087CE67D73BC17C0CD5E1713889
:10CD74007D18203B3E3D9412363572DC45064FC08B
:10CD8400BFD2BFD24FC0450672DC363594123E3D49
:10CD9400203B7D187138D5E17C0C3BC167D787CE29
:10CDA40000C0000067D779317C0CC53E71382B1E5A
:10CDB400203B83E79412C2C272DCCACA4FC0BBF9DB
:10CDC400BFD2412D4506B13F36358E233E3D6CED35
:10CDD4007D18E0C4D5E18FC73BC184F387CE992881
:10CDE4000000004079319928C53E84F32B1E8FC77B
:10CDF40083E7E0C4C2C26CEDCACA8E23BBF9B13F5B
:10CE0400412D412DB13FBBF98E23CACA6CEDC2C27C
:10CE1400E0C483E78FC72B1E84F3C53E992879317C
:10CE240000400000992887CE84F33BC18FC7D5E129
:10CE3400E0C47D186CED3E3D8E233635B13F45068A
:10CE4400412DBFD2BBF94FC0CACA72DCC2C2941210
:10CE540083E7203B2B1E7138C53E7C0C793167D7A4
:10CE6400000000C087CE67D73BC17C0CD5E1713888
:10CE74007D18203B3E3D9412363572DC45064FC08A
:10CE8400BFD2BFD24FC0450672DC363594123E3D48
:10CE9400203B7D187138D5E17C0C3BC167D787CE28
:10CEA40000C0000067D779317C0CC53E71382B1E59
:10CEB400203B83E79412C2C272DCCACA4FC0BBF9DA
:10CEC400BFD2412D4506B13F36358E233E3D6CED34
:10CED4007D18E0C4D5E18FC73BC184F387CE992880
:10CEE4000000004012363D22DA39A3E4D5077CC0A5
:10CEF40087CE67D73BC3131474F0143E212C5A2EEB
:10CF0400C53E84F308174AC4E1D999CC2DC0B504B1
:10CF1400D5E171388B1FAF37EC3F2303DA24ADCB57
:10CF240083E7E0C4F2C00FF506D56B2F1111AE3DB7
:10CF34003E3D9412763033D69CF6B2C07EC511E6DF
:10CF4400CACA8E239201FB3FE536E7202A393AE329
:10CF540045064FC08CCDA1D8BEC38F15FBF1713EE1
:10CF6400412D412D713EFBF18F15BEC3A1D88CCD4F
:10CF74004FC045063AE32A39E720E536FB3F9201E4
:10CF84008E23CACA11E67EC5B2C09CF633D676306B
:10CF940094123E3DAE3D11116B2F06D50FF5F2C034
:10CFA400E0C483E7ADCBDA242303EC3FAF378B1F18
:10CFB4007138D5E1B5042DC099CCE1D94AC408171C
:10CFC40084F3C53E5A2E212C143E74F013143BC333
:10CFD40067D787CE7CC0D507A3E4DA393D22123661
:10CFE400004000003D22EEC9A3E426C67CC02BF815
:10CFF40067D779311314C53C143E8C0F5A2EDFD3F6
:10D0040084F33BC14AC4F8E899CC1F26B504D33F46
:10D0140071382B1EAF3775E0230314C0ADCB26DB6C
:10D02400E0C47D180FF50E3F6B2FFA2AAE3DEFEEEC
:10D034009412C2C233D68ACFB2C0640911E6823ACE
:10D044008E233635FB3F6EFEE7201BC93AE3D6C676
:10D054004FC0BBF9A1D874328F15423C713E050E06
:10D06400412DBFD2FBF18FC1BEC371EA8CCD5F27C6
:10D074004506B13F2A39C61CE53619DF920105C0C1
:10D08400CACA72DC7EC5EF199CF64E3F7630CD29B4
:10D094003E3D6CED111152C206D595D0F2C0F10A95
:10D0A40083E7203BDA245334EC3FDDFC8B1F51C86B
:10D0B400D5E18FC72DC04BFBE1D967330817B63BC9
:10D0C400C53E7C0C212CA6D174F0ECC13BC3EDEB26
:10D0D40087CE9928D507843FDA395D1B1236C3DD24
:10D0E400000000C0EEC9C3DD26C65D1B2BF8843FDB
:10D0F40079319928C53CEDEB8C0FECC1DFD3A6D177
:10D104003BC17C0CF8E8B63B1F266733D33F4BFB8F
:10D114002B1E8FC775E051C814C0DDFC26DB5334C9
:10D124007D18203B0E3FF10AFA2A95D0EFEE52C249
:10D13400C2C26CED8ACFCD2964094E3F823AEF1901
:10D14400363572DC6EFE05C01BC919DFD6C6C61C97
:10D15400BBF9B13F74325F27423C71EA050E8FC1BF
:10D16400BFD2BFD28FC1050E71EA423C5F27743231
:10D17400B13FBBF9C61CD6C619DF1BC905C06EFE7C
:10D1840072DC3635EF19823A4E3F6409CD298ACFD5
:10D194006CEDC2C252C2EFEE95D0FA2AF10A0E3FEC
:10D1A400203B7D18533426DBDDFC14C051C875E0E8
:10D1B4008FC72B1E4BFBD33F67331F26B63BF8E8C4
:10D1C4007C0C3BC1A6D1DFD3ECC18C0FEDEBC53C8D
:10D1D40099287931843F2BF85D1B26C6C3DDEEC93F
:10D1E40000C00000C3DD12365D1BDA39843FD50769
:10D1F400992887CEEDEB3BC3ECC174F0A6D1212C6A
:10D204007C0CC53EB63B08176733E1D94BFB2DC0F8
:10D214008FC7D5E151C88B1FDDFCEC3F5334DA24B2
:10D22400203B83E7F10AF2C095D006D552C2111112
:10D234006CED3E3DCD2976304E3F9CF6EF197EC510
:10D2440072DCCACA05C0920119DFE536C61C2A3948
:10D25400B13F45065F278CCD71EABEC38FC1FBF198
:10D26400BFD2412D050E713E423C8F157432A1D8B8
:10D27400BBF94FC0D6C63AE31BC9E7206EFEFB3F9D
:10D2840036358E23823A11E66409B2C08ACF33D68A
:10D29400C2C29412EFEEAE3DFA2A6B2F0E3F0FF589
:10D2A4007D18E0C426DBADCB14C0230375E0AF3793
:10D2B4002B1E7138D33FB5041F2699CCF8E84AC415
:10D2C4003BC184F3DFD35A2E8C0F143EC53C131498
:10D2D400793167D72BF87CC026C6A3E4EEC93D227A
:10D2E4000000004012363D22DA39A3E4D5077CC0A1
:10D2F40087CE67D73BC3131474F0143E212C5A2EE7
:10D30400C53E84F308174AC4E1D999CC2DC0B504AD
:10D31400D5E171388B1FAF37EC3F2303DA24ADCB53
:10D3240083E7E0C4F2C00FF506D56B2F1111AE3DB3
:10D334003E3D9412763033D69CF6B2C07EC511E6DB
:10D34400CACA8E239201FB3FE536E7202A393AE325
:10D3540045064FC08CCDA1D8BEC38F15FBF1713EDD
:10D36400412D412D713EFBF18F15BEC3A1D88CCD4B
:10D374004FC045063AE32A39E720E536FB3F9201E0
:10D384008E23CACA11E67EC5B2C09CF633D6763067
:10D3940094123E3DAE3D11116B2F06D50FF5F2C030
:10D3A400E0C483E7ADCBDA242303EC3FAF378B1F14
:10D3B4007138D5E1B5042DC099CCE1D94AC4081718
:10D3C40084F3C53E5A2E212C143E74F013143BC32F
:10D3D40067D787CE7CC0D507A3E4DA393D2212365D
:10D3E400004000003D22EEC9A3E426C67CC02BF811
:10D3F40067D779311314C53C143E8C0F5A2EDFD3F2
:10D4040084F33BC14AC4F8E899CC1F26B504D33F42
:10D4140071382B1EAF3775E0230314C0ADCB26DB68
:10D42400E0C47D180FF50E3F6B2FFA2AAE3DEFEEE8
:10D434009412C2C233D68ACFB2C0640911E6823ACA
:10D444008E233635FB3F6EFEE7201BC93AE3D6C672
:10D454004FC0BBF9A1D874328F15423C713E050E02
:10D46400412DBFD2FBF18FC1BEC371EA8CCD5F27C2
:10D474004506B13F2A39C61CE53619DF920105C0BD
:10D48400CACA72DC7EC5EF199CF64E3F7630CD29B0
:10D494003E3D6CED111152C206D595D0F2C0F10A91
:10D4A40083E7203BDA245334EC3FDDFC8B1F51C867
:10D4B400D5E18FC72DC04BFBE1D967330817B63BC5
:10D4C400C53E7C0C212CA6D174F0ECC13BC3EDEB22
:10D4D40087CE9928D507843FDA395D1B1236C3DD20
:10D4E400000000C0EEC9C3DD26C65D1B2BF8843FD7
:10D4F40079319928C53CEDEB8C0FECC1DFD3A6D173
:10D504003BC17C0CF8E8B63B1F266733D33F4BFB8B
:10D514002B1E8FC775E051C814C0DDFC26DB5334C5
:10D524007D18203B0E3FF10AFA2A95D0EFEE52C245
:10D53400C2C26CED8ACFCD2964094E3F823AEF19FD
:10D54400363572DC6EFE05C01BC919DFD6C6C61C93
:10D55400BBF9B13F74325F27423C71EA050E8FC1BB
:10D56400BFD2BFD28FC1050E71EA423C5F2774322D
:10D57400B13FBBF9C61CD6C619DF1BC905C06EFE78
:10D5840072DC3635EF19823A4E3F6409CD298ACFD1
:10D594006CEDC2C252C2EFEE95D0FA2AF10A0E3FE8
:10D5A400203B7D18533426DBDDFC14C051C875E0E4
:10D5B4008FC72B1E4BFBD33F67331F26B63BF8E8C0
:10D5C4007C0C3BC1A6D1DFD3ECC18C0FEDEBC53C89
:10D5D40099287931843F2BF85D1B26C6C3DDEEC93B
:10D5E40000C00000C3DD12365D1BDA39843FD50765
:10D5F400992887CEEDEB3BC3ECC174F0A6D1212C66
:10D604007C0CC53EB63B08176733E1D94BFB2DC0F4
:10D614008FC7D5E151C88B1FDDFCEC3F5334DA24AE
:10D62400203B83E7F10AF2C095D006D552C211110E
:10D634006CED3E3DCD2976304E3F9CF6EF197EC50C
:10D6440072DCCACA05C0920119DFE536C61C2A3944
:10D65400B13F45065F278CCD71EABEC38FC1FBF194
:10D66400BFD2412D050E713E423C8F157432A1D8B4
:10D67400BBF94FC0D6C63AE31BC9E7206EFEFB3F99
:10D6840036358E23823A11E66409B2C08ACF33D686
:10D69400C2C29412EFEEAE3DFA2A6B2F0E3F0FF585
:10D6A4007D18E0C426DBADCB14C0230375E0AF378F
:10D6B4002B1E7138D33FB5041F2699CCF8E84AC411
:10D6C4003BC184F3DFD35A2E8C0F143EC53C131494
:10D6D400793167D72BF87CC026C6A3E4EEC93D2276
:10D6E4000000004000400000000000C000C0000036
:10D6F4000000004000400000000000C000C0000026
:10D704000000004000400000000000C000C0000015
:10D714000000004000400000000000C000C0000005
:10D724000000004000400000000000C000C00000F5
:10D734000000004000400000000000C000C00000E5
:10D744000000004000400000000000C000C00000D5
:10D754000000004000400000000000C000C00000C5
:10D764000000004000400000000000C000C00000B5
:10D774000000004000400000000000C000C00000A5
:10D784000000004000400000000000C000C0000095
:10D794000000004000400000000000C000C0000085
:10D7A4000000004000400000000000C000C0000075
:10D7B4000000004000400000000000C000C0000065
:10D7C4000000004000400000000000C000C0000055
:10D7D4000000004000400000000000C000C0000045
:10D7E4000000004000400000000000C000C0000035
:10D7F4000000004000400000000000C000C0000025
:10D804000000004000400000000000C000C0000014
:10D814000000004000400000000000C000C0000004
:10D824000000004000400000000000C000C00000F4
:10D834000000004000400000000000C000C00000E4
:10D844000000004000400000000000C000C00000D4
:10D854000000004000400000000000C000C00000C4
:10D864000000004000400000000000C000C00000B4
:10D874000000004000400000000000C000C00000A4
:10D884000000004000400000000000C000C0000094
:10D894000000004000400000000000C000C0000084
:10D8A4000000004000400000000000C000C0000074
:10D8B4000000004000400000000000C000C0000064
:10D8C4000000004000400000000000C000C0000054
:10D8D4000000004000400000000000C000C0000044
:10D8E4000000004000400000000000C000C0000034
:10D8F4000000004000400000000000C000C0000024
:10D904000000004000400000000000C000C0000013
:10D914000000004000400000000000C000C0000003
:10D924000000004000400000000000C000C00000F3
:10D934000000004000400000000000C000C00000E3
:10D944000000004000400000000000C000C00000D3
:10D954000000004000400000000000C000C00000C3
:10D964000000004000400000000000C000C00000B3
:10D974000000004000400000000000C000C00000A3
:10D984000000004000400000000000C000C0000093
:10D994000000004000400000000000C000C0000083
:10D9A4000000004000400000000000C000C0000073
:10D9B4000000004000400000000000C000C0000063
:10D9C4000000004000400000000000C000C0000053
:10D9D4000000004000400000000000C000C0000043
:10D9E4000000004000400000000000C000C0000033
:10D9F4000000004000400000000000C000C0000023
:10DA04000000004000400000000000C000C0000012
:10DA14000000004000400000000000C000C0000002
:10DA24000000004000400000000000C000C00000F2
:10DA34000000004000400000000000C000C00000E2
:10DA44000000004000400000000000C000C00000D2
:10DA54000000004000400000000000C000C00000C2
:10DA64000000004000400000000000C000C00000B2
:10DA74000000004000400000000000C000C00000A2
:10DA84000000004000400000000000C000C0000092
:10DA94000000004000400000000000C000C0000082
:10DAA4000000004000400000000000C000C0000072
:10DAB4000000004000400000000000C000C0000062
:10DAC4000000004000400000000000C000C0000052
:10DAD4000000004000400000000000C000C0000042
:10DAE4000000004000400000000000C000C0000032
:10DAF4000000004000400000000000C000C0000022
:10DB04000000004000400000000000C000C0000011
:10DB14000000004000400000000000C000C0000001
:10DB24000000004000400000000000C000C00000F1
:10DB34000000004000400000000000C000C00000E1
:10DB44000000004000400000000000C000C00000D1
:10DB54000000004000400000000000C000C00000C1
:10DB64000000004000400000000000C000C00000B1
:10DB74000000004000400000000000C000C00000A1
:10DB84000000004000400000000000C000C0000091
:10DB94000000004000400000000000C000C0000081
:10DBA4000000004000400000000000C000C0000071
:10DBB4000000004000400000000000C000C0000061
:10DBC4000000004000400000000000C000C0000051
:10DBD4000000004000400000000000C000C0000041
:10DBE4000000004000400000000000C000C0000031
:10DBF4000000004000400000000000C000C0000021
:10DC04000000004000400000000000C000C0000010
:10DC14000000004000400000000000C000C0000000
:10DC24000000004000400000000000C000C00000F0
:10DC34000000004000400000000000C000C00000E0
:10DC44000000004000400000000000C000C00000D0
:10DC54000000004000400000000000C000C00000C0
:10DC64000000004000400000000000C000C00000B0
:10DC74000000004000400000000000C000C00000A0
:10DC84000000004000400000000000C000C0000090
:10DC94000000004000400000000000C000C0000080
:10DCA4000000004000400000000000C000C0000070
:10DCB4000000004000400000000000C000C0000060
:10DCC4000000004000400000000000C000C0000050
:10DCD4000000004000400000000000C000C0000040
:10DCE4000000004000400000000000C000C0000030
:10DCF4000000004000400000000000C000C0000020
:10DD04000000004000400000000000C000C000000F
:10DD14000000004000400000000000C000C00000FF
:10DD24000000004000400000000000C000C00000EF
:10DD34000000004000400000000000C000C00000DF
:10DD44000000004000400000000000C000C00000CF
:10DD54000000004000400000000000C000C00000BF
:10DD64000000004000400000000000C000C00000AF
:10DD74000000004000400000000000C000C000009F
:10DD84000000004000400000000000C000C000008F
:10DD94000000004000400000000000C000C000007F
:10DDA4000000004000400000000000C000C000006F
:10DDB4000000004000400000000000C000C000005F
:10DDC4000000004000400000000000C000C000004F
:10DDD4000000004000400000000000C000C000003F
:10DDE4000000004000400000000000C000C000002F
:10DDF4000000004000400000000000C000C000001F
:10DE04000000004000400000000000C000C000000E
:10DE14000000004000400000000000C000C00000FE
:10DE24000000004000400000000000C000C00000EE
:10DE34000000004000400000000000C000C00000DE
:10DE44000000004000400000000000C000C00000CE
:10DE54000000004000400000000000C000C00000BE
:10DE64000000004000400000000000C000C00000AE
:10DE74000000004000400000000000C000C000009E
:10DE84000000004000400000000000C000C000008E
:10DE94000000004000400000000000C000C000007E
:10DEA4000000004000400000000000C000C000006E
:10DEB4000000004000400000000000C000C000005E
:10DEC4000000004000400000000000C000C000004E
:10DED4000000004000400000000000C000C000003E
:10DEE40000000040C53C13141F2699CC26DBADCBA3
:10DEF400C2C294126EFEFB3F423C8F155F278CCD4D
:10DF040072DCCACA52C21111DDFCEC3FB63B0817E1
:10DF1400992887CEC3DDEEC9ECC18C0F4BFBD33FF0
:10DF2400203B7D18CD298ACF19DF1BC98FC1050E6F
:10DF3400BBF9B13F823AEF19FA2A95D075E051C87E
:10DF44003BC17C0C2BF8843FDA395D1B212CA6D114
:10DF5400D5E18FC7F2C0F10A9CF64E3F2A39C61CA0
:10DF6400412DBFD23AE3D6C6B2C064090FF50E3FC5
:10DF740071382B1E5A2EDFD3A3E426C67CC0D507E6
:10DF840084F3C53EAF378B1F6B2F06D511E67EC5D4
:10DF94004FC04506FBF1713EE536E720763033D6B7
:10DFA40083E7E0C42DC0B50474F0143E12363D225C
:10DFB400793167D7F8E84AC414C02303EFEEAE3DC5
:10DFC40036358E237432A1D871EABEC305C09201DE
:10DFD4006CED3E3D5334DA246733E1D9EDEB3BC3BA
:10DFE40000C00000EDEBC53C67331F26533426DB2D
:10DFF4006CEDC2C205C06EFE71EA423C74325F270A
:10E00400363572DCEFEE52C214C0DDFCF8E8B63BE4
:10E01400793199281236C3DD74F0ECC12DC04BFB65
:10E0240083E7203B7630CD29E53619DFFBF18FC13C
:10E034004FC0BBF911E6823A6B2FFA2AAF3775E06D
:10E0440084F33BC17CC02BF8A3E4DA395A2E212C8B
:10E054007138D5E10FF5F2C0B2C09CF63AE32A3923
:10E06400412D412D2A393AE39CF6B2C0F2C00FF596
:10E07400D5E17138212C5A2EDA39A3E42BF87CC06F
:10E084003BC184F375E0AF37FA2A6B2F823A11E66D
:10E09400BBF94FC08FC1FBF119DFE536CD297630CE
:10E0A400203B83E74BFB2DC0ECC174F0C3DD12367B
:10E0B40099287931B63BF8E8DDFC14C052C2EFEE82
:10E0C40072DC36355F277432423C71EA6EFE05C05D
:10E0D400C2C26CED26DB53341F266733C53CEDEB1F
:10E0E400000000C03BC3EDEBE1D96733DA245334BD
:10E0F4003E3D6CED920105C0BEC371EAA1D87432F5
:10E104008E233635AE3DEFEE230314C04AC4F8E83F
:10E1140067D779313D221236143E74F0B5042DC010
:10E12400E0C483E733D67630E720E536713EFBF171
:10E1340045064FC07EC511E606D56B2F8B1FAF3742
:10E14400C53E84F3D5077CC026C6A3E4DFD35A2E8C
:10E154002B1E71380E3F0FF56409B2C0D6C63AE3E0
:10E16400BFD2412DC61C2A394E3F9CF6F10AF2C09B
:10E174008FC7D5E1A6D1212C5D1BDA39843F2BF85A
:10E184007C0C3BC151C875E095D0FA2AEF19823A4C
:10E19400B13FBBF9050E8FC11BC919DF8ACFCD2949
:10E1A4007D18203BD33F4BFB8C0FECC1EEC9C3DD84
:10E1B40087CE99280817B63BEC3FDDFC111152C2FB
:10E1C400CACA72DC8CCD5F278F15423CFB3F6EFEC2
:10E1D4009412C2C2ADCB26DB99CC1F261314C53CC6
:10E1E4000040000013143BC399CCE1D9ADCBDA2431
:10E1F40094123E3DFB3F92018F15BEC38CCDA1D836
:10E20400CACA8E231111AE3DEC3F230308174AC43A
:10E2140087CE67D7EEC93D228C0F143ED33FB50499
:10E224007D18E0C48ACF33D61BC9E720050E713EA2
:10E23400B13F4506EF197EC595D006D551C88B1F51
:10E244007C0CC53E843FD5075D1B26C6A6D1DFD313
:10E254008FC72B1EF10A0E3F4E3F6409C61CD6C65B
:10E26400BFD2BFD2D6C6C61C64094E3F0E3FF10AC8
:10E274002B1E8FC7DFD3A6D126C65D1BD507843FCF
:10E28400C53E7C0C8B1F51C806D595D07EC5EF19B1
:10E294004506B13F713E050EE7201BC933D68ACF30
:10E2A400E0C47D18B504D33F143E8C0F3D22EEC963
:10E2B40067D787CE4AC408172303EC3FAE3D11113C
:10E2C4008E23CACAA1D88CCDBEC38F159201FB3F41
:10E2D4003E3D9412DA24ADCBE1D999CC3BC313145F
:10E2E40000000040C53C13141F2699CC26DBADCB9F
:10E2F400C2C294126EFEFB3F423C8F155F278CCD49
:10E3040072DCCACA52C21111DDFCEC3FB63B0817DD
:10E31400992887CEC3DDEEC9ECC18C0F4BFBD33FEC
:10E32400203B7D18CD298ACF19DF1BC98FC1050E6B
:10E33400BBF9B13F823AEF19FA2A95D075E051C87A
:10E344003BC17C0C2BF8843FDA395D1B212CA6D110
:10E35400D5E18FC7F2C0F10A9CF64E3F2A39C61C9C
:10E36400412DBFD23AE3D6C6B2C064090FF50E3FC1
:10E3740071382B1E5A2EDFD3A3E426C67CC0D507E2
:10E3840084F3C53EAF378B1F6B2F06D511E67EC5D0
:10E394004FC04506FBF1713EE536E720763033D6B3
:10E3A40083E7E0C42DC0B50474F0143E12363D2258
:10E3B400793167D7F8E84AC414C02303EFEEAE3DC1
:10E3C40036358E237432A1D871EABEC305C09201DA
:10E3D4006CED3E3D5334DA246733E1D9EDEB3BC3B6
:10E3E40000C00000EDEBC53C67331F26533426DB29
:10E3F4006CEDC2C205C06EFE71EA423C74325F2706
:10E40400363572DCEFEE52C214C0DDFCF8E8B63BE0
:10E41400793199281236C3DD74F0ECC12DC04BFB61
:10E4240083E7203B7630CD29E53619DFFBF18FC138
:10E434004FC0BBF911E6823A6B2FFA2AAF3775E069
:10E4440084F33BC17CC02BF8A3E4DA395A2E212C87
:10E454007138D5E10FF5F2C0B2C09CF63AE32A391F
:10E46400412D412D2A393AE39CF6B2C0F2C00FF592
:10E47400D5E17138212C5A2EDA39A3E42BF87CC06B
:10E484003BC184F375E0AF37FA2A6B2F823A11E669
:10E49400BBF94FC08FC1FBF119DFE536CD297630CA
:10E4A400203B83E74BFB2DC0ECC174F0C3DD123677
:10E4B40099287931B63BF8E8DDFC14C052C2EFEE7E
:10E4C40072DC36355F277432423C71EA6EFE05C059
:10E4D400C2C26CED26DB53341F266733C53CEDEB1B
:10E4E400000000C03BC3EDEBE1D96733DA245334B9
:10E4F4003E3D6CED920105C0BEC371EAA1D87432F1
:10E504008E233635AE3DEFEE230314C04AC4F8E83B
:10E5140067D779313D221236143E74F0B5042DC00C
:10E52400E0C483E733D67630E720E536713EFBF16D
:10E5340045064FC07EC511E606D56B2F8B1FAF373E
:10E54400C53E84F3D5077CC026C6A3E4DFD35A2E88
:10E554002B1E71380E3F0FF56409B2C0D6C63AE3DC
:10E56400BFD2412DC61C2A394E3F9CF6F10AF2C097
:10E574008FC7D5E1A6D1212C5D1BDA39843F2BF856
:10E584007C0C3BC151C875E095D0FA2AEF19823A48
:10E59400B13FBBF9050E8FC11BC919DF8ACFCD2945
:10E5A4007D18203BD33F4BFB8C0FECC1EEC9C3DD80
:10E5B40087CE99280817B63BEC3FDDFC111152C2F7
:10E5C400CACA72DC8CCD5F278F15423CFB3F6EFEBE
:10E5D4009412C2C2ADCB26DB99CC1F261314C53CC2
:10E5E4000040000013143BC399CCE1D9ADCBDA242D
:10E5F40094123E3DFB3F92018F15BEC38CCDA1D832
:10E60400CACA8E231111AE3DEC3F230308174AC436
:10E6140087CE67D7EEC93D228C0F143ED33FB50495
:10E624007D18E0C48ACF33D61BC9E720050E713E9E
:10E63400B13F4506EF197EC595D006D551C88B1F4D
:10E644007C0CC53E843FD5075D1B26C6A6D1DFD30F
:10E654008FC72B1EF10A0E3F4E3F6409C61CD6C657
:10E66400BFD2BFD2D6C6C61C64094E3F0E3FF10AC4
:10E674002B1E8FC7DFD3A6D126C65D1BD507843FCB
:10E68400C53E7C0C8B1F51C806D595D07EC5EF19AD
:10E694004506B13F713E050EE7201BC933D68ACF2C
:10E6A400E0C47D18B504D33F143E8C0F3D22EEC95F
:10E6B40067D787CE4AC408172303EC3FAE3D111138
:10E6C4008E23CACAA1D88CCDBEC38F159201FB3F3D
:10E6D4003E3D9412DA24ADCBE1D999CC3BC313145B
:10E6E40000000040D33FB5046409B2C08FC1FBF100
:10E6F4006CED3E3DB63B08175D1B26C651C875E060
:10E7040072DC363574325F27FA2A95D0DFD3A6D16E
:10E7140087CE9928DA245334E53619DF3AE3D6C68E
:10E72400E0C47D181314C53C143E74F00FF5F2C018
:10E734004FC045069201FB3FEC3F2303D5077CC045
:10E744003BC184F3EFEEAE3D423C8F15EF197EC51D
:10E754008FC7D5E1C3DD123667331F26CD298ACF93
:10E76400BFD2BFD28ACFCD291F2667331236C3DD6D
:10E77400D5E18FC77EC5EF198F15423CAE3DEFEE54
:10E7840084F33BC17CC0D5072303EC3FFB3F9201DC
:10E7940045064FC0F2C00FF574F0143EC53C131487
:10E7A4007D18E0C4D6C63AE319DFE5365334DA24DB
:10E7B400992887CEA6D1DFD395D0FA2A5F27743261
:10E7C400363572DC75E051C826C65D1B0817B63BAA
:10E7D4003E3D6CEDFBF18FC1B2C06409B504D33F7B
:10E7E40000400000B5042DC0B2C09CF6FBF1713EA0
:10E7F4003E3D941208174AC426C6A3E475E0AF3719
:10E8040036358E235F278CCD95D006D5A6D1212C05
:10E8140099287931533426DB19DF1BC9D6C6C61CA7
:10E824007D18203BC53CEDEB74F0ECC1F2C0F10A5D
:10E834004506B13FFB3F6EFE230314C07CC02BF89A
:10E8440084F3C53EAE3D11118F15BEC37EC511E6DE
:10E85400D5E1713812363D221F2699CC8ACF33D6A2
:10E86400BFD2412DCD2976306733E1D9C3DDEEC95E
:10E874008FC72B1EEF19823A423C71EAEFEE52C267
:10E884003BC17C0CD507843FEC3FDDFC920105C005
:10E894004FC0BBF90FF50E3F143E8C0F13143BC34E
:10E8A400E0C483E73AE32A39E536E720DA24ADCB3E
:10E8B40087CE67D7DFD35A2EFA2A6B2F7432A1D8AA
:10E8C40072DCCACA51C88B1F5D1BDA39B63BF8E843
:10E8D4006CEDC2C28FC1050E64094E3FD33F4BFBA2
:10E8E400000000C02DC04BFB9CF64E3F713E050E50
:10E8F4009412C2C24AC4F8E8A3E4DA39AF378B1FD2
:10E904008E23CACA8CCDA1D806D56B2F212C5A2EA2
:10E91400793167D726DBADCB1BC9E720C61C2A3962
:10E92400203B83E7EDEB3BC3ECC18C0FF10A0E3FB8
:10E93400B13FBBF96EFE05C014C0DDFC2BF8843F6B
:10E94400C53E7C0C111152C2BEC371EA11E6823A73
:10E9540071382B1E3D22EEC999CCE1D933D67630DD
:10E96400412D412D763033D6E1D999CCEEC93D22E3
:10E974002B1E7138823A11E671EABEC352C21111DC
:10E984007C0CC53E843F2BF8DDFC14C005C06EFE34
:10E99400BBF9B13F0E3FF10A8C0FECC13BC3EDEB69
:10E9A40083E7203B2A39C61CE7201BC9ADCB26DBF5
:10E9B40067D779315A2E212C6B2F06D5A1D88CCD4F
:10E9C400CACA8E238B1FAF37DA39A3E4F8E84AC4E6
:10E9D400C2C29412050E713E4E3F9CF64BFB2DC0F5
:10E9E40000C000004BFBD33F4E3F6409050E8FC1AE
:10E9F400C2C26CEDF8E8B63BDA395D1B8B1F51C817
:10EA0400CACA72DCA1D874326B2FFA2A5A2EDFD309
:10EA140067D787CEADCBDA24E720E5362A393AE347
:10EA240083E7E0C43BC313148C0F143E0E3F0FF571
:10EA3400BBF94FC005C09201DDFCEC3F843FD50714
:10EA44007C0C3BC152C2EFEE71EA423C823AEF19B0
:10EA54002B1E8FC7EEC9C3DDE1D967337630CD29CC
:10EA6400412DBFD233D68ACF99CC1F263D221236F0
:10EA74007138D5E111E67EC5BEC38F151111AE3DC7
:10EA8400C53E84F32BF87CC014C023036EFEFB3F09
:10EA9400B13F4506F10AF2C0ECC174F0EDEBC53CA0
:10EAA400203B7D18C61CD6C61BC919DF26DB533490
:10EAB40079319928212CA6D106D595D08CCD5F2704
:10EAC4008E233635AF3775E0A3E426C64AC408174B
:10EAD40094123E3D713EFBF19CF6B2C02DC0B504CC
:10EAE40000000040D33FB5046409B2C08FC1FBF1FC
:10EAF4006CED3E3DB63B08175D1B26C651C875E05C
:10EB040072DC363574325F27FA2A95D0DFD3A6D16A
:10EB140087CE9928DA245334E53619DF3AE3D6C68A
:10EB2400E0C47D181314C53C143E74F00FF5F2C014
:10EB34004FC045069201FB3FEC3F2303D5077CC041
:10EB44003BC184F3EFEEAE3D423C8F15EF197EC519
:10EB54008FC7D5E1C3DD123667331F26CD298ACF8F
:10EB6400BFD2BFD28ACFCD291F2667331236C3DD69
:10EB7400D5E18FC77EC5EF198F15423CAE3DEFEE50
:10EB840084F33BC17CC0D5072303EC3FFB3F9201D8
:10EB940045064FC0F2C00FF574F0143EC53C131483
:10EBA4007D18E0C4D6C63AE319DFE5365334DA24D7
:10EBB400992887CEA6D1DFD395D0FA2A5F2774325D
:10EBC400363572DC75E051C826C65D1B0817B63BA6
:10EBD4003E3D6CEDFBF18FC1B2C06409B504D33F77
:10EBE40000400000B5042DC0B2C09CF6FBF1713E9C
:10EBF4003E3D941208174AC426C6A3E475E0AF3715
:10EC040036358E235F278CCD95D006D5A6D1212C01
:10EC140099287931533426DB19DF1BC9D6C6C61CA3
:10EC24007D18203BC53CEDEB74F0ECC1F2C0F10A59
:10EC34004506B13FFB3F6EFE230314C07CC02BF896
:10EC440084F3C53EAE3D11118F15BEC37EC511E6DA
:10EC5400D5E1713812363D221F2699CC8ACF33D69E
:10EC6400BFD2412DCD2976306733E1D9C3DDEEC95A
:10EC74008FC72B1EEF19823A423C71EAEFEE52C263
:10EC84003BC17C0CD507843FEC3FDDFC920105C001
:10EC94004FC0BBF90FF50E3F143E8C0F13143BC34A
:10ECA400E0C483E73AE32A39E536E720DA24ADCB3A
:10ECB40087CE67D7DFD35A2EFA2A6B2F7432A1D8A6
:10ECC40072DCCACA51C88B1F5D1BDA39B63BF8E83F
:10ECD4006CEDC2C28FC1050E64094E3FD33F4BFB9E
:10ECE400000000C02DC04BFB9CF64E3F713E050E4C
:10ECF4009412C2C24AC4F8E8A3E4DA39AF378B1FCE
:10ED04008E23CACA8CCDA1D806D56B2F212C5A2E9E
:10ED1400793167D726DBADCB1BC9E720C61C2A395E
:10ED2400203B83E7EDEB3BC3ECC18C0FF10A0E3FB4
:10ED3400B13FBBF96EFE05C014C0DDFC2BF8843F67
:10ED4400C53E7C0C111152C2BEC371EA11E6823A6F
:10ED540071382B1E3D22EEC999CCE1D933D67630D9
:10ED6400412D412D763033D6E1D999CCEEC93D22DF
:10ED74002B1E7138823A11E671EABEC352C21111D8
:10ED84007C0CC53E843F2BF8DDFC14C005C06EFE30
:10ED9400BBF9B13F0E3FF10A8C0FECC13BC3EDEB65
:10EDA40083E7203B2A39C61CE7201BC9ADCB26DBF1
:10EDB40067D779315A2E212C6B2F06D5A1D88CCD4B
:10EDC400CACA8E238B1FAF37DA39A3E4F8E84AC4E2
:10EDD400C2C29412050E713E4E3F9CF64BFB2DC0F1
:10EDE40000C000004BFBD33F4E3F6409050E8FC1AA
:10EDF400C2C26CEDF8E8B63BDA395D1B8B1F51C813
:10EE0400CACA72DCA1D874326B2FFA2A5A2EDFD305
:10EE140067D787CEADCBDA24E720E5362A393AE343
:10EE240083E7E0C43BC313148C0F143E0E3F0FF56D
:10EE3400BBF94FC005C09201DDFCEC3F843FD50710
:10EE44007C0C3BC152C2EFEE71EA423C823AEF19AC
:10EE54002B1E8FC7EEC9C3DDE1D967337630CD29C8
:10EE6400412DBFD233D68ACF99CC1F263D221236EC
:10EE74007138D5E111E67EC5BEC38F151111AE3DC3
:10EE8400C53E84F32BF87CC014C023036EFEFB3F05
:10EE9400B13F4506F10AF2C0ECC174F0EDEBC53C9C
:10EEA400203B7D18C61CD6C61BC919DF26DB53348C
:10EEB40079319928212CA6D106D595D08CCD5F2700
:10EEC4008E233635AF3775E0A3E426C64AC4081747
:10EED40094123E3D713EFBF19CF6B2C02DC0B504C8
:10EEE40000000040C53E7C0C7D18E0C4CACA72DC38
:10EEF400BFD2412D8E233635203B83E784F33BC1BB
:10EF040000C0000084F3C53E203B7D188E23CACA8E
:10EF1400BFD2BFD2CACA8E237D18203BC53E84F31C
:10EF2400000000C03BC184F383E7203B36358E23C9
:10EF3400412DBFD272DCCACAE0C47D187C0CC53E28
:10EF4400004000007C0C3BC1E0C483E772DC363532
:10EF5400412D412D363572DC83E7E0C43BC17C0C86
:10EF640000000040C53E7C0C7D18E0C4CACA72DCB7
:10EF7400BFD2412D8E233635203B83E784F33BC13A
:10EF840000C0000084F3C53E203B7D188E23CACA0E
:10EF9400BFD2BFD2CACA8E237D18203BC53E84F39C
:10EFA400000000C03BC184F383E7203B36358E2349
:10EFB400412DBFD272DCCACAE0C47D187C0CC53EA8
:10EFC400004000007C0C3BC1E0C483E772DC3635B2
:10EFD400412D412D363572DC83E7E0C43BC17C0C06
:10EFE40000000040C53E7C0C7D18E0C4CACA72DC37
:10EFF400BFD2412D8E233635203B83E784F33BC1BA
:10F0040000C0000084F3C53E203B7D188E23CACA8D
:10F01400BFD2BFD2CACA8E237D18203BC53E84F31B
:10F02400000000C03BC184F383E7203B36358E23C8
:10F03400412DBFD272DCCACAE0C47D187C0CC53E27
:10F04400004000007C0C3BC1E0C483E772DC363531
:10F05400412D412D363572DC83E7E0C43BC17C0C85
:10F0640000000040C53E7C0C7D18E0C4CACA72DCB6
:10F07400BFD2412D8E233635203B83E784F33BC139
:10F0840000C0000084F3C53E203B7D188E23CACA0D
:10F09400BFD2BFD2CACA8E237D18203BC53E84F39B
:10F0A400000000C03BC184F383E7203B36358E2348
:10F0B400412DBFD272DCCACAE0C47D187C0CC53EA7
:10F0C400004000007C0C3BC1E0C483E772DC3635B1
:10F0D400412D412D363572DC83E7E0C43BC17C0C05
:10F0E40000000040C53E7C0C7D18E0C4CACA72DC36
:10F0F400BFD2412D8E233635203B83E784F33BC1B9
:10F1040000C0000084F3C53E203B7D188E23CACA8C
:10F11400BFD2BFD2CACA8E237D18203BC53E84F31A
:10F12400000000C03BC184F383E7203B36358E23C7
:10F13400412DBFD272DCCACAE0C47D187C0CC53E26
:10F14400004000007C0C3BC1E0C483E772DC363530
:10F15400412D412D363572DC83E7E0C43BC17C0C84
:10F1640000000040C53E7C0C7D18E0C4CACA72DCB5
:10F17400BFD2412D8E233635203B83E784F33BC138
:10F1840000C0000084F3C53E203B7D188E23CACA0C
:10F19400BFD2BFD2CACA8E237D18203BC53E84F39A
:10F1A400000000C03BC184F383E7203B36358E2347
:10F1B400412DBFD272DCCACAE0C47D187C0CC53EA6
:10F1C400004000007C0C3BC1E0C483E772DC3635B0
:10F1D400412D412D363572DC83E7E0C43BC17C0C04
:10F1E40000000040C53E7C0C7D18E0C4CACA72DC35
:10F1F400BFD2412D8E233635203B83E784F33BC1B8
:10F2040000C0000084F3C53E203B7D188E23CACA8B
:10F21400BFD2BFD2CACA8E237D18203BC53E84F319
:10F22400000000C03BC184F383E7203B36358E23C6
:10F23400412DBFD272DCCACAE0C47D187C0CC53E25
:10F24400004000007C0C3BC1E0C483E772DC36352F
:10F25400412D412D363572DC83E7E0C43BC17C0C83
:10F2640000000040C53E7C0C7D18E0C4CACA72DCB4
:10F27400BFD2412D8E233635203B83E784F33BC137
:10F2840000C0000084F3C53E203B7D188E23CACA0B
:10F29400BFD2BFD2CACA8E237D18203BC53E84F399
:10F2A400000000C03BC184F383E7203B36358E2346
:10F2B400412DBFD272DCCACAE0C47D187C0CC53EA5
:10F2C400004000007C0C3BC1E0C483E772DC3635AF
:10F2D400412D412D363572DC83E7E0C43BC17C0C03
:10F2E40000000040C53E7C0C7D18E0C4CACA72DC34
:10F2F400BFD2412D8E233635203B83E784F33BC1B7
:10F3040000C0000084F3C53E203B7D188E23CACA8A
:10F31400BFD2BFD2CACA8E237D18203BC53E84F318
:10F32400000000C03BC184F383E7203B36358E23C5
:10F33400412DBFD272DCCACAE0C47D187C0CC53E24
:10F34400004000007C0C3BC1E0C483E772DC36352E
:10F35400412D412D363572DC83E7E0C43BC17C0C82
:10F3640000000040C53E7C0C7D18E0C4CACA72DCB3
:10F37400BFD2412D8E233635203B83E784F33BC136
:10F3840000C0000084F3C53E203B7D188E23CACA0A
:10F39400BFD2BFD2CACA8E237D18203BC53E84F398
:10F3A400000000C03BC184F383E7203B36358E2345
:10F3B400412DBFD272DCCACAE0C47D187C0CC53EA4
:10F3C400004000007C0C3BC1E0C483E772DC3635AE
:10F3D400412D412D363572DC83E7E0C43BC17C0C02
:10F3E40000000040C53E7C0C7D18E0C4CACA72DC33
:10F3F400BFD2412D8E233635203B83E784F33BC1B6
:10F4040000C0000084F3C53E203B7D188E23CACA89
:10F41400BFD2BFD2CACA8E237D18203BC53E84F317
:10F42400000000C03BC184F383E7203B36358E23C4
:10F43400412DBFD272DCCACAE0C47D187C0CC53E23
:10F44400004000007C0C3BC1E0C483E772DC36352D
:10F45400412D412D363572DC83E7E0C43BC17C0C81
:10F4640000000040C53E7C0C7D18E0C4CACA72DCB2
:10F47400BFD2412D8E233635203B83E784F33BC135
:10F4840000C0000084F3C53E203B7D188E23CACA09
:10F49400BFD2BFD2CACA8E237D18203BC53E84F397
:10F4A400000000C03BC184F383E7203B36358E2344
:10F4B400412DBFD272DCCACAE0C47D187C0CC53EA3
:10F4C400004000007C0C3BC1E0C483E772DC3635AD
:10F4D400412D412D363572DC83E7E0C43BC17C0C01
:10F4E40000000040C53E7C0C7D18E0C4CACA72DC32
:10F4F400BFD2412D8E233635203B83E784F33BC1B5
:10F5040000C0000084F3C53E203B7D188E23CACA88
:10F51400BFD2BFD2CACA8E237D18203BC53E84F316
:10F52400000000C03BC184F383E7203B36358E23C3
:10F53400412DBFD272DCCACAE0C47D187C0CC53E22
:10F54400004000007C0C3BC1E0C483E772DC36352C
:10F55400412D412D363572DC83E7E0C43BC17C0C80
:10F5640000000040C53E7C0C7D18E0C4CACA72DCB1
:10F57400BFD2412D8E233635203B83E784F33BC134
:10F5840000C0000084F3C53E203B7D188E23CACA08
:10F59400BFD2BFD2CACA8E237D18203BC53E84F396
:10F5A400000000C03BC184F383E7203B36358E2343
:10F5B400412DBFD272DCCACAE0C47D187C0CC53EA2
:10F5C400004000007C0C3BC1E0C483E772DC3635AC
:10F5D400412D412D363572DC83E7E0C43BC17C0C00
:10F5E40000000040C53E7C0C7D18E0C4CACA72DC31
:10F5F400BFD2412D8E233635203B83E784F33BC1B4
:10F6040000C0000084F3C53E203B7D188E23CACA87
:10F61400BFD2BFD2CACA8E237D18203BC53E84F315
:10F62400000000C03BC184F383E7203B36358E23C2
:10F63400412DBFD272DCCACAE0C47D187C0CC53E21
:10F64400004000007C0C3BC1E0C483E772DC36352B
:10F65400412D412D363572DC83E7E0C43BC17C0C7F
:10F6640000000040C53E7C0C7D18E0C4CACA72DCB0
:10F67400BFD2412D8E233635203B83E784F33BC133
:10F6840000C0000084F3C53E203B7D188E23CACA07
:10F69400BFD2BFD2CACA8E237D18203BC53E84F395
:10F6A400000000C03BC184F383E7203B36358E2342
:10F6B400412DBFD272DCCACAE0C47D187C0CC53EA1
:10F6C400004000007C0C3BC1E0C483E772DC3635AB
:10F6D400412D412D363572DC83E7E0C43BC17C0CFF
:10F6E4000000004067331F263E3D6CED8F15BEC3FE
:10F6F40072DCCACA14C0DDFC67D779318C0F143EA2
:10F70400203B7D18E53619DF45064FC095D006D558
:10F714003BC17C0CA3E4DA392B1E71384E3F6409DB
:10F72400412DBFD29CF6B2C08FC7D5E126C65D1B62
:10F7340084F3C53EFA2A6B2FB13FBBF9E7201BC9FE
:10F7440083E7E0C4ECC174F087CE99282303EC3F2F
:10F7540036358E23423C71EA9412C2C2E1D999CC67
:10F7640000C00000E1D9673394123E3D423C8F153E
:10F77400363572DC230314C087CE67D7ECC18C0FF7
:10F7840083E7203BE720E536B13F4506FA2A95D0CA
:10F7940084F33BC126C6A3E48FC72B1E9CF64E3FC1
:10F7A400412D412D4E3F9CF62B1E8FC7A3E426C648
:10F7B4003BC184F395D0FA2A4506B13FE536E720EC
:10F7C400203B83E78C0FECC167D787CE14C023039B
:10F7D40072DC36358F15423C3E3D94126733E1D9D5
:10F7E400000000C099CCE1D9C2C2941271EA423C33
:10F7F4008E233635EC3F2303992887CE74F0ECC171
:10F80400E0C483E71BC9E720BBF9B13F6B2FFA2A99
:10F81400C53E84F35D1B26C6D5E18FC7B2C09CF6F6
:10F82400BFD2412D64094E3F71382B1EDA39A3E44F
:10F834007C0C3BC106D595D04FC0450619DFE53693
:10F844007D18203B143E8C0F793167D7DDFC14C042
:10F85400CACA72DCBEC38F156CED3E3D1F266733EA
:10F86400004000001F2699CC6CEDC2C2BEC371EAF1
:10F87400CACA8E23DDFCEC3F79319928143E74F01A
:10F884007D18E0C419DF1BC94FC0BBF906D56B2F27
:10F894007C0CC53EDA395D1B7138D5E16409B2C010
:10F8A400BFD2BFD2B2C06409D5E171385D1BDA3969
:10F8B400C53E7C0C6B2F06D5BBF94FC01BC919DFA5
:10F8C400E0C47D1874F0143E99287931EC3FDDFCD6
:10F8D4008E23CACA71EABEC3C2C26CED99CC1F267C
:10F8E4000000004067331F263E3D6CED8F15BEC3FC
:10F8F40072DCCACA14C0DDFC67D779318C0F143EA0
:10F90400203B7D18E53619DF45064FC095D006D556
:10F914003BC17C0CA3E4DA392B1E71384E3F6409D9
:10F92400412DBFD29CF6B2C08FC7D5E126C65D1B60
:10F9340084F3C53EFA2A6B2FB13FBBF9E7201BC9FC
:10F9440083E7E0C4ECC174F087CE99282303EC3F2D
:10F9540036358E23423C71EA9412C2C2E1D999CC65
:10F9640000C00000E1D9673394123E3D423C8F153C
:10F97400363572DC230314C087CE67D7ECC18C0FF5
:10F9840083E7203BE720E536B13F4506FA2A95D0C8
:10F9940084F33BC126C6A3E48FC72B1E9CF64E3FBF
:10F9A400412D412D4E3F9CF62B1E8FC7A3E426C646
:10F9B4003BC184F395D0FA2A4506B13FE536E720EA
:10F9C400203B83E78C0FECC167D787CE14C0230399
:10F9D40072DC36358F15423C3E3D94126733E1D9D3
:10F9E400000000C099CCE1D9C2C2941271EA423C31
:10F9F4008E233635EC3F2303992887CE74F0ECC16F
:10FA0400E0C483E71BC9E720BBF9B13F6B2FFA2A97
:10FA1400C53E84F35D1B26C6D5E18FC7B2C09CF6F4
:10FA2400BFD2412D64094E3F71382B1EDA39A3E44D
:10FA34007C0C3BC106D595D04FC0450619DFE53691
:10FA44007D18203B143E8C0F793167D7DDFC14C040
:10FA5400CACA72DCBEC38F156CED3E3D1F266733E8
:10FA6400004000001F2699CC6CEDC2C2BEC371EAEF
:10FA7400CACA8E23DDFCEC3F79319928143E74F018
:10FA84007D18E0C419DF1BC94FC0BBF906D56B2F25
:10FA94007C0CC53EDA395D1B7138D5E16409B2C00E
:10FAA400BFD2BFD2B2C06409D5E171385D1BDA3967
:10FAB400C53E7C0C6B2F06D5BBF94FC01BC919DFA3
:10FAC400E0C47D1874F0143E99287931EC3FDDFCD4
:10FAD4008E23CACA71EABEC3C2C26CED99CC1F267A
:10FAE4000000004067331F263E3D6CED8F15BEC3FA
:10FAF40072DCCACA14C0DDFC67D779318C0F143E9E
:10FB0400203B7D18E53619DF45064FC095D006D554
:10FB14003BC17C0CA3E4DA392B1E71384E3F6409D7
:10FB2400412DBFD29CF6B2C08FC7D5E126C65D1B5E
:10FB340084F3C53EFA2A6B2FB13FBBF9E7201BC9FA
:10FB440083E7E0C4ECC174F087CE99282303EC3F2B
:10FB540036358E23423C71EA9412C2C2E1D999CC63
:10FB640000C00000E1D9673394123E3D423C8F153A
:10FB7400363572DC230314C087CE67D7ECC18C0FF3
:10FB840083E7203BE720E536B13F4506FA2A95D0C6
:10FB940084F33BC126C6A3E48FC72B1E9CF64E3FBD
:10FBA400412D412D4E3F9CF62B1E8FC7A3E426C644
:10FBB4003BC184F395D0FA2A4506B13FE536E720E8
:10FBC400203B83E78C0FECC167D787CE14C0230397
:10FBD40072DC36358F15423C3E3D94126733E1D9D1
:10FBE400000000C099CCE1D9C2C2941271EA423C2F
:10FBF4008E233635EC3F2303992887CE74F0ECC16D
:10FC0400E0C483E71BC9E720BBF9B13F6B2FFA2A95
:10FC1400C53E84F35D1B26C6D5E18FC7B2C09CF6F2
:10FC2400BFD2412D64094E3F71382B1EDA39A3E44B
:10FC34007C0C3BC106D595D04FC0450619DFE5368F
:10FC44007D18203B143E8C0F793167D7DDFC14C03E
:10FC5400CACA72DCBEC38F156CED3E3D1F266733E6
:10FC6400004000001F2699CC6CEDC2C2BEC371EAED
:10FC7400CACA8E23DDFCEC3F79319928143E74F016
:10FC84007D18E0C419DF1BC94FC0BBF906D56B2F23
:10FC94007C0CC53EDA395D1B7138D5E16409B2C00C
:10FCA400BFD2BFD2B2C06409D5E171385D1BDA3965
:10FCB400C53E7C0C6B2F06D5BBF94FC01BC919DFA1
:10FCC400E0C47D1874F0143E99287931EC3FDDFCD2
:10FCD4008E23CACA71EABEC3C2C26CED99CC1F2678
:10FCE4000000004067331F263E3D6CED8F15BEC3F8
:10FCF40072DCCACA14C0DDFC67D779318C0F143E9C
:10FD0400203B7D18E53619DF45064FC095D006D552
:10FD14003BC17C0CA3E4DA392B1E71384E3F6409D5
:10FD2400412DBFD29CF6B2C08FC7D5E126C65D1B5C
:10FD340084F3C53EFA2A6B2FB13FBBF9E7201BC9F8
:10FD440083E7E0C4ECC174F087CE99282303EC3F29
:10FD540036358E23423C71EA9412C2C2E1D999CC61
:10FD640000C00000E1D9673394123E3D423C8F1538
:10FD7400363572DC230314C087CE67D7ECC18C0FF1
:10FD840083E7203BE720E536B13F4506FA2A95D0C4
:10FD940084F33BC126C6A3E48FC72B1E9CF64E3FBB
:10FDA400412D412D4E3F9CF62B1E8FC7A3E426C642
:10FDB4003BC184F395D0FA2A4506B13FE536E720E6
:10FDC400203B83E78C0FECC167D787CE14C0230395
:10FDD40072DC36358F15423C3E3D94126733E1D9CF
:10FDE400000000C099CCE1D9C2C2941271EA423C2D
:10FDF4008E233635EC3F2303992887CE74F0ECC16B
:10FE0400E0C483E71BC9E720BBF9B13F6B2FFA2A93
:10FE1400C53E84F35D1B26C6D5E18FC7B2C09CF6F0
:10FE2400BFD2412D64094E3F71382B1EDA39A3E449
:10FE34007C0C3BC106D595D04FC0450619DFE5368D
:10FE44007D18203B143E8C0F793167D7DDFC14C03C
:10FE5400CACA72DCBEC38F156CED3E3D1F266733E4
:10FE6400004000001F2699CC6CEDC2C2BEC371EAEB
:10FE7400CACA8E23DDFCEC3F79319928143E74F014
:10FE84007D18E0C419DF1BC94FC0BBF906D56B2F21
:10FE94007C0CC53EDA395D1B7138D5E16409B2C00A
:10FEA400BFD2BFD2B2C06409D5E171385D1BDA3963
:10FEB400C53E7C0C6B2F06D5BBF94FC01BC919DF9F
:10FEC400E0C47D1874F0143E99287931EC3FDDFCD0
:10FED4008E23CACA71EABEC3C2C26CED99CC1F2676
:10FEE4000000004074325F27143E74F0EF197EC5A1
:10FEF400D5E18FC7F2C00FF595D0FA2AB504D33FE8
:10FF040036358E23C53CEDEB8F15BEC3C3DDEEC97C
:10FF14004FC0BBF9DFD35A2E64094E3FAF378B1F56
:10FF2400203B83E7111152C2E1D999CC05C06EFE82
:10FF340067D77931050E713EDA395D1B2A393AE308
:10FF44007C0C3BC133D68ACF14C0230326DB533445
:10FF540094123E3DB63B0817E53619DFD5077CC041
:10FF6400BFD2BFD27CC0D50719DFE5360817B63B30
:10FF74003E3D9412533426DB230314C08ACF33D678
:10FF84003BC17C0C3AE32A395D1BDA39713E050E1C
:10FF9400793167D76EFE05C099CCE1D952C21111EF
:10FFA40083E7203B8B1FAF374E3F64095A2EDFD3C4
:10FFB400BBF94FC0EEC9C3DDBEC38F15EDEBC53C25
:10FFC4008E233635D33FB504FA2A95D00FF5F2C007
:10FFD4008FC7D5E17EC5EF1974F0143E5F277432E4
:10FFE400004000005F278CCD74F0ECC17EC511E6A3
:0CFFF4008FC72B1E0FF50E3FFA2A6B2F53
:020000040801F1
:10000000D33F4BFB8E23CACAEDEB3BC3BEC371EAA1
:10001000EEC93D22BBF9B13F5A2E212C4E3F9CF632
:100020008B1F51C883E7E0C452C2EFEE99CC1F2664
:100030006EFEFB3F79319928713EFBF15D1B26C6B0
:100040003AE3D6C63BC184F38ACFCD292303EC3FE4
:100050005334DA243E3D6CED08174AC419DF1BC93E
:100060007CC02BF8BFD2412DD507843FE536E72071
:10007000B63BF8E89412C2C226DBADCB14C0DDFC5F
:1000800033D676307C0CC53E2A39C61CDA39A3E457
:10009000050E8FC167D787CE05C09201E1D96733BE
:1000A0001111AE3D203B7D18AF3775E06409B2C039
:1000B000DFD3A6D14FC04506C3DD12368F15423CB3
:1000C000C53C1314363572DCB5042DC095D006D569
:1000D000F2C0F10AD5E17138EF19823A143E8C0F63
:1000E0007432A1D8000000C08CCDA1D8ECC18C0F17
:1000F00011E6823A2B1E71380E3FF10A6B2F06D59E
:100100004BFB2DC0CACA72DC3BC3131471EA423CDC
:100110003D221236B13F4506212CA6D19CF6B2C035
:1001200051C875E0E0C47D18EFEEAE3D1F26673381
:10013000FB3F9201992887CEFBF18FC126C6A3E42D
:10014000D6C6C61C84F3C53ECD297630EC3FDDFC17
:10015000DA24ADCB6CEDC2C24AC4F8E81BC9E72073
:100160002BF8843F412D412D843F2BF8E7201BC9FC
:10017000F8E84AC4C2C26CEDADCBDA24DDFCEC3F3A
:100180007630CD29C53E84F3C61CD6C6A3E426C668
:100190008FC1FBF187CE99289201FB3F67331F2661
:1001A000AE3DEFEE7D18E0C475E051C8B2C09CF6DC
:1001B000A6D1212C4506B13F12363D22423C71EAC0
:1001C00013143BC372DCCACA2DC04BFB06D56B2F80
:1001D000F10A0E3F71382B1E823A11E68C0FECC1EA
:1001E000A1D88CCD00C00000A1D874328C0F143E71
:1001F000823AEF197138D5E1F10AF2C006D595D0EF
:100200002DC0B50472DC36351314C53C423C8F1545
:100210001236C3DD45064FC0A6D1DFD3B2C0640994
:1002200075E0AF377D18203BAE3D11116733E1D942
:10023000920105C087CE67D78FC1050EA3E4DA39D6
:10024000C61C2A39C53E7C0C763033D6DDFC14C082
:10025000ADCB26DBC2C29412F8E8B63BE720E53608
:10026000843FD507412DBFD22BF87CC01BC919DFB5
:100270004AC408176CED3E3DDA245334EC3F2303A7
:10028000CD298ACF84F33BC1D6C63AE326C65D1B8F
:10029000FBF1713E99287931FB3F6EFE1F2699CC08
:1002A000EFEE52C2E0C483E751C88B1F9CF64E3F6D
:1002B000212C5A2EB13FBBF93D22EEC971EABEC3D3
:1002C0003BC3EDEBCACA8E234BFBD33F6B2FFA2AFD
:1002D0000E3F0FF52B1E8FC711E67EC5ECC174F0E3
:1002E0008CCD5F270000004074325F27143E74F00D
:1002F000EF197EC5D5E18FC7F2C00FF595D0FA2A68
:10030000B504D33F36358E23C53CEDEB8F15BEC308
:10031000C3DDEEC94FC0BBF9DFD35A2E64094E3F8F
:10032000AF378B1F203B83E7111152C2E1D999CC23
:1003300005C06EFE67D77931050E713EDA395D1B57
:100340002A393AE37C0C3BC133D68ACF14C023034D
:1003500026DB533494123E3DB63B0817E53619DFD1
:10036000D5077CC0BFD2BFD27CC0D50719DFE53628
:100370000817B63B3E3D9412533426DB230314C0CA
:100380008ACF33D63BC17C0C3AE32A395D1BDA397C
:10039000713E050E793167D76EFE05C099CCE1D963
:1003A00052C2111183E7203B8B1FAF374E3F6409C8
:1003B0005A2EDFD3BBF94FC0EEC9C3DDBEC38F15C4
:1003C000EDEBC53C8E233635D33FB504FA2A95D0E4
:1003D0000FF5F2C08FC7D5E17EC5EF1974F0143E5A
:1003E0005F277432004000005F278CCD74F0ECC1B1
:1003F0007EC511E68FC72B1E0FF50E3FFA2A6B2F15
:10040000D33F4BFB8E23CACAEDEB3BC3BEC371EA9D
:10041000EEC93D22BBF9B13F5A2E212C4E3F9CF62E
:100420008B1F51C883E7E0C452C2EFEE99CC1F2660
:100430006EFEFB3F79319928713EFBF15D1B26C6AC
:100440003AE3D6C63BC184F38ACFCD292303EC3FE0
:100450005334DA243E3D6CED08174AC419DF1BC93A
:100460007CC02BF8BFD2412DD507843FE536E7206D
:10047000B63BF8E89412C2C226DBADCB14C0DDFC5B
:1004800033D676307C0CC53E2A39C61CDA39A3E453
:10049000050E8FC167D787CE05C09201E1D96733BA
:1004A0001111AE3D203B7D18AF3775E06409B2C035
:1004B000DFD3A6D14FC04506C3DD12368F15423CAF
:1004C000C53C1314363572DCB5042DC095D006D565
:1004D000F2C0F10AD5E17138EF19823A143E8C0F5F
:1004E0007432A1D8000000C08CCDA1D8ECC18C0F13
:1004F00011E6823A2B1E71380E3FF10A6B2F06D59A
:100500004BFB2DC0CACA72DC3BC3131471EA423CD8
:100510003D221236B13F4506212CA6D19CF6B2C031
:1005200051C875E0E0C47D18EFEEAE3D1F2667337D
:10053000FB3F9201992887CEFBF18FC126C6A3E429
:10054000D6C6C61C84F3C53ECD297630EC3FDDFC13
:10055000DA24ADCB6CEDC2C24AC4F8E81BC9E7206F
:100560002BF8843F412D412D843F2BF8E7201BC9F8
:10057000F8E84AC4C2C26CEDADCBDA24DDFCEC3F36
:100580007630CD29C53E84F3C61CD6C6A3E426C664
:100590008FC1FBF187CE99289201FB3F67331F265D
:1005A000AE3DEFEE7D18E0C475E051C8B2C09CF6D8
:1005B000A6D1212C4506B13F12363D22423C71EABC
:1005C00013143BC372DCCACA2DC04BFB06D56B2F7C
:1005D000F10A0E3F71382B1E823A11E68C0FECC1E6
:1005E000A1D88CCD00C00000A1D874328C0F143E6D
:1005F000823AEF197138D5E1F10AF2C006D595D0EB
:100600002DC0B50472DC36351314C53C423C8F1541
:100610001236C3DD45064FC0A6D1DFD3B2C0640990
:1006200075E0AF377D18203BAE3D11116733E1D93E
:10063000920105C087CE67D78FC1050EA3E4DA39D2
:10064000C61C2A39C53E7C0C763033D6DDFC14C07E
:10065000ADCB26DBC2C29412F8E8B63BE720E53604
:10066000843FD507412DBFD22BF87CC01BC919DFB1
:100670004AC408176CED3E3DDA245334EC3F2303A3
:10068000CD298ACF84F33BC1D6C63AE326C65D1B8B
:10069000FBF1713E99287931FB3F6EFE1F2699CC04
:1006A000EFEE52C2E0C483E751C88B1F9CF64E3F69
:1006B000212C5A2EB13FBBF93D22EEC971EABEC3CF
:1006C0003BC3EDEBCACA8E234BFBD33F6B2FFA2AF9
:1006D0000E3F0FF52B1E8FC711E67EC5ECC174F0DF
:1006E0008CCD5F2700030102010301000203020019
:1006F0000100020100020100020100021CF90208CF
:10070000E4B600081CF102081CE90208E4C600086F
:10071000E4FE0008E4F600081CE102081CD9020807
:10072000E4CE00081CD102081CC902081CC1020842
:100730001CB90208E4BE00081CB102081CA902088A
:100740001CA102081C990208E4DE00081C910208A2
:100750001C8902081C8102081C790208E4EE0008CA
:100760001C7102081C6902081C6102081C5902085D
:10077000E4E600081C5102081C490208E4D60008FF
:100780001C4102081C3902081C3102081C290208FD
:100790001C2102081C1902081C1102081C0902086D
:1007A0001C0102081CF901081CF101081CE90108E0
:1007B0001CE101081CD901081CD101081CC9010851
:1007C0000205070A0C0F111416191B1E0306080B4D
:1007D0000D101215171A1C1F0097B92EE5725CCB6D
:1007E0005DCAE473B82F0196BA2D03945FC8E67111
:1007F000E7705EC90295BB2CE3745ACD0691BF2801
:10080000BE2907905BCCE27559CEE077BC2B0592F0
:100810000493BD2AE17658CF51C6E87FB4230D9AE0
:100820000C9BB522E97E50C7EB7C52C50E99B720D0
:10083000B6210F9853C4EA7DB2250B9C57C0EE79C0
:10084000EF7856C10A9DB324089FB126ED7A54C3B0
:1008500055C2EC7BB027099EA2351B8C47D0FE69A0
:10086000FF6846D11A8DA334188FA136FD6A44D390
:1008700045D2FC6BA037198E41D6F86FA4331D8A80
:100880001C8BA532F96E40D7FB6C42D51E89A73070
:10089000A6311F8843D4FA6DF3644ADD1681AF3860
:1008A000AE3917804BDCF26549DEF067AC3B158250
:1008B0001483AD3AF16648DF1087A93EF5624CDB40
:1008C0004DDAF463A83F1186AA3D13844FD8F66130
:1008D000F7604ED91285AB3C00000040000000C01C
:1008E00000000040000000C000000040000000C008
:1008F00000000040000000C000000040000000C0F8
:1009000000000040000000C000000040000000C0E7
:1009100000000040000000C000000040000000C0D7
:1009200000000040000000C000000040000000C0C7
:1009300000000040000000C000000040000000C0B7
:1009400000000040000000C000000040000000C0A7
:1009500000000040000000C000000040000000C097
:1009600000000040000000C000000040000000C087
:1009700000000040000000C000000040000000C077
:1009800000000040000000C000000040000000C067
:1009900000000040000000C000000040000000C057
:1009A00000000040000000C000000040000000C047
:1009B00000000040000000C000000040000000C037
:1009C00000000040000000C000000040000000C027
:1009D00000000040000000C000000040000000C017
:1009E00000000040000000C000000040000000C007
:1009F00000000040000000C000000040000000C0F7
:100A000000000040000000C000000040000000C0E6
:100A100000000040000000C000000040000000C0D6
:100A200000000040000000C000000040000000C0C6
:100A300000000040000000C000000040000000C0B6
:100A400000000040000000C000000040000000C0A6
:100A500000000040000000C000000040000000C096
:100A600000000040000000C000000040000000C086
:100A700000000040000000C000000040000000C076
:100A800000000040000000C000000040000000C066
:100A900000000040000000C000000040000000C056
:100AA00000000040000000C000000040000000C046
:100AB00000000040000000C000000040000000C036
:100AC00000000040000000C000000040000000C026
:100AD00000000040000000C000000040000000C016
:100AE00000000040000000C000000040000000C006
:100AF00000000040000000C000000040000000C0F6
:100B000000000040000000C000000040000000C0E5
:100B100000000040000000C000000040000000C0D5
:100B200000000040000000C000000040000000C0C5
:100B300000000040000000C000000040000000C0B5
:100B400000000040000000C000000040000000C0A5
:100B500000000040000000C000000040000000C095
:100B600000000040000000C000000040000000C085
:100B700000000040000000C000000040000000C075
:100B800000000040000000C000000040000000C065
:100B900000000040000000C000000040000000C055
:100BA00000000040000000C000000040000000C045
:100BB00000000040000000C000000040000000C035
:100BC00000000040000000C000000040000000C025
:100BD00000000040000000C000000040000000C015
:100BE00000000040000000C000000040000000C005
:100BF00000000040000000C000000040000000C0F5
:100C000000000040000000C000000040000000C0E4
:100C100000000040000000C000000040000000C0D4
:100C200000000040000000C000000040000000C0C4
:100C300000000040000000C000000040000000C0B4
:100C400000000040000000C000000040000000C0A4
:100C500000000040000000C000000040000000C094
:100C600000000040000000C000000040000000C084
:100C700000000040000000C000000040000000C074
:100C800000000040000000C000000040000000C064
:100C900000000040000000C000000040000000C054
:100CA00000000040000000C000000040000000C044
:100CB00000000040000000C000000040000000C034
:100CC00000000040000000C000000040000000C024
:100CD00000000040000000C000005A2EEC3FCD296B
:100CE000BBF98CCDB2C026DB7C0C1236143E8B1FB8
:100CF0006CEDD6C6BEC311E67D18B63BDA391314C7
:100D0000D5E152C21BC9FBF18E230E3F6733D507D5
:100D100067D72DC095D06EFE412DFB3FFA2A4BFBC5
:100D200087CE7CC0E1D9F10A3635713EE720EFEE7F
:100D30008FC73BC3A3E40817203B823A8F153AE3E1
:100D4000C2C251C874F03D22C53E53346409A1D8D3
:100D50004FC08ACFDDFC212C0040212CDDFC8ACF46
:100D60004FC0A1D864095334C53E3D2274F051C828
:100D7000C2C23AE38F15823A203B0817A3E43BC373
:100D80008FC7EFEEE720713E3635F10AE1D97CC01E
:100D900087CE4BFBFA2AFB3F412D6EFE95D02DC02E
:100DA00067D7D50767330E3F8E23FBF11BC952C2AD
:100DB000D5E11314DA39B63B7D1811E6BEC3D6C6A9
:100DC0006CED8B1F143E12367C0C26DBB2C08CCD32
:100DD000BBF9CD29EC3F5A2E0000A6D114C033D662
:100DE000450674324E3FDA2484F3EEC9ECC175E057
:100DF00094122A39423CEF1983E74AC426C6EDEB28
:100E00002B1EAE3DE536050E72DCF2C099CC2BF8F8
:100E10009928D33F6B2F9201BFD205C006D5B504E8
:100E20007931843F1F260FF5CACA8FC119DF11110E
:100E30007138C53C5D1BF8E8E0C47EC571EAC61C8C
:100E40003E3DAF378C0FC3DD3BC1ADCB9CF65F277A
:100E5000B13F76302303DFD300C0DFD323037630E6
:100E6000B13F5F279CF6ADCB3BC1C3DD8C0FAF37E5
:100E70003E3DC61C71EA7EC5E0C4F8E85D1BC53C7A
:100E80007138111119DF8FC1CACA0FF51F26843FAF
:100E90007931B50406D505C0BFD292016B2FD33F7F
:100EA00099282BF899CCF2C072DC050EE536AE3DE0
:100EB0002B1EEDEB26C64AC483E7EF19423C2A39C4
:100EC000941275E0ECC1EEC984F3DA244E3F74321B
:100ED000450633D614C0A6D100005A2EEC3FCD29CA
:100EE000BBF98CCDB2C026DB7C0C1236143E8B1FB6
:100EF0006CEDD6C6BEC311E67D18B63BDA391314C5
:100F0000D5E152C21BC9FBF18E230E3F6733D507D3
:100F100067D72DC095D06EFE412DFB3FFA2A4BFBC3
:100F200087CE7CC0E1D9F10A3635713EE720EFEE7D
:100F30008FC73BC3A3E40817203B823A8F153AE3DF
:100F4000C2C251C874F03D22C53E53346409A1D8D1
:100F50004FC08ACFDDFC212C0040212CDDFC8ACF44
:100F60004FC0A1D864095334C53E3D2274F051C826
:100F7000C2C23AE38F15823A203B0817A3E43BC371
:100F80008FC7EFEEE720713E3635F10AE1D97CC01C
:100F900087CE4BFBFA2AFB3F412D6EFE95D02DC02C
:100FA00067D7D50767330E3F8E23FBF11BC952C2AB
:100FB000D5E11314DA39B63B7D1811E6BEC3D6C6A7
:100FC0006CED8B1F143E12367C0C26DBB2C08CCD30
:100FD000BBF9CD29EC3F5A2E0000A6D114C033D660
:100FE000450674324E3FDA2484F3EEC9ECC175E055
:100FF00094122A39423CEF1983E74AC426C6EDEB26
:101000002B1EAE3DE536050E72DCF2C099CC2BF8F6
:101010009928D33F6B2F9201BFD205C006D5B504E6
:101020007931843F1F260FF5CACA8FC119DF11110C
:101030007138C53C5D1BF8E8E0C47EC571EAC61C8A
:101040003E3DAF378C0FC3DD3BC1ADCB9CF65F2778
:10105000B13F76302303DFD300C0DFD323037630E4
:10106000B13F5F279CF6ADCB3BC1C3DD8C0FAF37E3
:101070003E3DC61C71EA7EC5E0C4F8E85D1BC53C78
:101080007138111119DF8FC1CACA0FF51F26843FAD
:101090007931B50406D505C0BFD292016B2FD33F7D
:1010A00099282BF899CCF2C072DC050EE536AE3DDE
:1010B0002B1EEDEB26C64AC483E7EF19423C2A39C2
:1010C000941275E0ECC1EEC984F3DA244E3F743219
:1010D000450633D614C0A6D10000DA39793174F050
:1010E0003BC1E1D92B1EEC3F7D1806D5C2C29CF650
:1010F0003635E536BBF9BEC3BFD28F15B13FE72009
:1011000072DCB2C06CED6B2F203B23038FC799CCF0
:101110007C0C143E9928A3E400C0A3E49928143E53
:101120007C0C99CC8FC72303203B6B2F6CEDB2C096
:1011300072DCE720B13F8F15BFD2BEC3BBF9E536E5
:1011400036359CF6C2C206D57D18EC3F2B1EE1D980
:101150003BC174F07931DA39000026C687CE8C0F96
:10116000C53E1F26D5E114C083E7FA2A3E3D640937
:10117000CACA1BC94506423C412D71EA4FC019DF5E
:101180008E234E3F941295D0E0C4DDFC7138673356
:1011900084F3ECC167D75D1B00405D1B67D7ECC1D2
:1011A00084F367337138DDFCE0C495D094124E3F70
:1011B0008E2319DF4FC071EA412D423C45061BC901
:1011C000CACA64093E3DFA2A83E714C0D5E11F2646
:1011D000C53E8C0F87CE26C60000DA39793174F00F
:1011E0003BC1E1D92B1EEC3F7D1806D5C2C29CF64F
:1011F0003635E536BBF9BEC3BFD28F15B13FE72008
:1012000072DCB2C06CED6B2F203B23038FC799CCEF
:101210007C0C143E9928A3E400C0A3E49928143E52
:101220007C0C99CC8FC72303203B6B2F6CEDB2C095
:1012300072DCE720B13F8F15BFD2BEC3BBF9E536E4
:1012400036359CF6C2C206D57D18EC3F2B1EE1D97F
:101250003BC174F07931DA39000026C687CE8C0F95
:10126000C53E1F26D5E114C083E7FA2A3E3D640936
:10127000CACA1BC94506423C412D71EA4FC019DF5D
:101280008E234E3F941295D0E0C4DDFC7138673355
:1012900084F3ECC167D75D1B00405D1B67D7ECC1D1
:1012A00084F367337138DDFCE0C495D094124E3F6F
:1012B0008E2319DF4FC071EA412D423C45061BC900
:1012C000CACA64093E3DFA2A83E714C0D5E11F2645
:1012D000C53E8C0F87CE26C60000DA39793174F00E
:1012E0003BC1E1D92B1EEC3F7D1806D5C2C29CF64E
:1012F0003635E536BBF9BEC3BFD28F15B13FE72007
:1013000072DCB2C06CED6B2F203B23038FC799CCEE
:101310007C0C143E9928A3E400C0A3E49928143E51
:101320007C0C99CC8FC72303203B6B2F6CEDB2C094
:1013300072DCE720B13F8F15BFD2BEC3BBF9E536E3
:1013400036359CF6C2C206D57D18EC3F2B1EE1D97E
:101350003BC174F07931DA39000026C687CE8C0F94
:10136000C53E1F26D5E114C083E7FA2A3E3D640935
:10137000CACA1BC94506423C412D71EA4FC019DF5C
:101380008E234E3F941295D0E0C4DDFC7138673354
:1013900084F3ECC167D75D1B00405D1B67D7ECC1D0
:1013A00084F367337138DDFCE0C495D094124E3F6E
:1013B0008E2319DF4FC071EA412D423C45061BC9FF
:1013C000CACA64093E3DFA2A83E714C0D5E11F2644
:1013D000C53E8C0F87CE26C60000DA39793174F00D
:1013E0003BC1E1D92B1EEC3F7D1806D5C2C29CF64D
:1013F0003635E536BBF9BEC3BFD28F15B13FE72006
:1014000072DCB2C06CED6B2F203B23038FC799CCED
:101410007C0C143E9928A3E400C0A3E49928143E50
:101420007C0C99CC8FC72303203B6B2F6CEDB2C093
:1014300072DCE720B13F8F15BFD2BEC3BBF9E536E2
:1014400036359CF6C2C206D57D18EC3F2B1EE1D97D
:101450003BC174F07931DA39000026C687CE8C0F93
:10146000C53E1F26D5E114C083E7FA2A3E3D640934
:10147000CACA1BC94506423C412D71EA4FC019DF5B
:101480008E234E3F941295D0E0C4DDFC7138673353
:1014900084F3ECC167D75D1B00405D1B67D7ECC1CF
:1014A00084F367337138DDFCE0C495D094124E3F6D
:1014B0008E2319DF4FC071EA412D423C45061BC9FE
:1014C000CACA64093E3DFA2A83E714C0D5E11F2643
:1014D000C53E8C0F87CE26C60000C53C1F2626DBE6
:1014E000C2C26EFE423C5F2772DC52C2DDFCB63BDC
:1014F0009928C3DDECC14BFB203BCD2919DF8FC1FF
:10150000BBF9823AFA2A75E03BC12BF8DA39212C73
:10151000D5E1F2C09CF62A39412D3AE3B2C00FF56D
:1015200071385A2EA3E47CC084F3AF376B2F11E6D9
:101530004FC0FBF1E536763083E72DC074F01236EC
:101540007931F8E814C0EFEE3635743271EA05C02F
:101550006CED53346733EDEB00C0EDEB6733533480
:101560006CED05C071EA74323635EFEE14C0F8E860
:101570007931123674F02DC083E77630E536FBF111
:101580004FC011E66B2FAF3784F37CC0A3E45A2E13
:1015900071380FF5B2C03AE3412D2A399CF6F2C0FA
:1015A000D5E1212CDA392BF83BC175E0FA2A823AD1
:1015B000BBF98FC119DFCD29203B4BFBECC1C3DD4B
:1015C0009928B63BDDFC52C272DC5F27423C6EFEBE
:1015D000C2C226DB1F26C53C00003BC3E1D9DA248A
:1015E0003E3D9201BEC3A1D88E23AE3D23034AC423
:1015F00067D73D22143EB504E0C433D6E720713EE0
:1016000045067EC506D58B1FC53ED50726C6DFD34A
:101610002B1E0E3F6409D6C6BFD2C61C4E3FF10A30
:101620008FC7A6D15D1B843F7C0C51C895D0EF19A4
:10163000B13F050E1BC98ACF7D18D33F8C0FEEC971
:1016400087CE0817EC3F1111CACA8CCD8F15FB3F0E
:101650009412ADCB99CC13140040131499CCADCB9C
:101660009412FB3F8F158CCDCACA1111EC3F08179D
:1016700087CEEEC98C0FD33F7D188ACF1BC9050ECC
:10168000B13FEF1995D051C87C0C843F5D1BA6D1AA
:101690008FC7F10A4E3FC61CBFD2D6C664090E3FA3
:1016A0002B1EDFD326C6D507C53E8B1F06D57EC5AC
:1016B0004506713EE72033D6E0C4B504143E3D2212
:1016C00067D74AC42303AE3D8E23A1D8BEC392017F
:1016D0003E3DDA24E1D93BC30000C53C1F2626DB92
:1016E000C2C26EFE423C5F2772DC52C2DDFCB63BDA
:1016F0009928C3DDECC14BFB203BCD2919DF8FC1FD
:10170000BBF9823AFA2A75E03BC12BF8DA39212C71
:10171000D5E1F2C09CF62A39412D3AE3B2C00FF56B
:1017200071385A2EA3E47CC084F3AF376B2F11E6D7
:101730004FC0FBF1E536763083E72DC074F01236EA
:101740007931F8E814C0EFEE3635743271EA05C02D
:101750006CED53346733EDEB00C0EDEB673353347E
:101760006CED05C071EA74323635EFEE14C0F8E85E
:101770007931123674F02DC083E77630E536FBF10F
:101780004FC011E66B2FAF3784F37CC0A3E45A2E11
:1017900071380FF5B2C03AE3412D2A399CF6F2C0F8
:1017A000D5E1212CDA392BF83BC175E0FA2A823ACF
:1017B000BBF98FC119DFCD29203B4BFBECC1C3DD49
:1017C0009928B63BDDFC52C272DC5F27423C6EFEBC
:1017D000C2C226DB1F26C53C00003BC3E1D9DA2488
:1017E0003E3D9201BEC3A1D88E23AE3D23034AC421
:1017F00067D73D22143EB504E0C433D6E720713EDE
:1018000045067EC506D58B1FC53ED50726C6DFD348
:101810002B1E0E3F6409D6C6BFD2C61C4E3FF10A2E
:101820008FC7A6D15D1B843F7C0C51C895D0EF19A2
:10183000B13F050E1BC98ACF7D18D33F8C0FEEC96F
:1018400087CE0817EC3F1111CACA8CCD8F15FB3F0C
:101850009412ADCB99CC13140040131499CCADCB9A
:101860009412FB3F8F158CCDCACA1111EC3F08179B
:1018700087CEEEC98C0FD33F7D188ACF1BC9050ECA
:10188000B13FEF1995D051C87C0C843F5D1BA6D1A8
:101890008FC7F10A4E3FC61CBFD2D6C664090E3FA1
:1018A0002B1EDFD326C6D507C53E8B1F06D57EC5AA
:1018B0004506713EE72033D6E0C4B504143E3D2210
:1018C00067D74AC42303AE3D8E23A1D8BEC392017D
:1018D0003E3DDA24E1D93BC3EC180108F0180108B9
:1018E00001000001C0070108CC0701080104201D08
:1018F0000E0913180000000000000000010203049C
:1019000006070809400203084C02030858020308AE
:10191000600203086C020308740203080000203B05
:10192000BFD283E7004083E7BFD2203B0000E0C482
:10193000412D7D1800C07D18412DE0C40000203BE2
:10194000BFD283E7004083E7BFD2203B0000E0C462
:10195000412D7D1800C07D18412DE0C40000203BC2
:10196000BFD283E7004083E7BFD2203B0000E0C442
:10197000412D7D1800C07D18412DE0C40000203BA2
:10198000BFD283E7004083E7BFD2203B0000E0C422
:10199000412D7D1800C07D18412DE0C40000203B82
:1019A000BFD283E7004083E7BFD2203B0000E0C402
:1019B000412D7D1800C07D18412DE0C40000203B62
:1019C000BFD283E7004083E7BFD2203B0000E0C4E2
:1019D000412D7D1800C07D18412DE0C40000203B42
:1019E000BFD283E7004083E7BFD2203B0000E0C4C2
:1019F000412D7D1800C07D18412DE0C40000203B22
:101A0000BFD283E7004083E7BFD2203B0000E0C4A1
:101A1000412D7D1800C07D18412DE0C40000203B01
:101A2000BFD283E7004083E7BFD2203B0000E0C481
:101A3000412D7D1800C07D18412DE0C40000203BE1
:101A4000BFD283E7004083E7BFD2203B0000E0C461
:101A5000412D7D1800C07D18412DE0C40000203BC1
:101A6000BFD283E7004083E7BFD2203B0000E0C441
:101A7000412D7D1800C07D18412DE0C40000203BA1
:101A8000BFD283E7004083E7BFD2203B0000E0C421
:101A9000412D7D1800C07D18412DE0C40000203B81
:101AA000BFD283E7004083E7BFD2203B0000E0C401
:101AB000412D7D1800C07D18412DE0C40000203B61
:101AC000BFD283E7004083E7BFD2203B0000E0C4E1
:101AD000412D7D1800C07D18412DE0C40000203B41
:101AE000BFD283E7004083E7BFD2203B0000E0C4C1
:101AF000412D7D1800C07D18412DE0C40000203B21
:101B0000BFD283E7004083E7BFD2203B0000E0C4A0
:101B1000412D7D1800C07D18412DE0C40000203B00
:101B2000BFD283E7004083E7BFD2203B0000E0C480
:101B3000412D7D1800C07D18412DE0C40000203BE0
:101B4000BFD283E7004083E7BFD2203B0000E0C460
:101B5000412D7D1800C07D18412DE0C40000203BC0
:101B6000BFD283E7004083E7BFD2203B0000E0C440
:101B7000412D7D1800C07D18412DE0C40000203BA0
:101B8000BFD283E7004083E7BFD2203B0000E0C420
:101B9000412D7D1800C07D18412DE0C40000203B80
:101BA000BFD283E7004083E7BFD2203B0000E0C400
:101BB000412D7D1800C07D18412DE0C40000203B60
:101BC000BFD283E7004083E7BFD2203B0000E0C4E0
:101BD000412D7D1800C07D18412DE0C40000203B40
:101BE000BFD283E7004083E7BFD2203B0000E0C4C0
:101BF000412D7D1800C07D18412DE0C40000203B20
:101C0000BFD283E7004083E7BFD2203B0000E0C49F
:101C1000412D7D1800C07D18412DE0C40000203BFF
:101C2000BFD283E7004083E7BFD2203B0000E0C47F
:101C3000412D7D1800C07D18412DE0C40000203BDF
